:020000040000FA
:040000006FD00400B9
:101000006F00106A00000000000000009020002027
:10101000A4220020A9BDF9F55C23002000000000F7
:10102000000000005C230020902000200000000051
:101030000000000090200020000000009020002010
:101040000000000090200020902000209020002030
:101050009020002090200020142E00204A24002000
:10106000000000009020002090200020F0230020AD
:1010700090200020C22300209020002090200020FB
:101080009020002090200020902000209020002020
:101090009020002001A04111B7170040985F3AC688
:1010A000945F3247E39CE6FE3245410182800111A4
:1010B00013078008F337078093F787083EC20100C3
:1010C0000100B7170040930570052380B70413068D
:1010D00080FA2380C7040100010083C6B70493F699
:1010E000F60DA385D704238007049246F3A6068055
:1010F0000100010093760502D5CEF336078093F602
:10110000860836C4010001002380B7042380C70489
:1011100001000100B70614007D89558D88C70100C4
:1011200001000100010023800704A246F3A6068007
:101130000100010073370780137787083AC6010062
:1011400001002380B7042380C704010001000100CF
:1011500001003727004093061005A303D7802380A2
:101160000704B247F3A70780010001009307800836
:10117000F3B7078093F787083ECE01000100B71749
:101180000040130770052380E704130780FA2380CB
:10119000E7040100010003C7B70413670708A3852C
:1011A000E70423800704F247F3A70780010001004A
:1011B0000561828093760504BDC6F336078093F6F9
:1011C000860836C8010001002380B7042380C704C5
:1011D00001000100B7061400938606047D89558D31
:1011E00088C7010001000100010023800704C246F6
:1011F000F3A6068001000100733707801377870884
:101200003ACA010001002380B7042380C70401000B
:1012100001003727004093062005A303D7802380D1
:101220000704D24781B773370780137787083ACC12
:10123000010001002380B7042380C70401000100DE
:1012400098471367070C98C723800704E24719BF24
:101250000111814601468145114506CE19239307A8
:101260008008F3B7078093F787083EC601000100A6
:10127000B7170040130770052380E704130780FAAF
:101280002380E7040100010003C767041367170008
:101290002383E70423800704B247F3A707800100F4
:1012A0000100F2400561828041118146014681457D
:1012B0001145452913078008F337078093F78708FE
:1012C0003EC401000100B7170040130670052380DB
:1012D000C704930680FA2380D70401000100FD555E
:1012E0002396B70223800704A245F3A505800100D9
:1012F000010073370780137787083AC601000100A1
:101300002380C7042380D7040100010003C76704BA
:10131000136717002383E70423800704B247F3A76A
:1013200007800100010001A0BD473305F50201005F
:101330007D1575FD8280411122C426C206C6AA848D
:10134000014463179400B2402244924441018280D8
:1013500005041305803E4204C13F4180DDB7000013
:101360009305000273A04580824573901534924026
:101370002242B2424243D2436244F2440255925561
:101380002256B2564257D2576258F25806499649E9
:10139000264AB64A464BD64B664CF64C065D965DE1
:1013A000265EB65E465FD65F09617300203041114C
:1013B000B7170040985F3AC6945F3247E39CE6FE59
:1013C000324541018280B71700401307000323888C
:1013D000E702854723AAF19C73002030411122C403
:1013E00006C637040020975000E0E780400F1C40FD
:1013F0008297D5BF37370040834747009146BD8B62
:101400006389D70099466394D70083475740730098
:1014100020309736000083C6A61C93871600173627
:101420000000230FF61A03478700973700009387C1
:10143000270BB6972380E700B7E70400BC4F0946A7
:101440008945171500000345A5E48297C9B7B787FA
:10145000004003C76700098B6309071003C77700C3
:101460009306000313770703630DD70817380000AE
:101470000348985217360000130646510547B30635
:1014800006012380E60083C57700173700001307A5
:101490006750429793F5F50F2300B70003C5870007
:1014A000973500009385C54EC2951375F50F2380BF
:1014B000A5000347070089451377F703630CB70CB2
:1014C00063E7E50A6306071A8545630CB712973789
:1014D000000083C7774C3307F600034707001377F4
:1014E000F70F19CB850793F7F70F0D476363F71ACB
:1014F00017370000A302F74AB78700400947238344
:10150000E700B787004083C77700E207E18763DE23
:1015100007049737000083C73748173700001307C1
:10152000E7463E9785462300D7001737000013078C
:1015300067463E97930600032300D7001737000045
:10154000130707453E97A14685072300D70093F769
:10155000F70F0D476364F71417370000A30EF74227
:10156000B787004009472383E700730020309306C4
:1015700010026300D70E930620026305D706930678
:101580000002E316D7F403C727021377C70F1367C8
:101590002700D5A803C767001377070465CB03C7E7
:1015A000A702173800001308E81F173500001305BD
:1015B0002517134707082385E70203C7A7021377F8
:1015C000370F136787002385E7028147130700045D
:1015D000B305F5008C41B306F80091078CC2E3997E
:1015E000E7FEF5B503C7A702134707042385E70203
:1015F00003C7A7021377C70F136727002385E702E6
:10160000F9B503C767001377070449C303C7670227
:10161000173800001308C80C17350000130505041F
:10162000134707082383E70203C767021377370FBF
:10163000136787002383E702814713070004B3057C
:10164000F5008C41B306F80091078CC2E399E7FEE0
:10165000BDBD03C76702134707042383E70203C71F
:1016600067021377C70F136727002383E70285B547
:1016700003C767001377070411CB03C7270213774B
:10168000370F136787002381E70291B52380060097
:101690003DBD97370000A3810730B9BD97370000E3
:1016A000A38C072E75BD2303048015472303E48014
:1016B00001002302A480828083076480E3CE07FEBA
:1016C00023030480828083076480E3CE07FE034502
:1016D0004480828083076480E3CE07FE2302A480D7
:1016E0008280411126C44AC24EC006C61377F50B4C
:1016F000AD47AA892E8995446306F70019456537D9
:10170000653F8D444E854537FD59FD14639834017E
:10171000B240A24412498249410182801355090115
:101720001375F50F453F2209CDB7011126CC06CE22
:10173000B704080051371545BD37713769372AC6D8
:10174000A53F32459377150089EB13651500137596
:10175000F50FF240E24405618280FD14E9FC014589
:10176000CDBF397126DC4ADA4ED852D656D45AD279
:101770005ED006DE62CE66CCB7E700E07D5783AA76
:10178000070022C603AA470023A0E71823A2E718F0
:10179000B7170040130770052380E704130780FA8A
:1017A0002380E70483C74704930B75FFB684E207E1
:1017B00093FBFB0F8546AA892E8B32893724004084
:1017C000E187015763FA76016308D500894613075C
:1017D00000026313D5000157D98F93F7F70FB71C99
:1017E00000402382FC0411472303E4801305F00F1B
:1017F0005D3D094CD135636D7C11B7050700DA9565
:1018000037870700795563F2E504B3879500636E67
:10181000F702370B0800A94733EB65016399F90616
:1018200089E48144513D26850DA0DA850945553D61
:1018300005090345F9FFFD14050B693D81C4937744
:10184000FB0FFDF7DD3569FD7D55B7170040130728
:1018500070052380E704130780FA2380E70403C799
:101860004704418B2382E704F250B7E700E023A04E
:10187000571123A24711E25432445259C259325AE5
:10188000A25A125B825B724CE24C21618280A547B6
:101890006395F90685691309F00FB3069900B374CF
:1018A0002B01B6941349F9FFB3749900856B337912
:1018B0006901416B9387F9FFB3F7270199E363FC53
:1018C000340193D94900C147E3E637FF99BF056961
:1018D000C1697D19D9B71305800D638869011305A6
:1018E00000026384790113051008CA85DD3B353D8C
:1018F00021DD4E99B3843441D9B7DA852D45D533EE
:10190000CA94E30099F205097D3BA30FA9FED5BF58
:101910009387F9FF93F7F70F6361FC0C83C71C04EF
:1019200013073008631FF70437070800636BEB04E5
:10193000B3079B00B706100063F5D704334BEB00E9
:1019400089476393F9068980D549E38C04ECDA85ED
:101950000945413B11090327C9FF91472320E48032
:1019600003076480E34E07FE23033481FD17EDFB7C
:10197000FD14110B81C49377FB0FE9FF7D3371F5E3
:10198000E1B5B717004003C75704B707080013773E
:10199000070219E3B78707007955E378FBEA3307B5
:1019A0009B00E3FFE7F855B58547E382F9F2DA8556
:1019B0002D45053B9389F4FFE38504E6293393F72E
:1019C000390091EB8326048003270900930749001F
:1019D000E39AE6E43E89CE84F1BFB5476396F90009
:1019E0001305900BC93135BDB1471305B00AE38B20
:1019F000F9FE99476391F904B7050800B365BB0088
:101A00002D45C53181448D4BA149753963967401CB
:101A1000832704802320F9008504E39834FF83277B
:101A2000048013172B01635507002312F900D5BB5F
:101A30002322F900FDB39D476399F90281451305FF
:101A4000B0044531BD442320090023220900FD597B
:101A50009D3993F77400CA9703C70700FD14398DA9
:101A60002380A700E39634FF6DBBA1476392F9047E
:101A70006D398144630D0B008D479304C0036308E7
:101A8000FB009304000563048B0193044004137569
:101A9000C507E30895D8194539313939054521314C
:101AA00026850D3909453D314931E31C05D669BB11
:101AB00091476399F90013056006F536F53E130565
:101AC00090090DB7E38F09D4F154A9BBBD66014756
:101AD0001736000013068609938606A685458347B8
:101AE000060093F7F70F91C382800507E3F9E6FE3E
:101AF00097370000238CB706DDB77D166206618636
:101B000093178601E18763D407000145828093170C
:101B100026003307F500AE9718439C4363E7E700C0
:101B20007D16E37FF7FC7D55828005458280FD159B
:101B3000E205E18513978501618793F7F50F634807
:101B40000700FD15139725002A97584365D713857D
:101B500017006205618582803308B5021C4283A8A4
:101B60000600B335B502C29733B50701AE98469566
:101B700085486367B5006394A50063E30701814866
:101B80000C43C6950CC388C21CC282808147139740
:101B9000870161876343B7008280139727002A97E4
:101BA000232007008507E5B7814701479396870102
:101BB000E18663C5B600133517008280939627002F
:101BC000AA9694428507558FD5B793D755408A0773
:101BD000AA979C4305453315B5007D8D828017F388
:101BE000FFDFE702033B2A84993705C593172500D9
:101BF0003E940327C4FF814711EB7D1516053E95E2
:101C00004205418517F3FFDF6700E33A0583850747
:101C1000E5B70145C5BF81471397870161876343D6
:101C2000C700828013972700B386E50094422A9765
:101C3000850714C3D5B77D166206618601479317E1
:101C40008601E18763D5070013351700828093175B
:101C50002600B306F500AE9794429C437D16B58FDF
:101C60005D8FF1BF8A05AA9501476363B500828045
:101C700083A6C5FFF11593D71600D98F9CC1139782
:101C8000F601E5B72A830148014701456343D700C0
:101C90008280B387050183A80700B30706019C4330
:101CA000C697AA976384F80033B517010507B308F0
:101CB0000301620723A0F80061871108C1BF2A83CE
:101CC00001478147014563C3D70082803388E5001F
:101CD00083280800330EE600032E0E003388A84048
:101CE0003308C8416384080133B508018507B30888
:101CF000E300E20723A00801E1871107E9B717F322
:101D0000FFDFE70203290111B286B2842E86AA857D
:101D10000A8575372A84A6850A857935333480008B
:101D2000060413351500018D056117F3FFDF670009
:101D3000832817F3FFDFE70243234111AA89AE8A04
:101D4000328BB68402C202C402C60144131C840151
:101D5000135C8C4163499C02939B1400FD1B054955
:101D6000138CF4FFF15C3304890162046184634DD8
:101D7000740592478E04CE9423AEF4FE410117F30E
:101D8000FFDF6700032213192400B30B2B01014A64
:101D900093172A00D69783A50B0088437800340058
:101DA00050005D3B050A93178A01E187F11BE3515F
:101DB000FCFE92474E9905042320F900A2473EC23B
:101DC000B24702C63EC459B7131A8901135A8A4151
:101DD000131D240093178A01E18763CF9700924770
:101DE0000A044E941CC0A24705091379F90F3EC29C
:101DF000B24702C63EC485BFB3079A0313152A0033
:101E000056950841780034005000050AEA97DA97A1
:101E10008C439933C1B70000197106C212C416C6AB
:101E20001AC81ECA22CC26CE2AD02ED232D436D6FA
:101E30003AD83EDA42DC46DECAC0CEC2D2C4D6C6EA
:101E4000DAC8DECAE2CCE6CEEAD0EED2F2D4F6D6DA
:101E5000FAD8FEDA9385C19C8841E70005009240DC
:101E60002242B2424243D2436244F2440255925566
:101E70002256B2564257D2576258F25806499649EE
:101E8000264AB64A464BD64B664CF64C065D965DE6
:101E9000265EB65E465FD65F0961730020300000A3
:101EA00097210020938181E917510020130181952A
:101EB00017F5FFFF13054515970500209385851439
:101EC000171600201306C6FD63FAC500832205001D
:101ED00023A0550011059105E3EAC5FE17C50100D1
:101EE0001305C5D1971500209385C5FB1386818006
:101EF00063FAC5008322050023A055001105910552
:101F0000E3EAC5FE1385818097450020938505127D
:101F10006377B500232005001105E36DB5FEFD4292
:101F2000739002BC8D4273904280B722000093826E
:101F3000828873900230970200209382A20C93E271
:101F400032007390523097420000938202E87390FF
:101F500012346FC0E40A73002030397101436EC639
:101F600019A0397141536AC866CA62CC5ECE19A005
:101F7000397101535AD056D252D44ED64AD826DAA5
:101F800022DC06DE33016140828241114AC026C252
:101F900022C406C68282B24D4101024D924C224CAF
:101FA000B24B4101024B924A224AB24941010249D5
:101FB00092442244B240410182803D432A876373A8
:101FC000C3029377F700BDEFADE5937606FF3D8A38
:101FD000BA960CC34CC30CC74CC74107E36BD7FE82
:101FE00011E28280B306C3408A06970200009696EB
:101FF0006780A6002307B700A306B7002306B70033
:10200000A305B7002305B700A304B7002304B70056
:10201000A303B7002303B700A302B7002302B7004E
:10202000A301B7002301B700A300B7002300B70046
:10203000828093F5F50F93968500D58D93960501D3
:10204000D58D61B7939627009702000096968682F9
:10205000E78086FA9680C1171D8F3E96E374C3F819
:10206000A5B73367B500FD530D8B79E7B7877F7F41
:102070009387F7F710419441B372F6003363F6008B
:10208000BE92B3E262006397720C6318D6065041A9
:10209000D441B372F6003363F600BE92B3E262003D
:1020A0006398720A631BD60410459445B372F60018
:1020B0003363F600BE92B3E262006391720A631E5C
:1020C000D6025045D445B372F6003363F600BE9293
:1020D000B3E26200639A72086311D6021049944910
:1020E000B372F6003363F600BE92B3E2620063930C
:1020F00072085105D105E30FD6F613170601939721
:102100000601631CF7001357060193D70601330538
:10211000F7409375F50F91E982804183C1833305C0
:10212000F7409375F50F91E182801377F70F93F7DE
:10213000F70F3305F74082800346050083C605008C
:10214000050585056313D60065FA3305D640828000
:1021500011059105E312D6FE014582802105A105F6
:10216000E31CD6FC014582803105B105E316D6FC9F
:10217000014582804105C105E310D6FC01458280FE
:10218000B717004003C777051377E70FA38BE70462
:10219000130700F8A38DE7043D47238CE7041307DA
:1021A0005003A38CE70403C7A7051377D70F238D2C
:1021B000E7048280B717004003C7E7020D89411189
:1021C0001377C70F498F93068008F3B6068093F6FE
:1021D000860836C601000100930670052380D704E7
:1021E000930680FA2380D704010001002387E702C9
:1021F00023800704B247F3A70780010001004101D3
:10220000828041112A83014E930E407E130F0019E4
:10221000930F400663E56E129308001913034006FE
:10222000B3781503854E0D4FA14F337365020D89A9
:102230001335150063EFBE121308F6FF7946729846
:102240004208135808013307C70213D61700BE0708
:1022500032976146B3F6C60213068070B386C60293
:102260003697A166F58F42075D8FB716004083C78A
:10227000F60293F70708A303F1000346710083C732
:10228000F60293F70708E394C7FE83477100B71679
:10229000004093F7F70F6388071293078008F3B79E
:1022A000078093F787083EC401000100B71700407C
:1022B000930670052380D704930680FA2380D70401
:1022C0000100010023AA070383C6170393E606084B
:1022D000A388D70223800704A247F3A70780010041
:1022E00001001166B71700407D16D45BC85F938567
:1022F0004703A98EF18EF5FA93068008F3B606809F
:1023000093F6860836C60100010093067005238007
:10231000D704930680FA2380D7040100010098C1F6
:1023200003C7170313670704A388E7022380070482
:10233000B247F3A7078001000100410182807D13AD
:102340003368E3039308E016630E08003368F30371
:102350009308D016630808009378330093B81800E8
:102360009388D81633081E01131E0801135E0E0150
:1023700055B56393E5030548638608000148630388
:1023800003002A8871087298FD15131E0801C20502
:10239000135E0E01C18179BD13F8150063F4BF000F
:1023A0007908D5B713381800E5BF83C7F60293F74D
:1023B0000708A303F1000346710083C7F60293F7F1
:1023C0000708E394C7FE8347710093F7F70FF1DF27
:1023D000E9B531714AD966CB06DF22DD26DB4ED75F
:1023E00052D556D35AD15ECF62CD6AC96EC7AA8C78
:1023F00002D8EF00901C2A8993078008F3B7078062
:1024000093F787083EDA01000100B7170040130771
:1024100070052380E704130780FA2380E704010096
:10242000010003C7F7021377770FA387E70203C7FB
:10243000F70213678700A387E70223800704D257B8
:10244000F3A70780010001000545AD33130780C1E4
:102450003347E902116A93070AE893065002BD69FF
:10246000930BA004814A014B130480089304700568
:102470007D1AB347F9023307D7023EC0FD873ECC31
:10248000938709A69309803E3347F7023AC27D87B6
:102490003AC4334739038549B399990193D93940EF
:1024A000B306D702B30B7703B3C6F602B3CBFB0276
:1024B00036C6FD8636C893D6FB4136CEB7460F00EA
:1024C000938606243349D9028566938606FAB39625
:1024D0009601B389E902130760553309D9029306BF
:1024E0000010B389E9023349D902B3C9F90293163E
:1024F000390036CA37190040FD8636D0930D0904DD
:1025000093D7F9413ED2F336048093F6860836DC41
:1025100001000100930770052380FD00930680FAF7
:102520002380DD00010001008346390593F6860F04
:10253000A309D9048346390593E61600A309D904F3
:1025400023800D00E256F3A6068001000100130C63
:1025500080FA116DF336048093F6860836DE0100AA
:102560000100930770052380FD0023808D01010089
:10257000010083463905216693E60602A309D904C2
:1025800083560905B3E6A6012318D9048356090525
:10259000D18E2318D90423800D00F256F3A60680AD
:1025A000010001008346390593F60602638A061886
:1025B00003463905218A6DDE0818EF0010047336D2
:1025C000048013768608B2C20100010023809D00BA
:1025D00023808D0101000100B717004003C63705B5
:1025E0001376F60DA389C70403C6370513660602E2
:1025F000A389C704835609052166B3E6A6012318FB
:10260000D90483560905D18E2318D90423800D00DF
:102610009646F3A60680010001008346390593F62D
:1026200006026386061483463905A18AEDFE9700EB
:102630000020E78040A6AA8636D497000020E780D5
:1026400080A5A256E30AD5FE835609054255B3E696
:10265000A6012318D904C12783463905A18AEDDED6
:10266000035609058346290582473376CA00B30617
:10267000DA0293D5F641B296B388F640E24733B812
:10268000C6002E983308F840A247B3B616013308A7
:10269000D84063C70701631DF800924763FA17012A
:1026A000C247634DF80E63950701B24763E8F80E21
:1026B000894663E7660FF2469315180013D3F801B5
:1026C0005E8613951800B365B30042D646D4EF700A
:1026D000310D3258050B137BFB0F6347000163126A
:1026E0000838A258638F083613081500B336A800BF
:1026F000B69513D6F5013298B336C800AE96135886
:102700001800FE06B3E606017336048013768608C9
:10271000B2C60100010023809D0023808D010100CD
:1027200001000356C902B296C206C1822316D9021D
:1027300023800D00B646F3A606800100010019BDF6
:10274000F336048093F68608B6C0010001002380AA
:102750009D0023808D01010001008346390593E629
:102760000602A309D90423800D00864605BDF33671
:10277000048093F68608B6C40100010023809D0002
:1027800023808D01010001008346390593E606028E
:10279000A309D90423800D00A646A5BDE30D0BF0C7
:1027A000F336048093F68608B6C80100010093064C
:1027B00080FA23809D002380DD0001000100834614
:1027C000390593F5FC0F93F6860FA309D9048346C8
:1027D0003905CD8EA309D90423800D00C646F3A682
:1027E000068001000100130580FA034639059306AF
:1027F00039051D8A6314962973360480137686087A
:10280000B2CC01000100130680FA23809D002380D2
:10281000CD000100010003C606001376F60D2380EB
:10282000C60003C60600136606022380C600835650
:1028300009051166D18E2318D9048356090521662E
:10284000D18E2318D90423800D00E646F3A6068016
:1028500001000100130680FA8346390593F606024B
:102860006388062483463905130C3905A18AFDDAED
:1028700008186123F336048093F68608B6D0010069
:102880000100930680FA23809D002380DD00010073
:10289000010083460C00116693F6F60D2300DC0060
:1028A00083460C0093E606022300DC0083560905EC
:1028B000D18E2318D904835609052166D18E231899
:1028C000D90423800D008656F3A60680010001007E
:1028D000130680FA8346390593F6060263850620BF
:1028E00083463905A18AEDFE97F0FF1FE780A07AA5
:1028F0002A8C97F0FF1FE780007AE30C85FF835650
:10290000090511664255D18E2318D904292383461F
:10291000390513063905A18AFDDAF336048093F6EA
:102920008608B6D401000100930680FA23809D003A
:102930002380DD00010001008346060093F6F60DBA
:102940002300D60023800D00A656F3A606800100C2
:1029500001008356090503462905D247B376DA00FC
:102960003306CA021305800C9355F6413696330D93
:10297000F6408257333CD6002E9C3336A601330CEA
:10298000FC40330CCC403308850392564E86B33559
:10299000A5033305A503C295EF70816063468001EE
:1029A000631E0C16630C0D16130615003335A600B6
:1029B0002E959356F5013696B335D600AA95939683
:1029C000F50105828585D18E6346B000639D051AA9
:1029D000638B061A0356C90215823305D6003336B7
:1029E000C500B2956348B000639105241306F00F4B
:1029F000637DA622894663F3561593078008F3B7D3
:102A0000078093F78708BED6010001003717004002
:102A1000930770052300F704930780FA2300F70457
:102A2000010001008356C70289678117D58FC2074D
:102A3000C1832316F70223000704B657F3A70780C4
:102A400001000100FA506A54DA544A59BA592A5A14
:102A50009A5A0A5BFA4B6A4CDA4C4A4DBA4D2961D4
:102A600082801308F5FF3335A800FD152E95135607
:102A7000F5013298B336C800AA9651B1F3360480F6
:102A800093F68608B6CA0100010023809D002380CA
:102A9000AD000100010083463905CD8EA309D9049C
:102AA00023800D00D646F3A606800100010035BB49
:102AB000F336048093F68608B6CE01000100238029
:102AC0009D002380CD00010001008346390593E677
:102AD0000602A309D90423800D00F646F3A606805A
:102AE0000100010095BBF336048093F68608B6D248
:102AF0000100010023809D002380CD000100010022
:102B00008346390593E60602A309D90423800D0004
:102B10009656F3A60680010001006DBB9306F5FFF3
:102B200033B5A600FD152E959355F501AE96B3B5B8
:102B3000B600AA951396F501858269B5F33604802F
:102B400093F68608B6D801000100930680FA238028
:102B50009D002380DD00010001008356C902056647
:102B6000011693F6F60FD18EC206C1822316D90242
:102B700023800D00C656F3A6068001000100850AD9
:102B800093FAFA0F49B233E6B60045C20356C902BA
:102B90003305D0403338A000B305B040B3850541BC
:102BA00015826345B000D1E16371A608894663F0E0
:102BB000560593078008F3B7078093F78708BEDAB6
:102BC00001000100B7170040130770052380E704D8
:102BD000130780FA2380E7040100010003D7C7022E
:102BE0007D8B2396E70223800704D65781BDF336F9
:102BF000048093F68608B6DC01000100930680FA93
:102C000023809D002380DD00010001008356C9025E
:102C10000566011693F6F60FD18EC206C182231601
:102C2000D90223800D00E656B9B793078008F3B7A1
:102C3000078093F78708BEDE0100010037170040C8
:102C4000930770052300F704930780FA2300F70425
:102C5000010001000356C70293975600B297C207BE
:102C6000C1832316F70223000704F657C1BB91471F
:102C700063EEB70217970100130787028A05BA951A
:102C80009C41BA978287B717004003A7470B1345AB
:102C9000F5FF698F23AAE70A03A7070B698F23A80B
:102CA000E70A03A7070A798D23A0A70A8280B7172E
:102CB000004083A6470B1347F5FFF98E23AAD70AD6
:102CC00083A6070B558D23A8A70A83A6070A758F2D
:102CD00023A0E70A8280B717004003A7470B498F5C
:102CE00023AAE70A03A7070B1345F5FF45BFB7174C
:102CF000004083A6470B1347F5FF758F23AAE70A09
:102D000003A7070A598D4DB7B717004003A7470B14
:102D1000498FEDB7914763EEB7021797010013078C
:102D200067F98A05BA959C41BA978287B717004020
:102D300003A7470D1345F5FF698F23AAE70C03A7E7
:102D4000070D698F23A8E70C03A7070C798D23A033
:102D5000A70C8280B717004083A6470D1347F5FFE5
:102D6000F98E23AAD70C83A6070D558D23A8A70C8F
:102D700083A6070C758F23A0E70C8280B71700404D
:102D800003A7470D498F23AAE70C03A7070D134597
:102D9000F5FF45BFB717004083A6470D1347F5FF62
:102DA000758F23AAE70C03A7070C598D4DB7B717EA
:102DB000004003A7470D498FEDB7B717004088477C
:102DC000420541819377050491EB9377F5013755DF
:102DD000E801130505803345F50282809377050CE1
:102DE000130700046397E7009377F50137459C1CB0
:102DF000CDB72165130505D0828037E700E01C437D
:102E00005443A183E206D58F1CC1FD572320F71838
:102E10002322F718828013178500B7E700E023A06C
:102E2000E710618123A2A7108280B7F700E08847EE
:102E3000CC478280814737370040A14663C4C70032
:102E4000328582800345B740E38EA6FE3385F500C8
:102E50000345050085072304A740CDB79707002049
:102E6000938747049C43173700201307271C3E9580
:102E7000636EE500173700201307C7786368A70063
:102E8000170700202320A7023E858280FD57EDBF53
:102E90008280411122C406C62A8405372947B30718
:102EA000E502B2408D83B3D7870222449507B3D79A
:102EB000E70237370040C207C1832316F7004101FC
:102EC0008280716541111305052006C6D937B737D1
:102ED0000040130770F82381E7000D47A381E70046
:102EE00013070004A380E70005472387E700B240EB
:102EF0004101828037370040834727001A0593F746
:102F0000F703C98F93F7F70F2301F7008280B737D4
:102F1000004003C7170019C9D98DA380B70003C7A4
:102F20000700136787002380E700828093C5F5FFC1
:102F3000F98DA380B7008280AE872A87B73600401C
:102F400021463738004091E3A1B783C8B600E30CAF
:102F500016FF05078348F7FFFD17C2072304180172
:102F6000C183D5B7411122C406C62A84B935294781
:102F7000B307E502B2408D83B3D787022244950799
:102F8000B3D7E70237370040C207C1832316F740A3
:102F900041018280716541111305052006C6D937AC
:102FA000B7370040130770F82381E7400D47A3812E
:102FB000E74013070004A380E74005472387E74065
:102FC000B24041018280CC41411106C6328503C620
:102FD000150083C5050022064D8E42068D6541868B
:102FE000138875A2630A0611634BC804138845A2AF
:102FF000630E060B634AC800938535A26301B608C9
:1030000023900600294679A8138855A26303060D6C
:10301000938565A2E316B6FE8D451D4663E4E5087B
:103020001146198E63F3C7003E86B7E7040023906C
:10303000C600FC4797950100938505CA8DA01388AB
:1030400095A263010611634C060D1388A5A2630EB9
:103050000611938505A5E315B6FA99451D4663E368
:10306000E504198E63F3C7003E86B7E7040023909A
:10307000C600FC4797050020938505ED0DA09D45F2
:103080001D4663E1E5022146198E63F3C7003E86C3
:10309000B7E70400FC472390C60093850181BA95E9
:1030A00082970146B240328541018280AD451D467E
:1030B000E3EAE5FE3146198E63F3C7003E86B7E7C3
:1030C00004002390C600FC4797950100938545C3F3
:1030D000F9B7B1451D46E3E7E5FC3546198E63F3C4
:1030E000C7003E86B7E704002390C600FC479795CB
:1030F00001009385E5C165B78D451D46E3E4E5FA1A
:103100001146198E63F3C7003E86B7E7040023908B
:10311000C600FC47979501009385C5BC49B78D450E
:103120001D46E3E1E5F81146198E63F3C7003E86BC
:10313000B7E704002390C600FC47979501009385EC
:10314000E5BEB1BFA5451D46E3EEE5F42946198E5F
:1031500063F3C7003E86B7E704002390C600FC4730
:10316000979501009385C5B81DBFB5451D46E3EB96
:10317000E5F23946198E63F3C7003E86B7E70400CF
:103180002390C600FC47979501009385E5B301BFE6
:10319000B7E7040003A30713970600209386C6D958
:1031A0004146A54517050020130505D002832D458E
:1031B0005DE703C505000947631FE50803A845004F
:1031C000411106C60347180032850346080022074E
:1031D0004168518F930828FE6307170563E9E800EB
:1031E00005186303070323900600294591A81306D9
:1031F00048FE630AC7041518E31707FF15463E8704
:10320000637BF600154701A8130600023E8763742E
:10321000F60013070002B7E704002390E600FC471E
:103220001316070111A83E8691C30546B7E70400AF
:10323000FC472390C6004206CC4541828297014557
:10324000B24041018280130600083E87E375F6FC18
:1032500013070008C9B723900600054582808280C5
:10326000416779176302E504411122C406C6854708
:103270002A84639DF500B7E7040022852244B2400A
:1032800003A387139385419B410102838947639977
:10329000F500B7E7040083A7070B8545829761DD3A
:1032A000B2402244410182808280797122D452CC82
:1032B0002E842A8A97950100938545A917950100C8
:1032C000130545AB06D63AC626D24AD0B684328913
:1032D0004ECEEF702118A68517950100130585AA1B
:1032E000EF7041172945EF70211B8347840093F746
:1032F0000702F1E383490400894705453247639497
:10330000F908544083C7160083C60600A207D58F6C
:10331000C166138616FE638CC7028D16638DD706B1
:103320008D66938626902945639FD704B7E70400EE
:10333000A285225403A34714B250F249A6864A86B6
:10334000925402595285624A8547456102832D4550
:103350001DEB93070002354563E79702B7E70400CA
:10336000FC47484413060002CA8582978149938727
:10337000019C9C43014581CB9C4391C74E85268689
:10338000CA8582970145B250225492540259F2499B
:10339000624A456182802D457DF79307700F354560
:1033A000E3E397FEB7E70400FC4748441306700FB9
:1033B000CA8582976DBF2145F9B7411122C437E410
:1033C00004008327841326C2AA84416506C6938518
:1033D000419B7D1582978327C40A170500001305BA
:1033E00065E88588829795C0032304132244B24080
:1033F0009244970600209386A6C64146C545170508
:1034000000201305E5B441010283B24022449244F6
:1034100001454101828009C523A0A19C014582800C
:103420004545828011476360A70A979601009386FD
:10343000A6900A0536951841411106C63697AE8703
:10344000B2850287130700026145639BE700B7E777
:103450000400FC4713060002138581818297014511
:10346000B2404101828005476145E39BE7FEB7E733
:103470000400FC47054613858183CDB71307700F01
:103480006145E39FE7FCB7E70400FC471306700FB4
:103490001385C183E1B7130700086145E392E7FC98
:1034A000B7E70400FC4713060008138541937DB776
:1034B00015476145E396E7FAB7E70400FC47154670
:1034C0001385819B61BF09458280411126C2B7E403
:1034D000040083A7C41322C44AC006C62E84938561
:1034E000419B2A898297058905C597070020938704
:1034F00027A683D7A70BA28503A3440D2310F400AE
:103500002244B24092444A85024901464101028365
:10351000B2402244924402494945410182802382BB
:10352000019C23A4019CB717004003A7070CB70612
:10353000C0FFFD16758F23A0E70C03A7070DB70684
:103540004000558F23A8E70C03A7070C3D9B23A041
:10355000E70C03A7070D1367070123A8E70C828078
:10356000B717004003A5470C83A7470C59811345A3
:103570001500C18B058999E31365250083C7419C1C
:10358000638CA7002382A19C01C99387819C03A31C
:103590000700630303000283828011456FE07FE32D
:1035A000411193962500AA852D4506C697F0FF1F69
:1035B000E780201BB240014541018280011122CCED
:1035C00006CE3714004026CA4AC84EC652C48344A9
:1035D0007405034AB4058349840503499405EFE063
:1035E0003FBA8347A40593F4F40F137AFA0F93E7D5
:1035F0001700230DF40493F9F90F1379F90FB71796
:10360000004003C7A705058B6DFF03D5C705A38D34
:103610004705238C3705A38C2705A38B9704F2401D
:103620006244D2444249B249224A05618280411132
:103630009397050122C406C626C2C1872E8463DC87
:103640000700B7E40400FC54829719C1BC54829768
:103650002165218D2DA093F7150013C5150085E375
:1036600093F7250095C3ED3DB7E70400BC4F130663
:10367000000A894503C5019D829713452400B24085
:1036800022449244410182809397250163D307022B
:10369000B7E4040083A7C41E82970137BC4C37F6F9
:1036A0000200130606E0896503C5019D829709653E
:1036B0004DB7939715010145E3D307FC178501002A
:1036C00013054574EF60D16DB7E70400BC4F1306D6
:1036D0000064916503C5019D829711659DBF2D71A1
:1036E000232A9110FD74E98C232C811023282111A9
:1036F000232631112A84AE893289930600100A8666
:10370000A6852D45232E111097F0FF1FE780600539
:1037100013154401B7E70400FC4751810A051396CD
:103720002900CA850A958297A685856601462545A2
:1037300097F0FF1FE780E0020A86A6859306001037
:10374000294597F0FF1FE780C0018320C1110324A2
:10375000811183244111032901118329C1101561AD
:103760008280B7F7070003C70701411106C622C4CC
:1037700026C24AC0A547631AF7009537B2402244D3
:103780009244024901454101828013942500AA8494
:103790003289A286AA850146254597F0FF1FE7805A
:1037A00040FCA2864A86A685294597F0FF1FE78040
:1037B00040FBE9B71D71A2CC37E404005C5C4858BB
:1037C00086CE4946978501009385455F829701E93A
:1037D000178501001305C55FEF60915C01A0B7F686
:1037E00000E0795798CAFD57DCCA0567B7E700E0E3
:1037F00023A0E7101306F00290C223A0E7180100EF
:10380000010037070020184713060004814523A64E
:10381000E19C4157A38AE7403C44080882979717E8
:1038200000209387678B3EC8856713870740231A5C
:10383000E1001D673ACC37070105130707103ACEA0
:103840009387B7D31307B00F2310E1022312F102BD
:10385000054797F7FFFF9387875D2301E1023ED875
:1038600017070000130707D497070000938747D571
:10387000B7F50700BAC23EDC170700001307A7EE32
:10388000970700009387A7D181463000E1051945CD
:10389000BAC43EDE97F0FF1FE780A0EC180881470E
:1038A000994630003E960346060085070507A30BA0
:1038B000C700E398D7FEC24791C703574101856708
:1038C0006373F70001A0B7E7040083A7470A08085D
:1038D0008297AA8501C9178501001305A550EF60DD
:1038E000713701A0F640664425618280411126C2ED
:1038F000B7E4040083A7040806C622C41705000025
:10390000130525D382971384019D2300A400312839
:10391000393103450400224403A38405B240924494
:1039200013060032896541010283797106D622D4DB
:1039300013078008F337078093F787083EC201001A
:103940000100B7170040930570052380B7041306E4
:1039500080FA2380C7040100010083C6F70293F6B2
:10396000A60FA387D702238007049246F3A60680FA
:103970000100010073370780137787083AC40100FC
:1039800001002380B7042380C7040100010003C79E
:10399000F70213672700A387E70223800704A247E3
:1039A000F3A70780010001000545EFE0BF80F53671
:1039B000014781468147054685451305407EEFE076
:1039C0005F8437E404003C44680051468145829797
:1039D000B707C0A83EC8B787E803938707D03ECA99
:1039E00097F7FF1F9387A79C3EC67C586800829775
:1039F000B250225445618280411197950100938510
:103A0000A5A6178501001305E53606C6EF609124CB
:103A100017950100130505BEEF60D123B24029457B
:103A200041016F607127411197950100938505A5AC
:103A3000178501001305053406C6EF60B1211795FF
:103A400001001305E5B9EF60F120B24029454101BD
:103A50006F609124411122C406C6834705002A8461
:103A60009DC397950100938525A717850100130530
:103A70006530EF60311E4C40179501001305C5CB32
:103A8000EF60511D1DA058411DE7979501009385DA
:103A9000A5A4178501001305E52DEF60B11B17954F
:103AA00001001305E5CAEF60F11A2244B24029452E
:103AB00041016F60711EA1679386D7036311D7021E
:103AC00097950100938545A1178501001305852A67
:103AD000EF60511817950100130585C8E9B7ED0788
:103AE000979501009385459F17850100130585284B
:103AF0006319F700EF60111617950100130585C7CC
:103B00005DB7EF6031154C4017950100130585C86E
:103B100085BF411197950100938585971785010011
:103B20001305452506C6EF60F112B2402945410153
:103B30006F609116797122D426D24AD02E842A89B8
:103B40008145B2844800714606D6EFE00FC797F76B
:103B5000FF1F9387A771DC4783D707002314210138
:103B60002313F100EF30705C9547A305F100930734
:103B7000401F3EC6FD572305A100230AF100EF3088
:103B8000106D2686A2854800EF30105DB250225499
:103B9000925402594561828097270020239107A4FF
:103BA00097270020238A0792B7E70400BC474111FA
:103BB00006C641468145138541288297EF10B05FC4
:103BC000EF10303F0145EF40406E03C7412A930795
:103BD000F00A631DF7009307F0F889451385412A21
:103BE0002382F12AA382012AEF407018EF40D029E6
:103BF00081453705040023A00128239E0126238F39
:103C00000126239401202396011E239D0126239A39
:103C10000128EF2020380145EF40B01D97950100A5
:103C200093858589178501001305C514EF609102FE
:103C300017950100130545BCEF60D101B24029453D
:103C400041016F607105411122C406C626C293F777
:103C500015002E846389070C814617F6FF1F130693
:103C6000265E854503D5811EEF90906605C5979524
:103C7000010093852585178501001305A50FEF60C9
:103C8000617D178501001305A526EF60A17C2945FC
:103C9000EF609100979501009385C582178501001B
:103CA0001305450DEF60017B178501001305852580
:103CB000EF60417A2945EF60217E17F5FF1F13055C
:103CC000E55A5C4505472390E700EF00C1769785EC
:103CD00001009385257F178501001305A509EF6075
:103CE00061771785010013052523EF60A17629452B
:103CF000EF60817A930710F82382F12A83D7411E5F
:103D0000A382F12A1385412AA18391452383F12AB5
:103D1000A383012AEF40B00513451400B2402244AA
:103D200092444101828093F72500C1C303D7C12784
:103D300035CB938601289442979701009387C7ADAE
:103D400003C6E127814513854128EF50B065AA8459
:103D500031C9978501009385A57D1785010013055D
:103D60006501EF60216FA685178501001305451CCD
:103D7000EF60416E2945EF602172239E0126930773
:103D800010F82382F12A83D7411EA382F12AA1834E
:103D90002383F12A91458D471385412AA383F12A74
:103DA000EF40E07C1345240095BF93F74500A1CF79
:103DB000978501009385C57717850100130585FB5D
:103DC000EF6041691785010013054518EF608168B0
:103DD0002945EF60616C930720F82382F12A83D78D
:103DE0008120A382F12AA1832383F12A8547A3831B
:103DF000F12AEF30D0451385412A9145EF402077D5
:103E00001345440021BF93F785009DCB97850100A2
:103E100093850572178501001305C5F5EF60816371
:103E2000178501001305C513EF60C1622945EF60D6
:103E3000A166239E0126EF50D06313458400F9BD8F
:103E400093F70501A1CF854503D58120EF20C12D32
:103E5000978501009385C56D17850100130585F1D0
:103E6000EF60415F178501001305C510EF60815EAB
:103E70002945EF606162930730F82382F12A83D7E6
:103E80008120A382F12A1385412AA1838D452383B2
:103E9000F12AEF40C06D1345040149B593F70502BF
:103EA000B1CF978501009385A5681785010013059B
:103EB00065ECEF60215A178501001305E50DEF60F1
:103EC00061592945EF60415D930740F82382F12A4B
:103ED00083D7C11EA382F12AA1832383F12A8547B8
:103EE000A383F12A2396011EEF3070361385412AF1
:103EF0009145EF40C067134504020DB593F70504E3
:103F0000D9CF978501009385A56217850100130518
:103F100065E6EF6021541785010013056509EF6020
:103F200061532945EF60415783C7412A1307700A3F
:103F30006384E7041307800A6380E7061307600AB7
:103F40006395E702930760F82382F12A83D7A127BC
:103F5000A382F12AA1832383F12A8547A387F12A2B
:103F6000B1451385412AEF408060EF30502E134554
:103F70000404239D01265DB3930770F82382F12A80
:103F800083D7A127A382F12AA1832383F12A85471E
:103F9000A384F12A9945F1B7930780F8C5B793F741
:103FA00005080145E38C07D69785010093854558A0
:103FB00017850100130505DCEF60C1491785010075
:103FC00013058500EF6001492945EF60E14C930737
:103FD000A0F82382F12A83D74129A382F12AA18361
:103FE0002383F12A8547A383F12A239A0128EF30FE
:103FF00010261385412A9145EF4060571345040868
:1040000031BB411122C4978501009385254E2A8436
:1040100017850100130505D606C6EF60A1434C4085
:10402000178501001305C56EEF60C1422945EF6099
:10403000A146034704009307F00F6319F702978521
:1040400001009385A54A178501001305A5D2EF60ED
:1040500061404C40178501001305856CEF60813F7E
:104060002244B240294541016F600143B2402244DD
:104070004101828085CD411122C4178501001305BD
:1040800065CF2E84978501009385454106C6EF6074
:10409000613CA285178501001305C573EF60813B64
:1040A0002244B240294541016F60013F82804111A5
:1040B00022C426C22E84AA84978501009385C53E1A
:1040C00017850100130505CB06C6EF60A1381785DB
:1040D00001001305E570EF60E1372945EF60C13B52
:1040E000978501009385453C2394911E1785010017
:1040F000130545C885442392811E2393911E97176B
:104100000020239E874CEF60E1349715002083D573
:10411000054D178501001305256DEF60A133294575
:10412000EF608137971700202388973AEF10606877
:104130002285EF4080170545EF40A04B97F7FF1F02
:104140009387C712DC4703D70700C167FD176310C9
:10415000F7022244B7E70400B240924403A3870564
:1041600003C5819D1306000A854541010283B240C3
:104170002244924441018280011122CC37E40400A0
:104180005C5C06CE26CA3546978501009385C547F7
:10419000179501001305450C829701E91785010069
:1041A000130505C3EF60C13F01A097F7FF1F938779
:1041B00027573EC4B7F50700856793870780814678
:1041C0001386C19DE10519453EC697E0FF1FE780B4
:1041D00040597C4419469385C19D1385C12082971F
:1041E00034001386C19D979501009385E599179535
:1041F00001001305E59AEF506073AA8415C99785ED
:1042000001009385E531178501001305A5B6EF6020
:104210006124A6851785010013050540EF60812301
:104220002945EF606127F2406244D24405618280F3
:10423000EFB0500A1785010013050535EF40B00EA9
:10424000EF808078EF20011717F5FF1F130585FE1B
:10425000EF20E1031785010013050534EF20411716
:10426000AA84EF405069EFD0703CEF40A136EF6078
:104270006005EF508048EF00411997850100938554
:10428000252A178501001305E5AE89C8EF60811C5A
:10429000A685178501001305653A49B7EF60811BB4
:1042A000178501001305C53BEF60C11A2945EF6072
:1042B000A11EEFF0F07BEFC030266303050E8545AD
:1042C00037050400EF10104D9785010093854525B3
:1042D00017850100130505AAEF60C11717850100B6
:1042E00013058539EF6001172945EF60E11A97F74B
:1042F000FF1F938767E783D7070017170020231056
:10430000F72E8547171700202308F71CEF10A0652C
:10431000EF10204A171500200355652CEF30F07878
:1043200083C79139B9EFA30301008327441713060C
:10433000710085451305503082979785010093855C
:10434000251E178501001305E5A2EF60A110178552
:1043500001001305A534EF60E10F2945EF60C1139B
:10436000978501009385C51B17850100130585A05E
:10437000EF60410E1785010013054538EF60810D90
:1043800045B5978501009385A5191785010013058B
:10439000659EEF60210C178501001305A53365BFED
:1043A000978501009385C517178501001305859C26
:1043B000EF60410A1785010013050544EF6081098C
:1043C0002945EF60610D0145EF40A02251BF411129
:1043D00022C437E404008327041A06C68297EF300C
:1043E000B07583270408170500001305058682971A
:1043F000238CA19C17F5FF1F130545E7EF305012E2
:104400002244B24041018DBBB7E70400FC47117163
:10441000A2DDCAD986DFA6DBCED72E8432892E86CE
:10442000AA851385412A82971387412A834707006B
:10443000930680029387E70793F7F70F63E6F67416
:10444000BA898A07178701001307079CBA979C430C
:10445000BA9782878D47978501009385A50E1785AA
:10446000010013052591630BF400EF50B17E178511
:1044700001001305E5CBEF50F17DCDA2EF50917D0A
:1044800017850100130545CCEF50D17C2945EF601D
:10449000A100930720F811469385412A4A8523827B
:1044A000F12AA383012AEFF0EFE82A840DC597854E
:1044B000010093852509178501001305A58BEF5091
:1044C0007179A285178501001305C5CBEF5091784E
:1044D0002945EF50717C978501009385A5061785C6
:1044E000010013052589EF50F176178501001305AA
:1044F000A5CAEF5031762945EF50117A41659307EF
:1045000030FA05469385412A7D152382F12AEFF082
:104510006FE22A840DC5978501009385A502178552
:10452000010013052585EF50F172A2851785010062
:10453000130545C5EF5011722945EF50F175B7E7E6
:104540000400BC4F0566130606C8A14503C5819D3E
:104550008297FE506E54DE544E59BE5911618280CE
:1045600091476301F402978501009385A5FD1785A6
:10457000010013052580EF50F16D1785010013052B
:10458000E5C4D5BDB7E70400FC4F914503C5819D47
:104590008297978501009385E5FA17750100130549
:1045A000657DEF50316B178501001305E5C3EF50B2
:1045B000716A2945EF50516EEF3060499145C1A2B3
:1045C00085476301F402978501009385A5F7177568
:1045D00001001305257AEF50F167178501001305D7
:1045E00025C251BD23942121B7E704000566BC4FC5
:1045F000130606C8C14599BF8D476301F40297852C
:104600000100938525F4177501001305A576EF5079
:10461000716417850100130565C0B1BD930740F8AB
:1046200011469385412A4A852382F12AA383012AD0
:10463000EFF04FD02A84E30E05F0978501009385B3
:1046400065F0177501001305E572EF50B160A285A2
:1046500017850100130505B3EF50D15F2945EF50D1
:10466000B163C5BD9147E31CF4F8B7E70400FC4F04
:104670009305000203C5819D82979785010093856C
:1046800065EC177501001305E56EEF50B15C1785F9
:104690000100130525BA21BF894763E18702978589
:1046A0000100938525EA177501001305A56CEF50ED
:1046B000715A17850100130525B975BB83C4612A9A
:1046C00083C7512A978501009385C5E7A204177512
:1046D00001001305256ADD8CEF50D157A28517859F
:1046E00001001305A5B7EF50F156C2042945EF505C
:1046F000B15AC1849305D4FF93960401C1824A86BE
:1047000093F5F50F1385712AEF10500CE35390E4E5
:10471000930750F82382F12A83C7390022869385B4
:10472000412A85074A85A383F12AEFF0AFC02A8486
:10473000E30105E2978501009385C5E01775010047
:1047400013054563EF501151A2851785010013052C
:10475000650719B7894763E187029785010093854B
:1047600065DE177501001305E560EF50B14E178542
:104770000100130565B001B3EF30602DA2851385EC
:10478000412AEF30D05EF1B38D476301F402978583
:104790000100938525DB177501001305A55DEF501A
:1047A000714B178501001305E5AEF1B1B766020044
:1047B0000146B7750200054597E0FF1FE78060FAE4
:1047C000930760F82382F12AA383012A9307000646
:1047D0002384F12A8947A384F12A2385012AA3850A
:1047E000012AC1472386F12A930720F9A386F12ADB
:1047F0003146A387A12A9385412A4A852387012A26
:10480000EFF04FB32A84E30605D497850100938522
:1048100065D3177501001305E555EF50B143A28527
:1048200017850100130585A805BDB1476301F40292
:1048300097850100938505D11775010013058553F0
:10484000EF50514117850100130505A82DB1B7E7B9
:104850000400FC4F9305000403C5819D8297EF304F
:10486000001FB14529BF914763E187029785010089
:10487000938545CD177501001305C54FEF50913D48
:1048800017850100130505A6FDB683C4812A83C7D9
:10489000712AA204DD8C8E04B77702006D14BE94D9
:1048A0002286A68517850100130505A5EF50913ACC
:1048B000B7E70400FC4722869385912A2800829757
:1048C00093160401C1823000A685094597E0FF1FB9
:1048D000E78020E92A8419C517850100130585A3FF
:1048E000EF50114C930770F819469385412A4A8579
:1048F0002382F12AA384812AEFF0CFA32A84E30A3A
:1049000005C4978501009385E5C31775010013055C
:104910006546EF503134A28517850100130585A047
:1049200025BB99476301F41097850100938585C1E4
:104930001775010013050544EF50D13117850100AB
:104940001305C59F0DBE914763E18702978501005E
:10495000938545BF177501001305C541EF50912F91
:10496000178501001305059F39B683C4812A83C7C3
:10497000712AA204DD8C8E04B77702006D14BE94F8
:104980002286A685178501001305059EEF50912C00
:10499000B7E70400FC4722869385912A2800829776
:1049A00093160401C1823000A6850D4597E0FF1FD4
:1049B000E78020DB2A8419C5178501001305859C33
:1049C000EF50113E930780F819469385412A4A8596
:1049D0002382F12AA384812AEFF0CF952A84E30A67
:1049E00005B6978501009385E5B517750100130598
:1049F0006538EF503126A285178501001305C5994A
:104A0000A1B999476301F40297850100938585B3A5
:104A10001775010013050536EF50D12317850100E6
:104A20001305059989BCB7E70400FC4F9305000402
:104A300003C5819D8297EF308001994589B38D47E9
:104A40006301F402978501009385C5AF17750100D6
:104A500013054532EF501120178501001305C59647
:104A600019BC1785010013052597EF507133130505
:104A7000C01297E0FF1FE780008C0145EFE0EFB721
:104A80000D45EF00E07E294597E0FF1FE780A08AF3
:104A900097D0FF1FE780C07B6DBC99476301F4028C
:104AA00097850100938505AA177501001305852CCC
:104AB000EF50511A178501001305C5926DBA03C74F
:104AC000912A83C7812A22075D8F9166BA96C20612
:104AD0001166C1821306F6EF8D476363D60297E72E
:104AE000FF1F9387A7789C4B03C6712A9386C70044
:104AF00039C603D607004DCA8907E39CD7FE89470C
:104B00001307A0F811469385412A4A852382E12A9A
:104B1000A383F12AEFF00F822A84E30C05A2978584
:104B20000100938525A2177501001305A524EF50F8
:104B30007112A285178501001305058C31BE03D6BD
:104B400007006300E60A8907E39BF6FE8D474DBF29
:104B500091476302F402978501009385A59E17751E
:104B6000010013052521EF50F10E178501001305F3
:104B7000258A6FF05F90B7E70400FC4F93050008AB
:104B800003C5819D82970DBC978501009385859B08
:104B9000177501001305051EEF50D10B1785010095
:104BA000130585886FF03F8D2390E70017E5FF1F01
:104BB0001305C56BEFF0D0099785010093858598A3
:104BC000177501001305051BEF50D108178501006B
:104BD00013058586EF5011082945EF50F10B8147E9
:104BE00005B72390070017E5FF1F13052568EFF0B1
:104BF0003006978501009385E5941775010013052C
:104C00006517EF5031051785010013056584D9B785
:104C1000411122C406C6834705002A849DC3978597
:104C200001009385E58D177501001305A514EF505C
:104C300071024C4017850100130505BFEF5091012B
:104C400075A05841B707CF009387777D6313F706A8
:104C5000978501009385C58A177501001305851195
:104C6000EF50417F1C448356E4008355C40003C6C3
:104C70000700178501001305A5BCEF50A17D29454C
:104C8000EF5091010357E4009717002083D7279531
:104C90006307F7008355C4000844EFE0EFA903560B
:104CA000E4008355C40008442244B24041016FF03F
:104CB000AFF5B707CC009387777D631FF702978521
:104CC00001009385E583177501001305A50AEF50D0
:104CD00061781C448356E4008355C40003C6070072
:104CE000178501001305C5B5EF50C1762244B240C7
:104CF000294541016F50417AB707CE009387777DF0
:104D00006302F702977501009385857F177501008F
:104D100013054506EF5001744C401785010013053B
:104D200065A729BFB240224441018280B7E7040051
:104D3000FC4741112E8606C622C426C24AC02E84D4
:104D40002A89AA851385412A829797850100938530
:104D50002581177501001305E501EF50A16F83C58B
:104D6000412A177501001305A527EF50A16E2945AB
:104D7000EF5081729384412A83C70400414793878F
:104D8000070693F7F70F636BF746177701001307D2
:104D9000E7118A07BA979C43BA9782879D476303B6
:104DA000F402977501009385A57B17750100130523
:104DB00065FCEF50216A177501001305E522EF50DD
:104DC0006169D9A283C7512AADCF03C7712A83C7AE
:104DD000612A22075D8F83C7812AC2075D8F83C73F
:104DE000912AE207D98F23A0F12883C76400977521
:104DF00001009385E576177501001305A5F7238F4C
:104E0000F126EF502165938701288C4303C6E127E3
:104E1000177501001305051FEF50C1632945EF50B9
:104E2000A167A382012A2244B24092440249930717
:104E300000F82382F12A9D451385412A41016F30F4
:104E40000073EF40B06E2383A12A93578500A3839C
:104E5000F12A935705012A842384F12A9357850167
:104E60000145A384F12AEF40306D2385A12A97756F
:104E700001009385E56E177501001305A5EFEF504E
:104E8000615D03C6A12AA2851775010013050519E6
:104E900061B7CD476301F402977501009385456CB6
:104EA00017750100130505EDEF50C15A1775010084
:104EB0001305451829B737E404007C44414693851F
:104EC000512A13854128829713854128EF0010232A
:104ED000EF00300E83C7612B03C7512BA2070323BA
:104EE0008405D98F239EF1261306000A89452244A2
:104EF000B2409244024903C5819D410102838D471E
:104F00006301F402977501009385856517750100AB
:104F1000130545E6EF5001541775010013054521AF
:104F200079BD03C4612A83C7512A9775010093850F
:104F300025632204177501001305C5E35D8CEF504E
:104F40006151A2851775010013054510EF5081507E
:104F50002945EF5061540D469385412A2285EFE0A3
:104F60007FBDAA8415C9977501009385655F177584
:104F70000100130525E0EF50E14DA68517750100EE
:104F80001305050EEF50014D2244B24092440249F0
:104F9000294541016F50415023948120B7E7040017
:104FA000116603A38705130606E8914589B78D4767
:104FB0006301F402977501009385855A1775010006
:104FC000130545DBEF500149177501001305052551
:104FD000FDB303C4612A83C7512A977501009385E5
:104FE00025582204177501001305C5D85D8CEF50B4
:104FF0006146A285177501001305C507EF5081456D
:105000002945EF5061490D469385412A2285EFE0FD
:105010007FB2AA840DC197750100938565541775F9
:105020000100130525D5EF50E142A6851775010053
:105030001305850581BF2396811EB7E7040011661D
:1050400003A38705130606E8930500024DB58947BB
:1050500063E18702977501009385855017750100FC
:10506000130545D1EF50013F177501001305C51D0C
:10507000B9B383C4612A83C7512A97750100938508
:10508000254EA204177501001305C5CEDD8CEF5027
:10509000613CA6851775010013058500EF50813B23
:1050A0002945EF50613F22869385412A2685EFE00E
:1050B0007FA82A8463030516977501009385454AE6
:1050C00017750100130505CBEF50C138A285177580
:1050D0000100130525FE7DB5854763F087148345E0
:1050E00019002244B24092440249B335B000238EE5
:1050F000B12017750100130525FD41016F50813561
:10510000A2852244B24092444A85024941016DAAD7
:1051100099476301F40297750100938565441775FB
:105120000100130525C5EF50E13217750100130585
:10513000652B71B103C4612A83C7512A9775010099
:10514000938505422204177501001305A5C25D8CE5
:10515000EF504130A28517750100130565F8EF5037
:10516000612F2945EF50413319469385412A228505
:10517000EFE05F9CAA840DC1977501009385453EC1
:1051800017750100130505BFEF50C12CA6851775D3
:1051900001001305E5F5FDB3239A8128B7E7040064
:1051A000116603A38705130606E89305000881B37B
:1051B0008547977501009385A53A1775010013057A
:1051C00065BB6309F400EF50E12817750100130572
:1051D00065F3F5B6EF50012817750100130505F4C6
:1051E000EF5041272945EF50212B2244B2409244F1
:1051F0000249239E012641016F40B02797750100A7
:1052000093850536177501001305C5B6EF50812447
:1052100017750100130545215DB6B2402244924442
:10522000024941018280411106C622C4EFE09F90ED
:105230009377F50F95CB2A84977501009385C53335
:1052400017750100130505B3EF50C1209375F40FD6
:105250001775010013050557EF50C11F2244B240D6
:10526000294541016F504123B240224441018280CF
:10527000411122C491462A84138681389D652D45AB
:1052800006C697D0FF1FE780C04DB7F7070003C7DA
:105290000701A5476313F70001A09306001001461C
:1052A0009D65254597D0FF1FE780A04B238481385B
:1052B0002244B2409146138681389D6529454101BB
:1052C00017D3FF1F6700E3495171CAD137E90400C2
:1052D0008327C904A2D52E8686D7A6D32E84AA8575
:1052E0001385412A829783C7412A1307700A638B6B
:1052F000E70C636CF7001307600A6382E704BE5093
:105300002E549E540E596D6182801307800A63806B
:10531000E7121307900AE394E7FE8D476309F4163A
:10532000977501009385455D17750100130585A4E8
:10533000EF504112177501001305455915A08D470F
:105340006306F402977501009385055B17750100EC
:10535000130545A2EF5001101775010013054550C4
:10536000EF50410F2945EF50211351BF8547177565
:1053700001001305A550238EF120EF506122B7756F
:105380000200B76602000146054597D0FF1FE7807F
:10539000403D930760F82382F12AA383012A9307F3
:1053A000002623A4F12AE577938707212396F12A83
:1053B000B1452387012AA387A12A1385412AEF300B
:1053C000001B35BF914763E1870297750100938504
:1053D000A552177501001305E599EF50A107177540
:1053E00001001305A54BADBF83C4812A83C7712A71
:1053F000A204DD8C8327C9046D1422869385912A2B
:10540000280082978E0493160401B7750200C182AA
:105410003000A695094597D0FF1FE7808034930799
:1054200070F82382F12A9945A384A12A79B791477C
:1054300063E18702977501009385054C177501009C
:1054400013054593EF5001011775010013058546BB
:1054500001BF83C4812A83C7712AA204DD8C8327FC
:10546000C9046D1422869385912A280082978E04A0
:1054700093160401B7750200C1823000A6950D4550
:1054800097D0FF1FE780E02D930780F859BF17756D
:1054900001001305E544EF50A1101305C01297D089
:1054A000FF1FE78040E90145EFD03F950D45C93327
:1054B000294597D0FF1FE78000E897D0FF1FE780BE
:1054C00020D935BD41114AC09706002083D6261148
:1054D000328917E6FF1F035686DB22C426C206C6A2
:1054E0002A84AE84B12325C139CC994763FD970442
:1054F0008347140003470400A207D98F139787003E
:10550000A183D98FC2073167C1831307C755639C35
:10551000E70297E7FF1F83D787D7A301F400A18392
:105520002302F4009707002083D7670B91C7A302DB
:10553000F400A1832303F400A68517750100130569
:10554000A53FEF4031719707002083C7E7F8A9C74F
:1055500097E5FF1F83D5A5D3177501001305853F78
:10556000EF40516F2686A28517E5FF1F035525D210
:10557000EFF07FCB6309090283C781398DC785C4EA
:1055800083C7C1218DE322852244B2400249A6850A
:10559000924441016F20B07D177501001305853CD1
:1055A000EF500100C1BFB240224492440249410180
:1055B0008280834755008345450017750100130518
:1055C0006536A207DD8D6F40F16817750100130580
:1055D00065346F40F17C8D4763FAB708011126CA24
:1055E00006CE22CC0344350083C49139977501005F
:1055F00093850538B3378000A38CF13809C49775BB
:1056000001009385A537177501001305A537EF40F5
:10561000716483C7913963839700152483C79139D7
:105620009DC385472306F100B7E7040083A747170A
:1056300070008545130550308297177501001305DA
:105640006535EF40F1759967938757EE2316F100A2
:10565000680085479145A30781002307F100EF20EB
:105660001071F2406244D244056182808280894791
:1056700063F2B708011122CC06CE26CA8344250066
:1056800085472A846398F404914763F0B70403457F
:1056900045008347340022055D8D97E7FF1F23985F
:1056A000A7BE19299967938767EE2314F1008347F2
:1056B000340023059100A305F1008347440095457C
:1056C00028002306F100EF20906AF2406244D244A1
:1056D00005618280FDF89967938767EE2314F100D6
:1056E00097E7FF1F83D7A7BAA305F10023050100A1
:1056F000A183F1B782800111996722CCD5171704D5
:105700000020130464DD2314F1008347040026CA3B
:10571000970400209384A4EC2305F10083D70400B0
:1057200028009545A305F100A18306CE2306F100CC
:10573000EF20F06303D604008345040017750100D1
:105740001305C526EF401151F2406244D244056171
:1057500082809D677971D9172316F1009707002081
:1057600083C787D706D62307F1009DCBB7E7040090
:10577000FC474146938541281305F1008297680054
:10578000CD45EF20D05E9705002083C5E5D4177581
:1057900001001305A524EF40F14BB2504561828012
:1057A000B7E70400BC47414681451305F1008297E5
:1057B000F9B7B76702045D71938757AA3EC0970790
:1057C0000020938767D183C70700A2C4231201007A
:1057D0002303F10097070020938767E083D7070032
:1057E00037E40400A30301002314F10097E7FF1F2F
:1057F0009387E7A983D7070086C641462315F100A2
:105800007C446800938541288297F1450A85CD2222
:10581000231EA1007C448A850810794682973C4467
:105820001305E10309468145829710109305000294
:105830000145EFD03FBFB640264461618280B7C7C3
:10584000A55A01119387C7333EC483C791393EC619
:10585000B7F7070003C7070106CE22CCA54763139D
:10586000F70001A01164930504F0930600100146AF
:10587000254597D0FF1FE780C0EE3000930504F068
:10588000A146294597D0FF1FE780A0ED83C5913938
:105890001775010013054525EF40D13BF2406244E6
:1058A0000561828001119165A1463000938505F064
:1058B0002D4506CE97D0FF1FE780A0EA2247B7C745
:1058C000A55A9387C7336310F702B24517750100D5
:1058D0001305C514B335B000A38CB138EF40913730
:1058E000F240056182808145177501001305451559
:1058F000A38C0138EF4011369937DDB7B7C7A55AE9
:1059000079719387F7353EC6B7E70400FC47AA854F
:1059100006D622D4414608088297B7F7070003C786
:105920000701A5476313F70001A01164930504E87C
:10593000930600100146254597D0FF1FE78060E2DF
:105940007000930504E8D146294597D0FF1FE780F2
:1059500040E1177501001305E51CEF407144B2509A
:1059600022544561828079719165D146700093859A
:1059700005E82D4506D697D0FF1FE78080DE324729
:10598000B7C7A55A9387F735177501001305451357
:10599000631EF700B7E70400FC4713854128414622
:1059A0000C088297177501001305850FEF40513FD2
:1059B000B25045618280B7F7070003C70701A547CA
:1059C0006313F70001A09165411193060010014691
:1059D000938505E8254506C697D0FF1FE78060D868
:1059E000B240177501001305A50141016F40513BFD
:1059F000C16769768146FD17050613970601418345
:105A00006364B7003E8582803307D50003470700F3
:105A1000B98F214713F81700858363050800B18FFC
:105A2000C207C1837D171377F70F6DF78506F1B7AE
:105A300049C1A547054763FFB706834715000347DC
:105A400005003168A207D98F13978700A183D98FEA
:105A5000C207C1831308C8550547639D0705411157
:105A600006C622C426C203442500914763FD87026F
:105A70009307540063E9F502A301C50021822302C4
:105A8000C5009304340091C6A302D500A18223036C
:105A9000D5002A84A685A93F26942300A40021814D
:105AA000A300A4000147B240224492443A85410138
:105AB000828005473A858280B7C7A55A011193872E
:105AC000E7343EC42AC6B7F7070003C7070106CE6E
:105AD00022CC26CAA5476313F70001A091642A844B
:105AE000938504EE930600100146254597D0FF1FCD
:105AF000E78020C73000A146938504EE294597D062
:105B0000FF1FE78000C6A285177501001305C5FFBA
:105B1000EF405114EFF0FFC9F2406244D2440561F6
:105B2000828001119165A1463000938505EE2D45D7
:105B300006CE97D0FF1FE780C0C22247B7C7A55A3D
:105B40009387E7346314F702B24517750100130514
:105B500025F197D7FF1F239CB772C205C181EF4083
:105B6000710FEFF01FC5F24005618280D147D1452A
:105B7000177501001305C5F017D7FF1F2319F7701C
:105B8000EF40510D17D5FF1F035565703537E1BF45
:105B9000011126CA06CE22CC93F71500AE848DCB18
:105BA000AD67371700409387A7AA1CC3B7E7040067
:105BB000BC4F13060019854517D5FF1F0345056D1A
:105BC000829713C51400F2406244D244056182807A
:105BD00093F725006388071497750100938585F86E
:105BE0002D464800EF40A17B9705002083C5059F07
:105BF000854793C4240063EFB7028DC5854517051B
:105C000000201305A58DEF10F01083C7813999CBC3
:105C10009705002083C5859C170500201305058C7A
:105C2000EF20F01413950401970700202388079AAA
:105C3000418151BF170400200344448A9707002084
:105C400083C7D78922045D8CAD67C2059387B7559A
:105C5000C181630BF40A63EB8702A9679387A75599
:105C6000630BF40A1705002013054587EF10900A0F
:105C700083C78139D1C39705002083C525961705B1
:105C800000201305A585EF20900EBDA0B167938776
:105C9000C755630EF402B5679387D755E314F4FC38
:105CA0001705002013058583EF20700C9705002051
:105CB00083C5C592894763F1B704F915C205C1814F
:105CC000170500201305A581EF10D00435A0054667
:105CD0001705002013058580EFF0CFFE97F7FF1F13
:105CE00083C7877F91EB4800EF40D11393150501DF
:105CF000C1814800EFD04FA4A2851775010013059C
:105D000065E4EF40217539BF17F5FF1F1305057DC9
:105D1000EFF03F8AD5B717F5FF1F1305257CEFF08D
:105D2000DF8AD9BF93F745000145E38E07E8177571
:105D30000100130565E2EF40B106EF20B01613C570
:105D4000440051B5411122C437E404005C5C06C62E
:105D50003546977501009385258B1775010013054E
:105D6000A54F829701E917750100130565E0EF4023
:105D7000310301A08327041C82972A840545EF90F4
:105D8000D054EF207148EF20B126EF9040092285D2
:105D9000B2402244410182801567B71700401307C3
:105DA000575598C3D8439D66558FD8C3D843FD76C1
:105DB000758FD8C3D8431367F70FD8C33567130758
:105DC000C7CC98C3828041111305800406C622C443
:105DD00026C297C0FF1FE780802D85457D55EFC007
:105DE0001FE985457D55EFC0FFF23714004083273A
:105DF000840A8D451305002093E707202324F40A25
:105E0000EFC0FFE6B7E40400EFD0CF98C858EF40EA
:105E100021791775010013052544EF406178832728
:105E2000840C8545414593E707082324F40CEFC013
:105E30007FEE8D4513050008EFC0DFEDEFD06F88D2
:105E40000145EFD02F8B85450545894717F7FF1F83
:105E50002308F778EFD0AF8B37070004B7E700E0EF
:105E600023A0E710EFD01F95EFD05FA8E13DEFF042
:105E70007FA3EFF01FCBEFE08FD5F5205D2083A748
:105E80000408170500001305E5D0829797D7FF1F78
:105E9000238EA73EBC4C1306006485458297ED3DDA
:105EA00097C0FF1FE780805301458280B7F7070046
:105EB00003C70701A547AE866316F7009397450110
:105EC00091C301A0AA850146254517D3FF1F67008E
:105ED00043894111B2862E86AA852D4506C697D0E4
:105EE000FF1FE7800088B24001454101828093078F
:105EF000000463E6C7021D71A2CC2A84080886CE7E
:105F000032C6EF40C149B2461008A285294597D054
:105F1000FF1FE7800085F640664425618280395581
:105F2000828041110D658D4506C6EFC05FD4B7175D
:105F300000408D6623A6D70A17F5FF1F1305856A53
:105F40001387C70A9387870A1CC15CC58566896762
:105F50005CC958C114C518C9B7E70400B24003A30F
:105F6000871E4101028397F7FF1F83C7276989EFC7
:105F7000411106C6EF104055B240854717F7FF1F85
:105F8000230EF76641018280828001C599C16FC0EE
:105F9000BFFA8280411126C2AE848D4522C406C656
:105FA0002A84EFC03FD7B717004099C803A5C70C94
:105FB000418D23A6A70CB240224492444101828025
:105FC00003A5870C418D23A4A70CF5B783470500D3
:105FD00003471500A207D98FC2076177C18713074E
:105FE00027206397E70083452500370504005DB748
:105FF000828017F6FF1F1306A6608147B28613033F
:10600000F00FA9483308F6000348080013F7F70F0C
:106010006303A80C630668008507E39517FF29470B
:10602000B387E6002380A70097F7FF1F9387075EDB
:106030007DA0411113D765001347170006C693F6DC
:106040003500058B954791CA054699476387C60079
:1060500009469D476383C600A14713F645003336C2
:10606000C00093F68503050685C2A1456389B60481
:10607000E1456388B604930580026386B604930500
:1060800080036393B600914697F5FF1F2385F57E45
:1060900097F5FF1F2380C57E97F5FF1FA38CD57C46
:1060A000BE8517750100130525B6EF40A13AB24031
:1060B000854717F7FF1FA300F77C410182808546C3
:1060C000E1B78946D1B78D46C1B7177501001305F1
:1060D00025B66F40213817F7FF1F13072753BA97CC
:1060E0002380B700E147E306F5F493077002E30E5F
:1060F000F5FC82802A8723800500814717F5FF1F62
:10610000130505501308F00F2946B306F50083C6A2
:1061100006006396E60297F6FF1F9386264FB69712
:1061200083C7070005452380F5009947636EF70292
:106130009D4763FDE700E147630DF70082806385BB
:1061400006018507E393C7FC0145C5B72380050019
:106150008280B737004003C7370083C7050093F735
:106160000704D98F2380F5008280797126D24AD026
:106170009704002083C40482170900201309C980F2
:1061800006D622D44ECE52CC56CA5AC8B30799006E
:1061900083C7070093F7F70FA5C79387140093F7FA
:1061A000F70F0D476361F70C17F7FF1F2304F77E06
:1061B00097F7FF1F9387C77DA69783C7070013072D
:1061C000100293F7F7036383E7286363F70A054434
:1061D000638A871EE385076609476389E714130707
:1061E0000002E38CE750B7E700E03707400023A048
:1061F000E71801000100CA942380040023A0E710DF
:10620000B787004003C76700058BE309077097F65F
:10621000FF1F83C646780547E394E66E294723812E
:10622000E70209472383E7022385E70297F7FF1F69
:10623000A384076497F7FF1FA38F0774B7870040F5
:10624000A381070017F7FF1FA30A076205472383EF
:10625000E700B250225492540259F249624AD24A9B
:10626000424B4561828097F7FF1F2385077289B7EC
:10627000130730026386E70A63E0E714130740025E
:10628000638AE70813070003E39FE7F497F7FF1F0C
:106290009387C76FA69703C70700A1471377F70F28
:1062A000E31AF71617FAFF1F130A0A3783476A0023
:1062B00097F6FF1F2388F65A97F7FF1F83C73736D5
:1062C00091C7FD5797F6FF1F238EF65897F5FF1FCE
:1062D00083C5953497F7FF1FA386B75897F7FF1F1D
:1062E00083C7873393F907089306000493F70706DB
:1062F000639DD74E9307A0096381F51A63EEB71427
:106300009307F0056384F54C930750096386F52CD9
:106310000144BDA3FD5717F7FF1F2304F754E1B550
:10632000FD5717F7FF1F230DF75275BD17750100B5
:10633000130585A1EF40C12697F7FF1F93870765D7
:10634000A69703C40700814917FAFF1F130A4A459D
:106350001374F40F977A0100938A8A9F63C58904A6
:106360002945EF406113854717F7FF1FA308F74240
:1063700017F7FF1F2305874217F7FF1F230EF74E5E
:1063800037E700E0B70640002320D71801000100DE
:10639000378600408347A60293F7370F2305F6029E
:1063A0002320D71089B5B3073A0183C50700568566
:1063B0008509EF40210A5DB7854717F7FF1F230FB7
:1063C000F73C15B51775010013050598EF40411D01
:1063D00097F7FF1F9387875BA69703C40700814940
:1063E00017FAFF1F130A8A2F1374F40F977A01000C
:1063F000938A0A9663C389042945EF40E1098547DA
:1064000017F7FF1FA30AF72C17F7FF1F2307872C87
:1064100017F7FF1F2302F74637E700E0B7064000F3
:106420002320D71801000100378600408347660209
:1064300093F7370F2303F602A5B7B3073A0183C5D5
:10644000070056858509EF40E1006DB7854717F7CE
:10645000FF1F2303F72841BB9307400A6383F534EA
:106460009307200B638EF5349307100AE392F5EA45
:1064700083072A00014463D5074097F7FF1F83C7AE
:10648000D71993F637006384061A05466384C6223B
:106490000946639FC6181D4761AA17F5FF1F0345EC
:1064A000C517C94717FAFF1F034A3A1797F5FF1F89
:1064B00083C5C51617F4FF1F034454166317F51060
:1064C000CD476314FA1093077008639AF502130717
:1064D000300FB7170E006308E4001307900DB7B72D
:1064E00004006312E40817F7FF1F2323F738BE8563
:1064F0001775010013054586EF30D17511BD93075F
:106500008008639DF50033048040B777460013741C
:10651000F40F938787CDB3D78702F1B7930790081D
:10652000639AF5003304804091671374F40F9387E6
:10653000C766D5B79307A008639BF5003304804076
:10654000B7173D001374F40F93870790E9B79307CB
:10655000B008639AF5003304804091671374F40F18
:10656000938797D04DBF93F5F5078D47639BF50053
:1065700033048040B7975B001374F40F938707D8F8
:1065800059BF8947639BF50033048040B7770B0000
:106590001374F40F9387071BBDBF8547639AF500FB
:1065A00033048040DD671374F40F938767E3A5B766
:1065B00089E9330480408D671374F40F938777DC87
:1065C00099BFF1679387072039BFEFF09FA2A2859B
:1065D0005285EFF01FA22DBB9305610017F5FF1F39
:1065E0000345A50317F4FF1F03443403EFF09FB0E6
:1065F000930571002285EFF0FFAF3C0017F7FF1FF6
:106600002322F738834761002304F1008347710098
:10661000A304F100894717F7FF1F2305F7248357C9
:10662000810017F7FF1F2319F7FE094491AC1547A6
:1066300093F64700B336D00093F78703850685C3EA
:106640002146638BC7066146638AC706130680022C
:106650006388C706130680036393C700914717F644
:10666000FF1F2309D62097F6FF1FA385F62097F773
:10667000FF1F2382E72017F7FF1F034727FA9376B0
:10668000070497F7FF1F83C777F98DEE1377770C11
:1066900093067008630CD7021377F7078D46631EC5
:1066A000D70AB307F040B7955B0093F7F70F9385D0
:1066B00005D881A81947ADBF854755B7894745B764
:1066C0008D4771BF930670086311D7021307300F0F
:1066D000B7150E006389E7021307900DB7B50400E4
:1066E0006383E7021307700845BF9306800C6311AC
:1066F000D702B307F040B775460093F7F70F9385BD
:1067000085CDB3D5F50297F7FF1F23A3B716CDB3F9
:106710009306900C631AD700B307F040916593F786
:10672000F70F9385C566F1BF9306A00C631BD700D6
:10673000B307F040B7153D0093F7F70F9385059029
:10674000C9B79306B00CE319D7F4B307F0409165CD
:1067500093F7F70F938595D06DB78946631BD700E4
:10676000B307F040B7750B0093F7F70F9385051B40
:1067700049BF8546631AD700B307F040DD6593F73C
:10678000F70F938565E3B5BF09EBB307F0408D655F
:1067900093F7F70F938575DCADB7F1659385052009
:1067A0009DB783472A00C18B99C7854717F7FF1FFD
:1067B000230DF70AB1BE97F7FF1F2388070A89BE8A
:1067C000854717F7FF1FA308F70A99B63C0017F78C
:1067D000FF1F2329F71A0947930700032314F10029
:1067E00097F6FF1F2380E6082DBD639C0754A94739
:1067F00063E2B742176701001307473E8A05BA955F
:106800009C41BA97828717F4FF1F034414E1094A99
:106810006308440F636A8A0885476307F40A93078D
:10682000F00F17F7FF1F0347E70363F6E70017F7BB
:10683000FF1F2309F70217FAFF1F034AAA02930753
:1068400000041374FA0F63F447011304000497F76C
:10685000FF1F9387271383AA0700228617F5FF1FC0
:10686000130585DBD685330A8A40A29AEF3031338F
:1068700097F7FF1F238847FF97F7FF1F23A45711A0
:1068800097F7FF1F83C717FE15476390E75EB7E7CB
:1068900000E03707400023A0E71801000100B78699
:1068A00000402380860239A58D476306F40A994784
:1068B000E317F4F6976701009387C73817F7FF1FB0
:1068C0002322F70CA947B1BF17F7FF1F0347A70CF7
:1068D00097F7FF1F938707FB49469765010093854C
:1068E000653F63068700976501009385A53A3E855D
:1068F000EF30F12A17F7FF1F2326A708C94715B75E
:1069000097F6FF1F83C62609054797F7FF1F938752
:1069100067F76392E6023E851306700297650100F1
:106920009385C538EF30B12717F7FF1F232CA70435
:1069300093077002FDB53E8513063004976501008C
:1069400093850531EF30B12517F7FF1F232CA702E0
:1069500093073004F9B597F5FF1F83C505CC17657C
:1069600001001305A540EF30F12E854A17FBFF1FEC
:10697000034B6B0297F5FF1F83C525CA17650100FE
:106980001305C53E63145B0BEF30D12C97F7FF1F47
:1069900083C7A7C8A5CBE364F4E817640100130418
:1069A000A437638C6701176401001304643763869E
:1069B000470117640100130424382285EF30914603
:1069C0001375F50F93071500860717F7FF1F230BA5
:1069D000F7EA8D4717F7FF1FA306F7EA97F7FF1FA0
:1069E000938747EA0147BE861376F70F89076365E9
:1069F000A60297F7FF1F23A7D7F897F7FF1F83C7B4
:106A000067E805B5976701009387072A17F7FF1F07
:106A1000232AF7F6914731B53306E4000346060012
:106A2000A380070005072380C7007DBFEF309122B8
:106A300097F7FF1F83C767BEF1D7E362F4DE1764E1
:106A400001001304642A638C5701176401001304C6
:106A5000242A63864701176401001304E42A22856F
:106A6000EF30513C1375F50F93071500860717F7A4
:106A7000FF1F2309F7E08D4717F7FF1FA304F7E077
:106A800097F7FF1F938707E00147BE861376F70F3E
:106A90008907E370A6F63306E40003460600A380E8
:106AA000070005072380C700D5B797F5FF1F83C5EB
:106AB000C5B6176501001305252CEF30B11997F7FE
:106AC000FF1F83C7F7DB93E7470017F7FF1FA309F3
:106AD000F7DA83472A0017F7FF1FA301F7DA6FF0F1
:106AE0003F83176501001305652AEF30712B97F777
:106AF000FF1F9387A7D883C7070017F7FF1F230D32
:106B0000F7B017F4FF1F0344E4D5333480008DBB86
:106B1000176501001305C528EF30912897F7FF1F6F
:106B200083C717D693E7070117F7FF1FA30AF7D408
:106B300083472A0017F7FF1F2302F7D46FF04FFD9A
:106B40001765010013050527EF30912503470A005B
:106B50007D8B51EFB787004003C767021377C70BE0
:106B6000136727002383E70203C7A7021377C70B26
:106B7000136727002385E70203C7E7021377C70BD4
:106B8000136727002387E70203C727031377C70B81
:106B9000136727002389E702854717F7FF1F230D97
:106BA000F7B217F7FF1F230BF7BE17F7FF1F2309D5
:106BB000F7CA17F7FF1F2306F7CA97F7FF1FA38D22
:106BC00007B097F7FF1FA38B07BC97F7FF1FA38999
:106BD00007C897F7FF1FA38607C897F7FF1FA38D66
:106BE00007C897F7FF1FA38807DA6FF06FF289478E
:106BF0006312F70297F7FF1F83C747A29146638C82
:106C0000D70863E0F604638EE70C6369F70A05476B
:106C10006380E70EFD5717F7FF1FA305F7C437077B
:106C20004000B7E700E023A0E71801000100B786A5
:106C300000401306F0FC2381C60223A0E7106FF08A
:106C40008FDA130720086382E7086362F7021307ED
:106C50001008E391E7FC378700408347670293F70A
:106C6000C70B93E727002303F7026FF06FEA1307C0
:106C700030086389E70213074008E39DE7F8378788
:106C800000408347270393F7C70B93E727002309A7
:106C9000F7026FF0EFE7378700408347270393F74A
:106CA0003707F5B7378700408347E70293F7C70BED
:106CB00093E727002307F7026FF08FE5378700403F
:106CC0008347E70293F73707F5B7378700408347D5
:106CD000A70293F7C70B93E727002305F7026FF08E
:106CE0002FE3378700408347A70293F73707F5B7AD
:106CF000378700408347670293F73707ADB71765BB
:106D000001001305250CEF30B10997F7FF1F23850C
:106D10000790C5BB176501001305C50BEF3051087F
:106D200097F7FF1F239A078E97F7FF1F938787B365
:106D300003C40700894763F3870009441374F40F01
:106D400081B613070002E397E7EC639F0908638DA0
:106D5000F500930720026389F50617650100130506
:106D6000E50AEF30216F7DB5176501001305450772
:106D7000EF3011030144176B0100130BAB07A14A5D
:106D8000B3078A0083C507005A850504EF30816C7C
:106D9000E31854FF1755010013058564EF305100C7
:106DA00017F4FF1F0344848711E497F7FF1F23881C
:106DB0000784F9B48947E31FF4E4854717F7FF1FF9
:106DC000230FF7826FF0CFD417F6FF1F0346F68428
:106DD00097F5FF1F83C5658417650100130505023C
:106DE000EF3041676FF0CFD2638DF5049307100247
:106DF000E395F5F697F5FF1F83C5458217650100FA
:106E00001305C501EF30016597F7FF1F23AC47B7A6
:106E100097F7FF1F9387C7A5944383D7470017F7BA
:106E2000FF1F034747A517E6FF1F2327D67E1D44F4
:106E300097E6FF1F2394F67E97E7FF1F2381E77EE7
:106E400081B497E5FF1F83C5657D176501001305B4
:106E500065FEEF30216097E7FF1F2382077A97E7EF
:106E6000FF1F239B077A6FF04FFC2547E381E7A2C2
:106E700019476391E702B786004023808602B7E78F
:106E800000E03707400023A0E718010001001306C7
:106E900000FC55B31307100A6391E702B786004060
:106EA00023808602B7E700E03707400023A0E718F9
:106EB00001000100130680FCBDBB1307A009E38F8E
:106EC000E7FC1307400AE38BE7FC13072002E3808B
:106ED000E79C0547E38DE79AB7E700E037074000F6
:106EE00023A0E718E39B099A01000100B786004040
:106EF00023808602130620FC3DBB17F7FF1F0347C4
:106F000077966304F71E63E7E7029547630CF70E75
:106F100099476308F704B786004023800602B7E765
:106F200000E03707400023A0E71801000100130626
:106F3000A0FC11B39307F005630AF700930750090B
:106F40006306F70093071002E317F7FCB7E700E0CA
:106F50003707400023A0E71801000100B786004072
:106F600051BF97F9FF1F83C9E98F93070004CE8AA9
:106F700063F43701930A000497F7FF1F938787A0F4
:106F800003AA070013F4FA0F2286D28517E5FF1F24
:106F900013058568EF30A140B3878940529417F7F5
:106FA000FF1F2301F78C97F7FF1F23AD879C638E8C
:106FB0000902B787004023805703B7E600E0370691
:106FC000400023A0C6180100010003C72702134791
:106FD00007042381E70203C727021377C70F238122
:106FE000E70223A0C6106FF00FA0B78600402380F1
:106FF0000602B7E700E03707400023A0E7180100CA
:107000000100CDBD378700408347370097F6FF1F4B
:1070100083C6D68693F70708D58FA301F700B70676
:107020004000B7E700E023A0D718010001001306D5
:10703000A0FC2301C70223A0D7106FF0CF9A97F7C7
:10704000FF1F9387A794A69783C7070093F7F70FAF
:10705000C9CF97F7FF1F83C70794C1EB17F7FF1F2F
:1070600003475780930700026311F70897E7FF1F54
:107070009387875A03AB070097EAFF1F83CA0A5A10
:1070800017EAFF1F034A9A5997E9FF1F83C9295935
:10709000D2875687CE865A8697E5FF1F83C5255629
:1070A00017650100130585DAEF30C13A97E7FF1F36
:1070B00023A0677D97E7FF1F238E577B97E7FF1F6E
:1070C000A38A477B97E7FF1F2387377B97E7FF1F3D
:1070D000A3868752B7E700E03707400023A0E718F0
:1070E00001000100B7860040F1B3B7E700E03707C1
:1070F000400023A0E71801000100B786004005BD4D
:1071000029472381E70209472383E7022385E70212
:107110002387E7022389E7026FF04F9103C76700D7
:10712000118B6308079283C75700918BB5CF17F770
:10713000FF1F0347478685476313F70697E7FF1F3F
:10714000A38BE77297E7FF1F2388075897E7FF1F76
:107150002386076497E7FF1F2384077097E7FF1FC5
:107160002381077097E7FF1FA388075697E7FF1F44
:10717000A386076297E7FF1FA384076E97E7FF1FA9
:10718000A381076E97E7FF1FA388076E97F7FF1F7E
:10719000A3830780B787004011476FF04F8B17E735
:1071A000FF1FA30DF74479BF854717E7FF1F23058E
:1071B000F75217E7FF1F2303F75E17E7FF1F2301AF
:1071C000F76A17E7FF1F230EF76869BF854717E7C0
:1071D000FF1F2303F75017E7FF1F2301F75C17E793
:1071E000FF1F230FF76617E7FF1F230CF76617E74C
:1071F000FF1FA303074E17E7FF1FA301075A17E757
:10720000FF1FA30F076497E7FF1FA38C076482800B
:10721000411106C6653FB78700402380070013076A
:1072200040FC2386E7001307C004A386E70017E7A6
:10723000FF1F1307673E2398E70017E7FF1F130799
:10724000A741239AE70017E7FF1F1307274D239C49
:10725000E70017E7FF1F1307A758239EE7002947FA
:107260002381E70209472383E7022385E702238777
:10727000E7022389E702A3810700930600F8A380B1
:10728000D700930690022380D700FD562383D700B2
:107290002381E700B706400037E700E02320D7103E
:1072A00003C7170013671700A380E700B24097E7F2
:1072B000FF1F2395075C41018280411106C63937C3
:1072C000B787004023800700130700FC2386E700F0
:1072D0003147A386E70017E7FF1F1307E73323981B
:1072E000E70017E7FF1F13072737239AE70017E781
:1072F000FF1F1307A742239CE70029472381E702CA
:1073000009472383E7022385E702A3810700930649
:1073100000F8A380D700930690022380D700FD5683
:107320002383D7002381E700B706400037E700E05A
:107330002320D71003C7170013671700A380E700A7
:10734000B24097E7FF1F239B075241018280F167FC
:107350009387072017E7FF1F232CF750854717E770
:10736000FF1F2319F750A14717E7FF1F2305F75009
:1073700097E7FF1FA381075097E7FF1F238E074E54
:1073800097E7FF1F238D072697E7FF1FA388072690
:10739000814717E5FF1F1305A526FD5517E6FF1FBB
:1073A0001306C6262947B306F5002380B600B306A8
:1073B000F600238006008507E397E7FE97E7FF1FA7
:1073C0002384075C97E7FF1FA380075C97E7FF1FF5
:1073D000238D075A97E7FF1FA387074897E7FF1FEB
:1073E000A385074897E7FF1F2380074897E7FF1FFC
:1073F000238B074697E7FF1F238A074697E7FF1F60
:10740000A384074697E7FF1F2381074697E7FF1FDF
:10741000A38D0756828017E7FF1F0347C75785478D
:107420006314F7006FF07FE96FF09FDE411122C413
:1074300006C617E7FF1F0347075685472E8613F436
:10744000F50FAA856315F70417E5FF1F130505312E
:10745000EF20F17497E7FF1F23820734B7870040BE
:1074600023848702B7E600E03706400023A0C61851
:107470000100010003C7A7021377C70F2385E702A6
:10748000B240224423A0C61001454101828017E585
:10749000FF1F13056520EF20917097E7FF1F238DD5
:1074A0000722B787004023828702B7E600E037064D
:1074B000400023A0C6180100010003C7670213772C
:1074C000C70F2383E7026DBF411106C6EFF03FE807
:1074D000B240410189B7411106C6EFE01FC997E7E5
:1074E000FF1F83C7771F85C797E5FF1F83C5E51E6D
:1074F00099C517E5FF1F1305651EEFE01FA997E764
:10750000FF1FA38B071C97E7FF1F23870736B24097
:107510004101828041C5D9C197E7FF1F83C7073664
:10752000B5CF011122CC4AC84EC656C25AC006CEAB
:1075300026CA52C42E89AA890144930A0004371B23
:10754000030063772403B3078940C207C183BE8465
:1075500063F4FA0093040004C204C180130A1BD42C
:1075600097E7FF1F83C747178DE37D1A631C0A0047
:10757000F2406244D2444249B249224A924A024B02
:1075800005618280EFE07FBEE1BF338589002694EC
:10759000A6854204EFF09FE9418065B7828097E7B6
:1075A000FF1F9387E74218429C4383D6450003455B
:1075B000070083C5C700035646006396A50083D520
:1075C000E700638DD502011106CE2386A70023971D
:1075D000D700B705CF00DC4B9385757D05077D1679
:1075E0002EC2230001003AC42316C1002317D10084
:1075F00099C30A858297F240056182808280DC4DC2
:10760000DC4B81CFB7E70400904503A38705914584
:1076100017E5FF1F0345053C028382806D713C081E
:107620003EC6B707E500232291103EC8AA843C0855
:107630003285232611103ECA2324811023202111D4
:107640002E89EF2050682A849765010093858583F1
:107650001745010013050572EF20D15FA28517655C
:1076600001001305A592EF20F15E2945EF20D162BC
:10767000B705CB009385757D6800EF106044A28547
:107680006800EF20F059014781467000CA852685C1
:10769000EF10806315C52A84975501009385857E78
:1076A000174501001305056DEF20D15AA285176516
:1076B00001001305658EEF20F1592945EF20D15DBA
:1076C0008320C11003248110832441100329011059
:1076D0005161828097E7FF1F9387872F18429C4351
:1076E000797122D406D60348070083C807012A848B
:1076F00083D64500035546006396080183D82701C9
:10770000638DD8022388070105072399D70037081E
:10771000CC00DC4B1308787D3ACC1307F5FF42CA46
:1077200023080100231EE100231FD10099C7080888
:1077300032C62EC482973246A2452285EFF01FEE54
:10774000B2502254456182806D713C083EC0B7073B
:10775000E5003EC23C083EC42326111023248110BC
:10776000232291102317010023180100231901007F
:10777000231A0100231B010097C7FF1F83D787B37C
:1077800099E3C167FD172316F10097C7FF1F83D741
:1077900087B291EB97E7FF1F938787239C439C4316
:1077A000DC4783D7070017C4FF1F1304A4B0584C4D
:1077B0002317F10083574400484B2318F10005EDCF
:1077C0009755010093850573174501001305855AE8
:1077D000EF2051481755010013050573EF2091471D
:1077E0002945EF20714B8320C1100324811083248D
:1077F00041105161828097C7FF1F83C717AC89EB87
:10780000B7E70400BC5782975C4C23AA0700E1BF8E
:10781000FD1797C6FF1FA382F6AA035607018347E9
:1078200004014C470A85230BF100EF20903D97E7B8
:10783000FF1F9387E7199C430147814688430A86C7
:107840006C00EF106048AA841DC99755010093850C
:10785000656A174501001305E551EF20B13FA68584
:10786000175501001305056BEF20D13E2945EF2088
:10787000B142584CB7E70400BC57484B69B797C7AB
:10788000FF1F83C797A3F5D7B7E70400BC4F104489
:10789000854517E5FF1F0345E5138297A9B75C4EA1
:1078A000DC4BA9CBA1C9411122C417450100130526
:1078B000654C2E84975501009385056206C6EF201E
:1078C0007139A2851755010013058567EF2091389E
:1078D0002945EF20713CB7E704002244B24003A3DE
:1078E000870517E5FF1F0345E50E13064006914582
:1078F000410102838280411122C417C4FF1F130477
:1079000024991C4C06C689C7DC4399C34C4882970E
:10791000584CB7E70400BC57484B82975C4CB240C8
:10792000224423AA07004101828017C7FF1F1307C3
:107930002798834707009306F00B850793F7F70F07
:1079400063E9F60097C6FF1F2384F69603450700F8
:107950008280930700F8FDB7835745006386070EC2
:1079600001114AC817C9FF1F1309C99452C4032A39
:10797000C90106CE22CC03274A0126CA4EC656C2EA
:10798000F15721EF1307D00DFD576368C704B7E91E
:10799000040083A709072A84130586004205418154
:1079A000B284AE8A8297232AAA000325C9015C49C2
:1079B0009DEF97550100938525501745010013054C
:1079C000653BEF203129175501001305A55FEF2016
:1079D00071282945EF20512CDD57F2406244D244F2
:1079E0004249B249224A924A3E8505618280938784
:1079F0004400B705CF002319F5009385757D310547
:107A0000EF10000C0325C901834564003105EF2008
:107A100030210325C9012686D6853105EF20701E49
:107A20007146A2854A85EF209117504419CA83A751
:107A30008905854517E5FF1F0345C5F982978147ED
:107A400069BFEFF07FD0E5BFFD573E8582804111D1
:107A500026C297C4FF1F9384E485D84C22C437E420
:107A600004003C54484B06C68297DC4C0323C405F3
:107A70002244B240924423AA070017E5FF1F0345A2
:107A800065F5854541010283411126C297E4FF1F38
:107A9000938404F49C4006C622C44AC0D1CBDC4384
:107AA000C1CB5CC12300B5002A84975501009385A2
:107AB000E53B174501001305E52BEF20B1192945DA
:107AC000EF20911D9C4023A4070023A2070097B735
:107AD000FF1F9387E77BDC4FDC4B81C72955EFF015
:107AE0009FE197B7FF1F9387E77CDC4FDC4B99C37F
:107AF000EFF0FFF537E904008327C905894517E54D
:107B0000FF1F034525ED82978327C905914517E59A
:107B1000FF1F034525EC82979C4003A3470163099F
:107B2000030022852244B24092440249410102836B
:107B3000B2402244924402494101828001113285BF
:107B400006CE22CC26CA2E84EF20F017AA849755A1
:107B500001009385E534174501001305A521EF20A9
:107B6000710F030784000356640083554400A68602
:107B7000175501001305C53EEF20D10D2945EF2013
:107B8000B11197B7FF1F83C707716399970001452C
:107B9000EFF07FD681450A85EFF01FEFF240624497
:107BA000D244056182806D71232481102326111037
:107BB0002322911093F745002E84638507123C0819
:107BC0003EC0B707E5003EC23C083EC42317010093
:107BD0002318010023190100231A0100231B0100AF
:107BE00097B7FF1F83D7C76A99E3C167FD172316AD
:107BF000F10097B7FF1F83D7C76991EB97E7FF1F86
:107C0000938707DD9C439C43DC4783D7070017B766
:107C1000FF1F1307E7672317F100544F83574700EF
:107C20002318F100DC4A95EF975501009385852BC9
:107C30001745010013050514EF20D1011755010068
:107C40001305852CEF2011012945EF20F104134580
:107C500044008320C110032481108324411051610A
:107C6000828097B7FF1F83C717632555ADCBFD17DC
:107C700017B6FF1FA301F66203D60601834707016B
:107C8000CC460A85230BF100EF20A07797E7FF1F72
:107C9000938707D49C4317B7FF1F1307675F975657
:107CA00001009386662988430A866C00EF10C001A4
:107CB000AA8451DD975501009385C522174501001F
:107CC0001305450BEF200179A68517550100130513
:107CD0006524EF2021782945EF20017C2685EFF0EF
:107CE0009FC1B5B793F725009DC3B7E70400BC4714
:107CF00041468145280882972555EFF0DFBF2808C7
:107D00009305F00FEFF05FD81345240099B793F770
:107D1000150001459DDFEFF03FA31345140015BF8B
:107D20005C4D411106C688C317E7FF1F2322F7CA1F
:107D3000B7E7040083A70708170500001305E5E669
:107D40008297B24097E7FF1F2386A7C801454101EC
:107D5000828001119307700F2316F10006CE97E77A
:107D6000FF1F83C7B7C88DE7B7E7040083A7870D58
:107D700017B6FF1F034606576C0017E5FF1F035594
:107D800025C782973335A00097E7FF1FA380A7C6BA
:107D9000F2400561828041119397050122C406C615
:107DA00026C2C1872E8463D40702B7E40400FC54C2
:107DB00017B5FF1F03450553829719C1BC5482971D
:107DC0002165218DB240224492444101828093F783
:107DD00015008DC7B7E7040083A7471A17B6FF1F22
:107DE0001306464F97E5FF1F938585BF17B5FF1F05
:107DF0000345454F829713451400E9B793F72500D3
:107E000099CFB7E70400BC4F13060064894517B546
:107E1000FF1F0345254D82971345240065B793F74F
:107E200085009DC7B7E7040003A8871A1307401F02
:107E300097B7FF1F83C7074B814613064006994536
:107E400017E5FF1F0355C5BA0298134584009DBF6F
:107E500093F745000145BDD7B7E4040083A7041894
:107E600017E5FF1F0355C5B88297BC4C1306006485
:107E7000914517B5FF1F0345E5468297134544001A
:107E800091B797E7FF1F83D7A7B66396A70217E7B7
:107E9000FF1F2310B7B617E7FF1F231DC7B417E74F
:107EA000FF1F231AD7B42E86175501001305852806
:107EB000BE856F20215A17550100130525296F2013
:107EC000216E03574500011106CE22CC97E7FF1F14
:107ED00083D707B21755010013054527631EF70422
:107EE000C167F91717E7FF1F2324F7B037E4040031
:107EF00097E7FF1F23A007B07C4C894517B5FF1FEC
:107F00000345453E82977C4C914517B5FF1F0345BD
:107F1000653D829783C7913995C78547A307F100CF
:107F2000832744171306F1008545130550308297C7
:107F3000175501001305C515EF208166F240624414
:107F40000561828097D7FF1F83C707591755010026
:107F50001305C518F5F38547A307F10083274417D8
:107F60001306F1008545130550308297175501001F
:107F700013054514D1B77D15954763ECA71817571E
:107F800001001307A70D0A053A951C41011122CCE7
:107F900006CE26CABA972E8482871755010013058C
:107FA000651BEF20E15F29AA03C725009947631DE0
:107FB000F7002E85EFF0FFF08345640017550100B0
:107FC0001305451AEF200149238C0138175501008C
:107FD0001305051BF9B703C7250095476317F7027B
:107FE000C16717E7FF1F0357A7A0F91703D5A5001F
:107FF0006305F702B7E7040083A7C71782971755F1
:1080000001001305E518EF20A1598547238CF138AD
:10801000175501001305451A69B797E7FF1F239904
:10802000A79C83D7E500B7E40400096617E7FF1FA4
:108030002311F79C83D705011306069017B5FF1F80
:108040000345452A17E7FF1F2316F79A83D7250113
:10805000A14517E7FF1F2310F79ABC4C8297BC4C31
:1080600013060064914517B5FF1F0345A5278297A6
:108070000356E4008355A40017550100130585122B
:10808000EF20413D59B7175501001305A51311BF46
:1080900083C525009147639AF5028547175501006E
:1080A0001305C513A307F100EF20814FB7E70400C4
:1080B00083A747171306F1008545130550308297B3
:1080C000F2406244D244056182809947639EF50084
:1080D0002285EFF01FDF834564001755010013056B
:1080E0006508EF202137E9BF9547639FF500834777
:1080F0001400175501001305650EE39407EA1755A0
:1081000001001305650F71BD175501001305450FDB
:10811000C9BF82806D712324811023261110232270
:108120009110328401CD89476306F5028320C11086
:10813000032481108324411051618280175501006E
:108140001305C50CAE84EF20A145A2852685EFC09E
:10815000FFBDE9BFB7E70400FC4728008297175529
:1081600001001305650BEF20A1438347810029C05F
:108170001307000B638EE7001387A7051377F70F2C
:108180008D4663E7E602A2852800EFD0EF9379BF22
:108190008547E3FD87F883459100174501001305E6
:1081A000A5F2B335B000238EB120EF20A12ABDBFC8
:1081B00003479100A207D98F35671307D755638D01
:1081C000E7066366F7022D671307B7556381E70675
:1081D00031671307C7556386E70429671307A75557
:1081E0006392E702A2852800EFD02FBE81B73967DE
:1081F0009306E7656383D70663E9F6001307E7553F
:108200006388E704A285280099B73D679306F75570
:10821000638AD7041307F766E396E7FEEFD06FD3C0
:1082200031B70146A2852800EFD0CFA901B7A285BA
:108230002800EFD00FB8DDBD8947E3F987EE93053D
:10824000E4FFC205C1811305A100EFA0FFCEF9BD77
:10825000A2852800EFD02FB8D1BDA2852800EFD08D
:108260000FC1E9B5EFD02FC9D1B5411122C417B460
:10827000FF1F13046408AA8617560100130686DF41
:108280002285C14506C6EF20A1320357440097B7A7
:10829000FF1F938767072393E70003576400239426
:1082A000E700B240224441018280011106CE22CC77
:1082B000EFF0BFFB37E404008327841417B6FF1FD9
:1082C00013068603D54501458297832784179305B6
:1082D000F1001305503082978347F100A1C7A3072F
:1082E0000100832744171306F1008545130550301C
:1082F00082978327441717B6FF1F1306E600CD4564
:108300001305703082978547A307F1008327441730
:108310001306F1008545130550308297F240624400
:10832000056182808327441717B6FF1F1306C6FD19
:10833000CD4513057030D5B761712324811A37E418
:108340000400832704082326111A2322911A2320CC
:10835000211B232E311917050000130505A4829750
:1083600017B9FF1F130909F8994785442300A9008D
:10837000231CF100975501009385C5D8930740064B
:10838000174501001305059F231CF10823089100E0
:1083900097D9FF1F9389A924EF20C10B83D509002A
:1083A000175501001305C5CDEF20C10A2945EF205F
:1083B000A10E03D509008569EFF03FEB8327441731
:1083C000100885451305503082978327441717B648
:1083D000FF1F130666F3CD45130570308297832780
:1083E000441717B6FF1F130626F0B5451305603076
:1083F00082978327441730088945130510318297E7
:108400008327441730098945130520318297832734
:108410004415938509C80D45829783274415938594
:1084200009C811458297A3059100230691002308EE
:10843000910002CD230C0100832784163009914559
:10844000130570408297832784161306B100854573
:108450001305004082978327841670008545130515
:1084600010408297832784163008854513052040E5
:1084700082978327841610088545130550408297FC
:10848000832704157D558297832744137D55829752
:108490007D55EFA09FF28327440C8297EFA05FCF1A
:1084A0008327841417B6FF1F130606E5D54501453B
:1084B000829789471306700F814528092306F1002A
:1084C000EF90BFAF8D471306000881452808230CA5
:1084D000F108EF909FAE9147230CF1009737010010
:1084E0009387C77A984383C747003AC8230AF100A5
:1084F000EFD02FAC700085450545EFA0BFF23009E5
:108500009305700F0945EFA0FFF1300893050008AF
:108510000D45EFA03FF1100895451145EFA09FF0E4
:10852000C16717D7FF1F1307A74CF9171CC32322D6
:10853000070017B5FF1F1305A5DAEFA0DFED8327AE
:10854000C41D17D5FF1F1305254982973C480345D5
:108550000900854582978320C11A0324811A832448
:10856000411A0329011A8329C1195D618280C167FB
:1085700017D8FF1F0358C847F917630BF8062DC912
:10858000A5C9011126CAB7E4040083A7841222CC2E
:108590002E862315B10006CE2A8401478146ED457B
:1085A000428582972AC601ED17550100130585B64D
:1085B000EF10117FF2406244D24405618280FC4496
:1085C0000356A100A28582972C0017D5FF1F0355E3
:1085D0002542EFA09FEF79DD175501001305C5B4C3
:1085E000EF10117C83A7C412ED4528008297D9B7FC
:1085F0008280011106CE22CC2DC9854717B7FF1FF7
:10860000A309F7CE97B7FF1F238607CE37E40400F0
:10861000832784179305F100130550308297834711
:10862000F100A9CBA3070100832744171306F1002B
:1086300085451305503082978327441717B6FF1FCF
:10864000130686CAB5451305603082978547A30790
:10865000F100832744171306F100854513055030B8
:108660008297F24062440561828097B7FF1FA38220
:1086700007C849BF8327441717B6FF1F1306C6C68E
:10868000B54513056030E9BFC16717D5FF1F035516
:108690002536F9176307F500B7E7040003A3C717EA
:1086A0000283828001118547A307010017D7FF1FAE
:1086B000230EF732B7E7040083A7471706CE130649
:1086C000F1008545130550308297F24005618280A4
:1086D000EF921F8A2A8408452E89B28909C900C1F0
:1086E000970500009385C5746105EF008101814401
:1086F0007D5AEF10C00963C3A4048144EF10200A1F
:1087000063C6A40497D7FF1F9387072F9C43DC47BA
:10871000B307F94091872302F4006381090483279A
:10872000C900B307F4409587A302F4001C4C89C725
:108730009C4799C3228582976F90DF865C4413978C
:1087400014008504BA972390470165B71C48139716
:1087500014008504BA97239007004DB7832789003A
:108760000547B307F4409587A302F400835704003C
:10877000638EE7028DC309476384E7040D47E397DF
:10878000E7FA975701009387E7FB1CCC9757010046
:10879000938747FC11A897570100938727C21CCCE9
:1087A00097570100938787C25CC849B79757010064
:1087B0009387C7AD1CCC97570100938727AEEDB7C1
:1087C000975701009387C7FC1CCC975701009387EC
:1087D00027FDD9BF85E1EF924FFB00461844834740
:1087E000940075839D8B6315F700EF00501C48C4FF
:1087F0006F90EFFB8280EF92AFF713893500C16471
:1088000042094111AA890144F11413590901054A89
:108810002EC6EF00D077B2456346A4000145410162
:108820006F904FF883A7090013171400BA9783D7E6
:1088300007006388B7006394970063742A010504F6
:10884000C1BF0545E9BFEF92CFF1AA892E89328BCE
:10885000B6843A8ABE8AEF80204C55C12685EF1037
:1088600030368D4763E5A7007D556F900FF383DBAE
:108870004400EF00D0772A84EF00B07893077400AB
:1088800031443305850263C5A702EF005076EF003F
:1088900010762A84EF00F076930774003144330594
:1088A000850263CDA702EF0090749307450019A8D5
:1088B000EF003075330585021307F0179307C017D3
:1088C000E357A7FC2D55E3C277FB63000B02D68666
:1088D0005286A6854A85EFE0106341BFEF007072B3
:1088E000330585029307C5FFF1BF83274900138530
:1088F000C90083D52700EFF01FF071F9B5B76955AE
:10890000ADB797D7FF1F239BA70E97D7FF1F93875E
:10891000A70E904381470C463307F5004207418379
:108920006393B70082805446139847008507C29628
:108930002390E600D5B797D7FF1F9387E70B9C439B
:1089400003C58700828017D5FF1F0355250B828042
:10895000EF92AFE3C1671387D7FF6307E502636850
:10896000A700F117630EF50001456F904FE41387E0
:10897000E7FF630EE500FD171D8D13351500F5B7F4
:10898000EF40003D7D15D5BFEF40801AE5BFEF40B9
:10899000E018CDBFEF926FDF4111AA8401442EC6CB
:1089A000EF00F05FB2456346A400014541016F90BE
:1089B0000FE09C48131514003E9583570500E3878C
:1089C000B7FE0504E9BF03485500814693F7F60F4B
:1089D00063E5070181473E8582805845939756009D
:1089E000BA9703D727006316B70003D70700E3043D
:1089F000C7FE8506E1BF8346450001479377F70F21
:108A000063E4D700814711A81C45131657000507DA
:108A1000B29703D60700E313B6FE3E858280EF923D
:108A20002FD593170501C18797DAFF1F938ACAFCD8
:108A30006355F00883A70A00C0479C47035704000A
:108A4000198D420541816366F500014422856F90CE
:108A50006FD512052A94DDBFDC4713944900014A03
:108A60003E94834744006341FA02014A834754001D
:108A70006347FA028509C20993D9090183A70A004D
:108A80009847E3EBE9FCD1B71C4413195A00A685BB
:108A90003E994A85EFF01FF011ED050AD9B75C4405
:108AA00013195A00A6853E994A85EFF0BFEE19E1E9
:108AB000050A6DBFE30009FC51BFAA8481497DBF4F
:108AC000EF92AFCC1C452A8481E79307C5001CC5F3
:108AD0001C44231204001CC09307F00F63E9B70085
:108AE00093F5F50F2285EF10B0136F904FCC939450
:108AF0000501C167C18063F7F500A6852285EF10E7
:108B0000D015E5B7C18193F5F50F2285EF1050110F
:108B1000A6852285EF101012C9BF97D7FF1F938734
:108B2000A7ED884382801C4599C797D7FF1F23A5CF
:108B3000A7EC014582807D55828097D7FF1F9387E0
:108B4000A7EB984383474500484792073E958280AC
:108B5000EF92AFC3617100451C183EC6B707800194
:108B60003EC81C183ECA8357440002CE02D002CC35
:108B7000231EF100834784002A8902D22301F102D7
:108B80003C083ED402D6EFF05FFB83570500231666
:108B9000F102EF30706B2307A1025C4003556400C3
:108BA000F18313F717008347F10252055181F99BB6
:108BB000D98FA307F102EFE0702639C5AA840355C7
:108BC0000500EF80401683D704002AD26800231CDA
:108BD000F10083D72400231DF1001C4803D6470071
:108BE0008C43EF1010028347B400CA861746010079
:108BF000130646638117A305F4006C004810EFE0EC
:108C000090305D616F90AFBA2155E5BF1C45B1CF83
:108C100003C5A700894613576500630BD7028D462D
:108C2000630ED70285466300D7021307400633055B
:108C3000E50203C7B700418B15CB83C7B700BD8BD7
:108C40003355F54082801375F5031307803EC5B791
:108C500009671375F50313070771D1BF372709009B
:108C60001375F5031307077CD9B701458280EF928E
:108C7000CFB103A98500630509048347B900AE8419
:108C800093F7070E91CF03459900930520030D81BB
:108C90000505B305B50288446105EFF0B0320DA0BB
:108CA0002E85EFF0BFF62A8401CD11238325C9005C
:108CB000B307B54063F887002E94B305A440E1FDE7
:108CC0006F90EFAE8545C1BFEF922FAC2A8403D5DC
:108CD0000500011132C636C43AC22EC002CA02CC07
:108CE00002CEEF80400482452ACA22852ECCEFF0C6
:108CF000DFE403570500231EE100EF30F054A246E5
:108D000032469247230FA10036874C08B28622854F
:108D10000146EFF05FB305616F906FA9EF92EFA688
:108D200061711C183EC6B70780013EC81C183ECAB8
:108D30003C0800453ED4AA8402CC02CE02D002D226
:108D400002D6EFF09FDF8357050035592316F10255
:108D5000EF30904F2307A10209C48357440091E7E5
:108D600021594A855D616F908FA4035564005205B7
:108D70005181EFE0B00A2A8965D58347B40093F7A3
:108D8000070E89C713058401EFF05025835744006F
:108D9000231EF100834784002301F1025C40035548
:108DA0000900D98313F7070883471102231CA10088
:108DB00093F7F707D98FA300F10283572900231DEA
:108DC000F1005C40F18313F717008347F102F99B30
:108DD000D98FA307F102EF7010752AD251D18347C2
:108DE00094006800139757008347B400FD8BD98F18
:108DF000A305F4001C4803D647008C43EF106060C5
:108E0000A687174701001307E741740005464C1079
:108E10002685EFF05FA32A8929D58347B400A6856C
:108E2000FD8BA305F400EFF09FE425BFEF92EF95D3
:108E3000832485FE2A8441112685EFF03FDD834798
:108E400034FF93F7070E9DC32AC62685EFF05FD047
:108E500019C9834734FFB245FD8BA309F4FE81C5D0
:108E60002285EFF0301641016F906F946DDD8327FE
:108E7000C4FF2685829765F9834734FF93F7070E71
:108E800081C72285EFF09015032584FEEFF01FE9DE
:108E9000D9BFEF928F8C9C4141112A8903C70700EB
:108EA00089472E8493566700638CF6020D466382D1
:108EB000C6049307F0076302F7022E85EF10A06047
:108EC000AA848149C16B130C490097D7FF1F938770
:108ED000A7B29C43984763ECE90241016F90AF8BC6
:108EE00003D745008547E3FAE7FE2E85EF10806142
:108EF000C1BF03D74500E3F2E7FE2E85EF10A05C6B
:108F0000AA842285EF10805DC204C98C5DBFDC4756
:108F10000355A900139A49003E9A93170501C1878A
:108F2000635DF00083570A006395A70263E574034D
:108F30008327CA00034D5A001DA0A1672167A98F8E
:108F40001307F7EFE374F7FE63950900EFF05FA0F6
:108F500071FD85099DBF83278A00034D4A00835D0B
:108F6000A90003576900216A138BC7003AC6814ADA
:108F700033CA4D01631E5D0197D7FF1F938747A832
:108F80009C43E1DBA2866286814526858297D1B724
:108F9000A1679387F7EF930C4BFF63F04703B2454C
:108FA0005A85EFF05F8519CD03278B00104719CA4A
:108FB00010436380C4023107D5BFEE856685EFF0AC
:108FC0007F9D71FD93861A0093FAF60F130B0B0227
:108FD00055B7835644005C43E3EDF6F622853AC666
:108FE000EF10603DA1679387D7042A8A035D440090
:108FF000324763E897008347D90093E707F8A30651
:10900000F9001C4766852286E2858297C16708447D
:10901000FD17337AFA00529508C02312A40115BF38
:1090200097D7FF1F9387479D9843814715C31447E0
:10903000814763FFD500939745004C47BE9519C9FA
:1090400003C7550081476375E600DC451606B297F5
:109050003E85828003C745008147E37BE6FE160616
:109060009C45F5B7EF82DFF0AA892E8A814497DA12
:10907000FF1F938A6A9883A70A00984763E4E40075
:109080006F805FF2DC471394440001493E9413BBA8
:10909000140083474400634BF900014913BB1400DB
:1090A00083475400634FF9008504F1B708449317D0
:1090B00059005287DA860146A2853E9582990509B4
:1090C000C9BF4844931759005287DA860546A285DE
:1090D0003E9582990509E9B7EF823FEB814517F587
:1090E000FFFF1305255F97D7FF1F23990790EFF028
:1090F0007FF76F80DFEB97D7FF1F9387E78F9C4346
:1091000081CFEF829FE8814517F5FFFF1305855C4E
:10911000EFF05FF56F80BFE98280EF827FE537E493
:1091200004008327841241112315E100AE8932899E
:10913000368A3A8681460147ED45AA8482972AC637
:1091400021C50356A100D285EF1061258327C413E2
:10915000CE8526858297058915C58327440D23145E
:10916000210101462C00268582972A8401C9B7E790
:10917000040083A7C712ED4528008297228541018C
:109180006F805FE24944E5B76554CDBF5C41FD1790
:109190005CC18280EF827FDFB7E70400FC5F8297CB
:1091A00095473305F50281450D816F805FE0EF82C1
:1091B000DFDDB7E70400FC5F829795473305F502D2
:1091C0000D816F80DFDEEF825FDCB7E7040083A7ED
:1091D000870B0355050082976F807FDDEF82FFDAF2
:1091E000035505003287AE8617A6FF1F0356E61704
:1091F00097D5FF1F93850581EFF03FF26F803FDB2E
:10920000EF82BFD8B7E7040083A7C71782976F80A4
:109210001FDAEF829FD7B7E7040083A7871397C5AC
:10922000FF1F9385257E829701456F805FD8EF826F
:10923000DFD5B7E7040083A7C71F814517A5FF1F28
:109240000355A50E82976F809FD6EF821FD4B7E794
:10925000040083A7871397C5FF1F9385A57B82977B
:1092600001456F80DFD4EF825FD2B7E7040083A7A8
:10927000C71F814517A5FF1F0355251182976F80D2
:109280001FD3EF829FD02E85EF600055EF60900DC9
:109290006F80FFD1EF827FCFEF60D0176F803FD11B
:1092A0005C49E1175CC95CC583572501A1072319F7
:1092B000F50083570501A1072318F5008280F147C7
:1092C0003305F50297C7FF1F9387C7769C433E95EA
:1092D00082808D476317F60603D74600854763F201
:1092E000E706EF829FCA368536842E89EF10A01DCF
:1092F00039C18357440093140501C18063ED97027F
:109300002285EF10401CFD14231294009307A00245
:10931000630EF5009307B0026301F5029307900214
:10932000631BF5002285EFC0B07E31A00146CA85DF
:109330002285EF80000F6F809FC72285EF001059B4
:10934000DDBF828097C6FF1F9386066F9C42014552
:1093500099CF9843D44217C6FF1F232FE66C63961C
:10936000D70097C6FF1F23ABE66C1385C7FE82802C
:10937000EF82BFC1E9267144330585029145EF7044
:10938000606201E565556F809FC297C7FF1F23A1EB
:10939000A76A7526330585029145EF70A0607DD1DF
:1093A00097C7FF1F23A8A768592E97C7FF1F239BA6
:1093B000A766712697C7FF1F2397A76697470100E7
:1093C000938787EB17C7FF1F2322F76697070000D5
:1093D000938747ED17C7FF1F2328F764014565B73B
:1093E000EF82BFBAAA8517C5FF1F1305A563EF104B
:1093F00060216F80DFBBEF825FB9EFF07FFEEF107F
:10940000E02197C7FF1F938727639C4381CF138772
:10941000C7FE09CB83D5C7FF17C5FF1F13054562DC
:10942000EFF0403A6F80BFB8EF823FB6EFF09FF1A8
:1094300019C9834785002A8493F7070499E70355E0
:10944000E500EFF05FFB6F809FB68347C500930494
:10945000450117C9FF1F1309295E85E3832709000A
:109460005CC997C7FF1F23A9975C83274900E1FFC9
:1094700097C7FF1F23A4975CF9B7FD172306F500D4
:109480006105EF60E07E8307840063CB07048347B8
:10949000840093E707F82304F400B7E704009C5F17
:1094A00082974205A94741813375F50283478400BD
:1094B00093F707FCC98F2304F4008347D4003E953B
:1094C0001C402318A40089CF984319CB8347C400BC
:1094D0005040814585073305F502420541810297D9
:1094E000832709005CC897C7FF1F23A797548327CA
:1094F000490089E797C7FF1F23A297548347C400F9
:10950000B9D38355040117C5FF1F13056553EFF049
:10951000602B15BFEF827FA797C7FF1F93878777C1
:109520009C4701448583858B81EFAE84B2853A8662
:10953000EF1020142A8409C5EF10200B829408CC68
:1095400022856F80DFA6EF82BFA241112E8932C62D
:10955000AA89712C324713060502CA8697050000B6
:10956000938525D617C5FF1F1305C54BEFF09FFA4E
:109570002A8429CD9304C50065261946AA85268527
:10958000EF00306885452685EF001065174501001E
:10959000130545CC4E95834505002685EF005068A0
:1095A0005C4831468145A1075CC85CC483572401EF
:1095B000E1172319F40083570401E1172318F4007D
:1095C0001C4C3E85EF807F9FA3042501228541012D
:1095D0006F805F9DEF827F9B4111AA842EC632C4AB
:1095E000EF100003004DB2452246834784000CC0B3
:1095F00050C093F7F70393E707042304F4002318FC
:1096000004002685EF00707E83479400A946231747
:10961000A40013D7370005073307D7029D8B8507B2
:109620002306F400A306E40083C70401D848850795
:10963000230FF7FE17C7FF1F130707405843232ABE
:109640000400930744011DEB17C7FF1F2328F73EB3
:1096500017C7FF1F2322F73E17C4FF1F1304443E02
:109660002285EFF0A00B1C44858B5D8D09E58145BB
:109670002285EFF0201541016F807F931CC317C72F
:10968000FF1F232DF73AC9BFEF823F9097050000D7
:10969000938565C40145EFF0DFBE01456F803F91C2
:1096A000EF82BF8EEFF01FBF6F807F908347C500B2
:1096B000A1E7EF829F8D2A840355E500EFF05FD28A
:1096C00015C98347840093F7F7FB2304F4001C407B
:1096D00091C7DC4381C74C4001458297EFF09FC69C
:1096E00017C5FF1F1305C535EFF0400F0355E40004
:1096F000EFF07FD06F80BF8B8280EF821F8997C78A
:10970000FF1F9387673397050000938525D217C500
:10971000FF1F1305E53223A0070023A20700EFE097
:10972000507E6F80DF881C4D91CBDC4381CBEF8274
:10973000DF858345070082976F807F87828097C788
:10974000FF1F938727329C4303C50700828097C77A
:10975000FF1F938727319C4303C51700828097C75B
:10976000FF1F938727309C4303C52700828097C73C
:10977000FF1F9387272F9C4303C54700828097C70D
:10978000FF1F9387272E9C4303C53700828097C70E
:10979000FF1F9387272D9C4303C55700828097C7DF
:1097A000FF1F9387272C9C4303C56700828097C7C0
:1097B000FF1F9387272B9C4303C57700828097C7A1
:1097C000FF1F9387272A9C4303C58700828097C782
:1097D000FF1F938727299C4303C59700828097C763
:1097E000FF1F938727289C4303C5A700828097C744
:1097F000FF1F938727279C4303C5B70011E11D4531
:10980000828097C7FF1F9387E7259C4303C5C70046
:10981000828097C7FF1F9387E7249C4303C5D70027
:10982000828097C7FF1F9387E7239C4303C5E70008
:10983000828097C7FF1F9387E7229C4303D50701C8
:10984000828097C7FF1F9387E7219C4303C52701A9
:10985000828097C7FF1F9387E7209C4303D547016A
:10986000828097C7FF1F9387E71F9C4303D567013B
:10987000828097C7FF1F9387E71E9C4303D587010C
:10988000828097C7FF1F9387E71D9C4303C5A701ED
:10989000828097C7FF1F9387E71C9C4303C5B701CE
:1098A000828097C7FF1F9387E71B9C4303C5C701AF
:1098B000828097C7FF1F9387E71A9C4303C5D70190
:1098C000828097C7FF1F9387E7199C438857828040
:1098D00097C7FF1F938707199C4303D5C702828050
:1098E00097C7FF1F938707189C4303D5E70219E129
:1098F0001305800C828097C7FF1F9387A7169C4390
:1099000003C50703828097C7FF1F9387A7159C4352
:10991000C85B828097C7FF1F938747148843828064
:1099200097C7FF1F9387C7138843828019E17D552E
:109930008280F5DE984265DFFDD917C7FF1F130748
:1099400067351847AA877155058B6319072203C528
:1099500007001547E37DA7FC03C737001305F00593
:109960007D171377F70FE364E5FC03C35700E300AB
:1099700003FC83C86700E38C08FA03C777004945F6
:1099800079171377F70FE364E5FA03C7A7001148C7
:109990001305F7FF1375F50FE36BA8F803CE9700D7
:1099A0000D481305FEFF1375F50FE362A8F803C811
:1099B000B7006309080065181378F80F1305600DE8
:1099C000E36705F703C5C700794879151375F50FE7
:1099D000E36FA8F403C8D7000D457D181378F80F7E
:1099E000E36705F503D80701930E401751184208A5
:1099F00013580801E3ED0EF303C8E7007D18137850
:109A0000F80FE36605F303C827017D181378F80FF4
:109A1000E36F05F103C88700C54E75181378F80F7A
:109A2000E3E70EF103D86701856E938EBEE06D18F3
:109A3000420813580801E3EC0EEF03D847016D18F4
:109A4000420813580801E3E40EEF03D887017918A0
:109A5000420813580801E36C05ED03C8A7017D18FF
:109A60001378F80FE36505ED03C5B7011D487D15B3
:109A70001375F50FE36DA8EA03C5D7017148791591
:109A80001375F50FE365A8EA03D5E7011308E00FA6
:109A90007D1542054181E36CA8E803C507024948EA
:109AA00079151375F50FE364A8E8C85301C937C8E1
:109AB00034005915130858BFE36BA8E603A88702C2
:109AC00037C53400130555BF5918E36205E717C5BC
:109AD000FF1F2327C5F803C6050117C5FF1F232352
:109AE000F5F80545E375C5E403D82501D04933767B
:109AF0000603E31E06E203C61501E30A06E217C6E3
:109B0000FF1F232DB6F483C5270001466387A500F8
:109B100003C61700F1453306B60283C70703930552
:109B2000C00272971A071307C70516031A979608FB
:109B30004697B387B70241553E9732974207418314
:109B4000636EE802EF826FC43685EF60D06FEFD0AE
:109B5000B0212A84EF80B01D2A94EFC090252A946A
:109B6000EF7040072A94EFF0BF802A94EF205063F3
:109B70002A94EF50406622956F806FC38280EF82F7
:109B8000CFC04111A307A100EF80801E9305F10013
:109B900017050000130565B9EFF0CFCC0145410171
:109BA0006F80EFC0EF82EFBB17C4FF1F1304840E5A
:109BB0000328840079599368180097C4FF1F23AFC6
:109BC000140D13781800631E0800BA84BE89368B02
:109BD000328A2E89AA8AEFE01FD67D15269509E5DF
:109BE00031594A856F806FBBEFE0FFD47D15269514
:109BF000A167E357F5FE97C7FF1F9387A7409843D8
:109C00003E8C814B11C70145EFC0B03E933B150020
:109C10004A85DA865686D285EF7070372A8911CD4B
:109C20001C44F99B17C7FF1F232AF70683270C0044
:109C3000CDDBE3880BFA82976DB7268597C7FF1FA8
:109C400023AC0704EFE0FFCB4146CE8517C5FF1FCD
:109C50001305C50DEF00A174EFA070080325040BD8
:109C6000EFA0700A0545EFA070100545EFF03FF139
:109C70008DBF97C7FF1F9387E7019C47858BD5C78B
:109C8000EF82AFB017C5FF1F1305850897C7FF1FE9
:109C900023A2070097C7FF1F23A0070097C7FF1F36
:109CA00023AE07FEEFE09033EF40C002EFE0F00A92
:109CB000EFE0700F97C7FF1F938747FC9C4381C756
:109CC0000545EF60B03397C7FF1F9387E7E49C43D8
:109CD00089C741657D15EF50A06BEFC0703AEFA0CA
:109CE000F00097C7FF1F9387E70F9C431397170157
:109CF00063540700EFC0A04597C7FF1F23A80702C2
:109D000097C7FF1F23A6070297C7FF1F23A40702B9
:109D100097C7FF1F23A20702EFF09F984923EFF098
:109D2000AFBBEFC080676F808FA8828097C7FF1F8F
:109D3000938747F688438280EF822FA5EF60B07E3D
:109D4000EF7080006F80AFA6EF828FA22A84930409
:109D5000140201112E85B289A685214636C63A899C
:109D6000EF0081611DE1B24638082686CE851305D5
:109D70009404EF40604321462C084A85EF00C15F00
:109D80001335150005616F80EFA10145E5BFEF8236
:109D9000CF9F9305450617C5FF1F1305E5CCEFE0E0
:109DA00070226F80CFA0EF824F9E41112EC6EFF040
:109DB0000FC0B24588C141016F806F9FEF824F9BFA
:109DC000AA842E84EF605078AA8985452285892D42
:109DD00083C7E4011389940899E313890403CE85AA
:109DE00022853D2D2146930519022285192D97C7FD
:109DF000FF1F938727EA8C432285EF00E068214606
:109E0000938584022285F52B6F80CF99EF826F9521
:109E10003971EFC0E04E9305400645EDEF60D06F1D
:109E2000630E051097C7FF1F83C7C7C513B7170079
:109E300097C6FF1F2388E6C4014489CFC16417C9B0
:109E4000FF1F130929E59309400EFD14EFF03F9819
:109E50006348A408EFF0AFB54169B7290900096A62
:109E6000FD7A2A8B81447D199389F97B130A0A7143
:109E7000938A8AC7EFF0BF9563D5A4041304400EFC
:109E8000B387840217C7FF1F1307C7E00324070B1C
:109E90003E948357C4016386270918403307EB407B
:109EA00063EAE900834744008507B3874703D697F1
:109EB0006369F706014681450945EFF0CFE8AA8BB3
:109EC00029E1EF20105A8547631FF50489659385C2
:109ED000057117C5FF1F130525B9EFE0B00EA1A846
:109EE000B30734030327090BBA9703D7C7016308E5
:109EF000970003C75700A38207002382E7000504E9
:109F0000B1B79305C5002285EFF05FEB5E85228631
:109F10009735010093854535EFF0CFEB5E85EF0077
:109F2000E06F850481BF97C7FF1F9387A7D69C4723
:109F30008D83858BC1FF21616F802F86014685450A
:109F4000094502D002D202D402D6EFF0CFDFAA84B4
:109F50007DD1EFC0203A1389C4002A8481454A8507
:109F6000C1210C4041464A85692983294400638800
:109F700009084E8502D802DA02DC02DEEF00816AAF
:109F80002ACE141005462C0808184ECCEF40601954
:109F90001375F50F2DE58355840093E525004A855B
:109FA0006D2911460C104A85A929014697350100F3
:109FB0009385052C2685EFF0EFE12685EF000066FE
:109FC0005C40B5DB014685450D45EFF0CFD7AA844F
:109FD0003DD148401389C400EF00C1642AC64A85B8
:109FE000C5263246636AC5004C404A851929014698
:109FF00081452685EFF00FDE26850D252DBF835583
:10A00000840071BFEF727FF897C7FF1F938787C8DF
:10A010009C4719CD93E7870017C5FF1F1305C5A4FB
:10A0200017C7FF1F232CF7C6EFE060786F703FF86B
:10A03000DD9B17C7FF1F2323F7C6EF2090427DF556
:10A0400017C5FF1F130545A2EFE04079C5B7EF72B2
:10A050005FF14169AA892E8AB28A368BBA8B814414
:10A0600017CCFF1F130C0CC3930C400E7D19EFF09F
:10A070000FF663C4A40001442DA033849403832706
:10A080000C0B3E948357C401638027055A87D686FC
:10A090005286CE8513050403EFF01FCB11C5238034
:10A0A0000B0022856F707FEF8347F40191CF5A87B1
:10A0B000D6865286CE8513059408EFF0FFC809C5F1
:10A0C00085472380FB00F1BF850455B783574500C2
:10A0D000638D0716EF72DFE901112A84ED2619C599
:10A0E0008547630AF50405616F70DFEBEFC040211F
:10A0F0007DF9835744004947ED9BE396E7FEC14550
:10A1000022854524AA842285F52E0357440002CED9
:10A1100091472A896317F700228539293C082ACC00
:10A120003ECEEFC0201D5C55DDDF74084A86A68553
:10A13000054582974DBF03574400D147E3F5E7FA41
:10A14000032A0400C169014997CAFF1F938A8AB490
:10A15000130B400EFD19EFF08FE76344A90C228525
:10A16000032A04008D26A1452A8922851D2CAA8454
:10A170002285D92614402A86AA8978082685CA8588
:10A18000EFF0FFECAA8425D103C7F40189476315DA
:10A19000F7008347C101A1DB5546D28513856400D2
:10A1A000EF00E11F0145EF60103801C583D7C401FE
:10A1B000B1EB97C7FF1F9387E7AD9C4793551900F5
:10A1C000858913D73700058B11CB8983858B6397DE
:10A1D000B70001452EC6EFF0FFE2B2454E85EF60B5
:10A1E000703C0346C1012A84937519002685EF70DF
:10A1F000703131C92685EF607037268511C0014561
:10A20000EF60D061EF20F0258547E31EF5EC83C7B2
:10A2100054001307F00FE388E7EC8507A382F400EE
:10A22000D9B5B304690383A70A0BBE9483D7C401CD
:10A23000638937015546D28513856400EF00C11349
:10A2400071D1050909BF5DDC5DBF8280EF725FD20D
:10A25000EF60902C11CDC164014417C9FF1F130991
:10A2600069A39309400EFD14EFF06FD6634AA40072
:10A2700017B5FF1F1305457FEFE060536F709FD246
:10A28000330534038327090B3E958357C501638645
:10A29000970023120500EF60702D0504F1B797C7F2
:10A2A000FF1F9387279F9C478D83858B99EBEF72C8
:10A2B000DFCD17B5FF1F1305257BEFE020526F7030
:10A2C0001FCF8280EF727FCC97050000938545B445
:10A2D00017B5FF1F13054579EFE0A0426F703FCD22
:10A2E000EF72BFCA8841B7E70400BC5B05054205B1
:10A2F0004181829709C585472300F50005056F70E8
:10A300001FCB83C7F5FF2E858507A38FF5FE8280BF
:10A3100083C7F5FFFD1793F7F70FA38FF5FE99EBB2
:10A32000EF72BFC6B7E70400BC571385F5FF8297ED
:10A330006F70FFC782801C41035745008D8FBA950F
:10A340001CC12312B5003E85828093D78500A205EB
:10A350001441DD8D835745001387E6FF18C1890737
:10A360002312F50013D685004111238FB6FEA38F6B
:10A37000C6FE4101828018419307F7FF1CC1835735
:10A38000450085072312F500A30FB7FE828083578F
:10A3900045008D8F2312F5001C41BE950CC12E8502
:10A3A0008280AA8703D7470008410D8FAA95239280
:10A3B000E7008CC38280184108453305A74082809E
:10A3C00083574500035765001D8F1C4108453385A1
:10A3D000A7403305A7408280EF723FBB41112EC6D4
:10A3E0002A84EFF0FFFDB2456373B50001A08357E7
:10A3F00044000840BE952312B4003E9541016F70A1
:10A400001FBBEF729FB841112E84B28532C6EFF0A8
:10A41000BFFC3246A285EFF0907841016F703FB9E2
:10A42000EF72BFB62E848545EFF01FFB2300850039
:10A430006F70FFB7EF727FB541112317B1008945E7
:10A44000EFF09FF98347E1002300F5008347F10017
:10A45000A300F50041016F709FB5EF721FB393D752
:10A460008500A2054111DD8D2317B1008945EFF06C
:10A47000BFF68347E1002300F5008347F100A30006
:10A48000F50041016F70BFB2EF723FB013978501C5
:10A4900093D78501C166938606F0D98F13D78500BF
:10A4A000758FD98FA2053707FF00F98D4111DD8D1A
:10A4B0002EC69145EFF05FF26C001146EFF0306E62
:10A4C00041016F70DFAEEF725FAC1C41854503C484
:10A4D0000700EFF0DFEB22856F707FADEF72FFAA10
:10A4E0001C414111894503C7070083C71700230793
:10A4F000E100A307F100EFF09FE90355E1004101FE
:10A500006F70FFAAEF727FA81C414111894503C7F4
:10A51000070083C717002307E100A307F100EFF04E
:10A520001FE78357E100410113D58700A2075D8D26
:10A53000420541816F70BFA7EF723FA50C414111E9
:10A540002A8411466800EFF0906591452285EFF06E
:10A550001FE4B247C166938606F01397870113D5AF
:10A560008701598D13D78700758F598DA20737073B
:10A57000FF00F98F5D8D41016F707FA31C45BE9573
:10A580000CC18280AE87944391E6584101EF0CC123
:10A590005CC1828003C7570013671700A382E700DE
:10A5A000B687D5B70CC3EDB7AA87084119CD1841B6
:10A5B000D44398C36313D500D8C32A8703465700F2
:10A5C0009376160081E6232007008280944381CA97
:10A5D0008C4203A847008CC363930601CCC3799ACD
:10A5E00014C3A302C7003687D1BF1C45DC471D8DAD
:10A5F000B777DBB6938777DB09853305F50242052C
:10A6000041818280F147B385F50248452E958280CD
:10A610008347450085072302F5008280EF72FF968D
:10A620002A8419E06F70BF9883474400E5DFFD1767
:10A6300093F7F70F2302F400F5F71C4403D7270024
:10A6400005072391E700DC4399C3228582974C4894
:10A6500089CD83475400898B99E71C4422859C4708
:10A660009C439C478297232A040000402320040037
:10A670004DBFEF729F918357250041112EC691E780
:10A680000144228541016F709F9203570500814765
:10A69000F146E307F7FEB385D702404585072E94C0
:10A6A0008345440008C4F5F5B247AA8481E7232A0C
:10A6B000040009A81C456C0022859C439C4382979A
:10A6C00048C85DDD85472312F400B247232004000B
:10A6D000231804002319F4005C485CC483D72400C9
:10A6E000FD172391F40071BFEF723F8A97B7FF1FE8
:10A6F00093878739884323260500232405004105D5
:10A70000EFE0C00D6F70BF8AEF723F8817B4FF1F74
:10A71000130484371C40411189CF9C472300B500A6
:10A720002AC65CC1EFF05FFC1C40DC4399C3324594
:10A73000829741016F70BF87034745001DEB584D5D
:10A74000AA877D550DCBEF725F841CC3DC4797B69B
:10A75000FF1F23ABE632F156130507012390D70004
:10A760009705000093858501EFD0B07901456F70A2
:10A770001F847D5582808280EF723F810111614686
:10A7800081452800EF707F8397B7FF1F9387C72FFE
:10A790009C4328009305F00FDC473EC6EFF0DFF640
:10A7A00005616F70DF8097B7FF1F9387E72D9C438C
:10A7B000D847A1679387C7026312F70A397106DE8B
:10A7C00022DC26DA80004AD84ED652D456D23285C0
:10A7D000B284EFF05FCFAA892685EFF03FD023182F
:10A7E000A4FC2685EFF09FCF2319A4FC2685EFF06B
:10A7F000FFCE83D744000A8A231AA4FC858393F7EB
:10A80000F70F230EF4FC8607BD0793F7073F3301CC
:10A81000F1408A8A01498347C4FD6365F902CE8508
:10A82000130584FC232C54FDEFF01FEE528113011D
:10A8300004FCF2506254D2544259B259225A925AEC
:10A84000216182802685EFF07FC993171900D69782
:10A8500005092390A7001379F90F75BF828097B778
:10A86000FF1F938767229C43D847A1679387A7025E
:10A870006310F70A397106DE22DC26DA80004AD836
:10A880004ED652D456D23285B284EFF0DFC3AA89B5
:10A890002685EFF0BFC4FD572318A4FC2685231995
:10A8A000F4FCEFF0BFC383D744000A8A231AA4FC48
:10A8B000858393F7F70F230EF4FC8607BD0793F704
:10A8C000073F3301F1408A8A01498347C4FD63652C
:10A8D000F902CE85130584FC232C54FDEFF0DFE252
:10A8E0005281130104FCF2506254D2544259B259BD
:10A8F000225A925A216182802685EFF03FBE93173B
:10A900001900D69705092390A7001379F90F75BF91
:10A91000828097B7FF1F938727179C43D847A1676B
:10A9200089076318F708397106DE22DC26DA800011
:10A930004AD84ED652D456D232853289EFF0BFB8BB
:10A94000AA894A85EFF09FB9835749000A8A2318DC
:10A95000A4FC858393F7F70F230CF4FC8607BD074F
:10A9600093F7073F3301F1408A8A8144834784FD8E
:10A9700063E5F402CE85130584FC232A54FDEFF031
:10A98000BFD85281130104FCF2506254D254425990
:10A99000B259225A925A216182804A85EFF01FB43F
:10A9A00093971400D69785042390A70093F4F40F8F
:10A9B00075BF828097B7FF1F9387070D9C43D847C9
:10A9C000A1679387E7046312F70A397106DE22DC78
:10A9D00026DA80004AD84ED652D456D23285B28476
:10A9E000EFF07FAEAA892685EFF05FAF2318A4FCB5
:10A9F0002685EFF0BFAE231AA4FC2685EFF01FAE2C
:10AA000083D744000A8A2319A4FC858393F7F70FA0
:10AA1000230EF4FC8607BD0793F7073F3301F1408F
:10AA20008A8A01498347C4FD6365F902CE8513050F
:10AA300084FC232C54FDEFF03FCD5281130104FC24
:10AA4000F2506254D2544259B259225A925A216158
:10AA500082802685EFF09FA893171900D6970509E5
:10AA60002390A7001379F90F75BF828097B7FF1F56
:10AA7000938787019C43D847A1679387C7046310D6
:10AA8000F70A397106DE22DC26DA80004AD84ED673
:10AA900052D456D23285B284EFF0FFA2AA8926851D
:10AAA000EFF0DFA3FD572318A4FC2685231AF4FC3E
:10AAB000EFF0DFA283D744000A8A2319A4FC858320
:10AAC00093F7F70F230EF4FC8607BD0793F7073FB4
:10AAD0003301F1408A8A01498347C4FD6365F90265
:10AAE000CE85130584FC232C54FDEFF0FFC1528169
:10AAF000130104FCF2506254D2544259B259225A02
:10AB0000925A216182802685EFF05F9D931719008C
:10AB1000D69705092390A7001379F90F75BF828096
:10AB200097B7FF1F938747F69C43D847A167DD0778
:10AB3000631BF702EF726FC5797132853284EFF0D3
:10AB40009F982AC62285EFF07F992311A1022285C2
:10AB5000EFF07F97B2452300A1022808EFF0DFBA9B
:10AB600045616F70CFC4828097B7FF1F9387C7F18D
:10AB70009C43D847A16793878704631BF702EF7252
:10AB8000CFC0797132853284EFF0FF932AC62285D7
:10AB9000EFF0DF942311A1022285EFF0DF92B2459E
:10ABA0002300A1022808EFF03FB645616F702FC067
:10ABB000828097B7FF1F938727ED9C43D847A167F3
:10ABC0009387A704631CF700EF722FBC01112800C4
:10ABD0008145EFF07FB305616F706FBD828097B7DD
:10ABE000FF1F938767EA9C43D847A1679387570263
:10ABF0006311F702EF726FB901113285EFF0BF8C6C
:10AC00002308A10081452800EFF01FB005616F7097
:10AC10000FBA828097B7FF1F938707E79C43D847F7
:10AC2000A1679387E702631FF702EF720FB6011166
:10AC300032853284EFF09F8AAA842285EFF01F8A42
:10AC4000854719E52285EFF01F884205B337A0003C
:10AC500028008145231891003ECAEFF0FFAA056144
:10AC60006F70EFB4828097B7FF1F9387E7E19C4333
:10AC7000D8479947631FF704EF722FB17971328576
:10AC80003284EFF05F842AC62285EFF03F852310DF
:10AC9000A1022285EFF03F832301A1022285EFF07C
:10ACA0009F82A301A1022285EFF0FF812302A1026E
:10ACB0002285EFF05F812313A1022285EFF0BF8090
:10ACC000B2452314A1022808EFF01FA445616F705C
:10ACD0000FAE828097B7FF1F938707DB9C43D8474F
:10ACE000A1679387C703631FF704EF720FAA7971F7
:10ACF00032853284EFF02FFD2AC62285EFF00FFE59
:10AD00002310A1022285EFF06FFD2311A1022285FD
:10AD1000EFF06FFB2302A1022285EFF0CFFAA3022E
:10AD2000A1022285EFF02FFA2303A1022285EFF082
:10AD30008FF9B245A303A1022808EFF0FF9C4561FB
:10AD40006F70EFA68280EF724FA401112A84EFF09A
:10AD50008FF7AA842285EFF06FF82285EFF00FF8C5
:10AD6000035744008D4763F5E7002285EFF00FF7A6
:10AD70002285EFF0AFF62800A685EFF0FF98056179
:10AD80006F70EFA297B7FF1F938707D09C43D847F8
:10AD9000A167FD076319F700EF722F9F3285EFF06F
:10ADA0009FFA6F70CFA0828097B7FF1F9387C7CDA0
:10ADB0009C43D847A167E5076311F706EF72EF9C44
:10ADC000797132853284EFF00FF02AC62285EFF0D8
:10ADD000EFF02285EFF08FF02310A1022285EFF033
:10ADE000EFEF520551812311A102228523020102B6
:10ADF000EFF06FEDA302A1022285EFF0CFEC230369
:10AE0000A1022285EFF02FECB245A303A10228088E
:10AE1000EFF09F8F45616F708F99828097B7FF1F0A
:10AE2000938787C69C43D847A1679387E703631935
:10AE3000F700EF728F953285EFF0FFF06F702F976C
:10AE4000828097B7FF1F938727C49C43D847A16789
:10AE5000938747046314F702EF722F937971328559
:10AE60003284EFF04FE62AC62285EFF02FE7B24595
:10AE70002808EFF07F8945616F706F93828097B7E4
:10AE8000FF1F938767C09C43D847A16793878702BA
:10AE90006316F702EF726F8F797132853284EFF0AB
:10AEA0008FE22AC62285EFF00FE2B2452300A1020D
:10AEB0002808EFF07F8545616F706F8F8280EF7299
:10AEC000CF8C0111EFF02FE0AA852800EFF0DF838F
:10AED00005616F70CF8D97B7FF1F9387E7BA9C43CB
:10AEE000D847A167D1076319F700EF720F8A32853F
:10AEF000EFF0FFFC6F70AF8B828097B7FF1F9387D7
:10AF0000A7B89C43D847A167C5076319F700EF723C
:10AF1000CF873285EFF0BFFA6F706F89828097B765
:10AF2000FF1F938767B69C43D847A167B90763198A
:10AF3000F700EF728F853285EFF07FF86F702F8703
:10AF4000828097B7FF1F938727B49C43D847A16798
:10AF5000AD076319F700EF724F833285EFF03FF6CC
:10AF60006F70EF84828097B7FF1F9387E7B19C4390
:10AF7000D84789476310F702EF722F81011132859C
:10AF800032C8EFF04FD4AA852800EFF0EFF7056143
:10AF90006F70EF81828097B7FF1F9387E7AE9C4366
:10AFA000D847A1678D076317F702EF621FFE0111F3
:10AFB00032853284EFF02FD113066100AA844C0051
:10AFC0002285EF20D00C2800A685EFF0EFF3056175
:10AFD0006F60FFFD828097B7FF1F938727AB9C436D
:10AFE00081CBDC4391C7EF625FFA82976F603FFCD1
:10AFF0008280EF629FF979713C08AE843ED2A165F0
:10B00000B7070A002A843ED448103C08DD053ED626
:10B0100036C432C63AC2EFD0BFAA12474810BA852A
:10B02000EFF00FC032464810B285EFF0AFC0A24635
:10B030004810B685EFF0CFBE501001478146A68577
:10B040002285EFD07FC845616F607FF6EF62FFF326
:10B0500001117C000329C501AE843ECAA165B70772
:10B0600007002A843ECC48087C00C5053ECEEFD0C0
:10B070003FA58345D9004808EFF08FBA5008014733
:10B080008146A6852285EFD03FC405616F603FF2FF
:10B09000EF62BFEF83C7950093F7F707A384F5002E
:10B0A000EFF0DFFA6F60BFF0EF623FEE79713C08BE
:10B0B000AE843ED2A165B70709002A843ED4481069
:10B0C0003C08938545043ED632C636C4EFD05F9F18
:10B0D000A2464810B685EFF0AFB432464810B285AC
:10B0E000EFF04FB5501001478146A6852285EFD07D
:10B0F000BFBD45616F60BFEBEF623FE983C795005D
:10B1000041112A8493F7F707A384F50032852EC6F0
:10B11000EFF0CFBC85672AC4637CF500EF50B040E8
:10B120002246B24509E9114781462285EFF07FECBE
:10B1300041016F60DFE701478346F501FDB7EF622C
:10B140003FE301113C003ECAB7070A003ECC3C0079
:10B150003ECE83C79500AA89328593F7F707A3846B
:10B16000F5002E84EFF08FB785676371F504A16554
:10B17000AA84938585044808EFD09F942685EF50D4
:10B18000903A2A891DE591454808EFF06FA9A685F8
:10B190004808EFF02FAACA854808EFF06FA80147CA
:10B1A00081465008A2854E85EFD01FB205616F60C1
:10B1B0007FDF81454808EFF0AFA603490902C1BF10
:10B1C000EF621FDB79711C103ECAB7070F003ECC3F
:10B1D000404D1C10AA84AE894808994532C636896C
:10B1E0003ECEEFD0FF8D32464808B285EFF04FA338
:10B1F00063040902A5454808EFF00F9E2546CA855D
:10B20000EFF0E019500801478146CE852685EFD042
:10B21000BFAB45616F601FD98355C4024808EFF08A
:10B220006FA10355E402814515C185478545630F2C
:10B23000F500C167FD179305F00F6309F5007D1553
:10B24000EF5020749305150093F5F50F4808EFF0C3
:10B250002F9D834504034808EFF08F9C834514031A
:10B260004808EFF0EF9B835524034808EFF08F9CCC
:10B27000835544034808EFF0EF9B69B7EF62FFD0B6
:10B2800083C795008146014693F7F707A384F5002D
:10B29000EFF01FF36F60BFD1EF623FCF79713E8453
:10B2A0001C103ECA2E89B7070F00A1653ECCFD05D4
:10B2B0001C10AA84480842C03AC23ECE36C432C6E8
:10B2C000EFD01F8032464808B285EFF06F95A24656
:10B2D0004808B685EFF00F9612474808BA85EFF098
:10B2E0006F9502486304080291454808EFF0CF8E3D
:10B2F0001146A285EFF0A00A500801478146CA8591
:10B300002685EFD07F9C45616F607FCA89454808DC
:10B31000EFF08F8C834704002300F500834714006F
:10B32000A300F500D1BFEF62BFC483C79500011130
:10B330002A8A93F7F707A384F5003285AE8432C6D4
:10B34000EFF0CF9932462A893285EFF0CF978567A3
:10B35000637FF900AA894A85EF50F01C2A8419E915
:10B36000114781464A86A6855285EFF09FC8056140
:10B370006F605FC39387E9FF93F7F70F0547E368B3
:10B38000F7FE8347F50195E78947E382F9FE834697
:10B39000F401528501474A86A685EFF09FC5A16753
:10B3A000D90748083ECC230A010002CEEFF0BFC205
:10B3B0007DBF639CE7008947639CF90093071020D9
:10B3C000231FF500EF50901AD9B70947E391E7FC26
:10B3D0008D47E39EF9FA2285EF50D03B97B7FF1FC8
:10B3E0009387C7899C4399E797A7FF1F9387C772E5
:10B3F0009C4389C703D50400EF60300C231F040071
:10B400002285C9B7EF627FB801113C003ECAB70779
:10B410000B003ECC3C003ECE83C795002A89328586
:10B4200093F7F707A384F500AE84EFF02F8B931703
:10B430000501C187635EF004A1652A849385E50256
:10B440004808EFD0EFE7A2854808EFE0BFFE97A7D6
:10B45000FF1F9387676C9C439DEF01449375F40F26
:10B460004808EFE0FFFB9355844093F5F50F48083B
:10B47000EFE01FFB9355044193F5F50F4808EFE00B
:10B480003FFA014781465008A6854A85EFD0DF8301
:10B4900005616F60DFB1416585460546A2857D1572
:10B4A000EF3070675DD95105EFD040271304400697
:10B4B0003344850265B7EF625FAD0111B70706003F
:10B4C0003EC683C7950021642A8993F7F707A384B2
:10B4D000F500AE8428009305A4040AC40AC8EFD07E
:10B4E0002FDE300001478146A6854A85EFD0CFFD8B
:10B4F000EFE02FF813049404480822CC230A01003B
:10B5000002CEEFF05FAD05616F607FAAEF625FA6CC
:10B51000C1642A89014497A9FF1F9389A977130A57
:10B520008002FD14EFE0AFAB6345A40001456F60FE
:10B530007FA7B307440303A7C90ABA9703D7070035
:10B540006306970083D72700638427010504D9BFCA
:10B550000545F1BFEF62DFA12A8A2E8999C123A098
:10B5600005008149814497AAFF1F938A6A52614B63
:10B57000EFE02FAD63C5A4004E856F60BFA233849A
:10B58000640383A70A003E948357040099E7630489
:10B590000900232089008504E1BF4146D2851305B7
:10B5A0004400EFE0705D65F9A289F5B7EF625F9C3A
:10B5B00039717C083ED4B7070A003ED67C083ED8D5
:10B5C00083C795002A8A328593F7F707A384F5008D
:10B5D0002E8932C6EFE09FF085676373F506324629
:10B5E000AA843285EFE03FEE8547AA8963EAA70483
:10B5F000A165938585042810EFD08FCC2685EF5068
:10B6000080722A8429E191452810EFE07FE1A68528
:10B610002810EFE03FE2CE852810EFE07FE0014701
:10B6200081463010CA855285EFD00FEAA167938713
:10B63000770448183EDC230A010202DEEFF0BF99CE
:10B6400021616F603F9681452810EFE07FDDA68580
:10B650002810EFE03FDE97B7FF1F9387679A9C4360
:10B6600091C7228563870900EFB0600C834504020F
:10B6700065B7EFB0200BDDBFEF629F8F83C79500EA
:10B680004111AA8993F7F707A384F5003285AE84A8
:10B69000328AEFE0BFE48567637BF5022A89EF50C9
:10B6A00080682A84914621C18347F5010547638359
:10B6B000E70291C70D47636EF702AD462DA09305D3
:10B6C000050303250A004146EFE0104B1DE141014F
:10B6D0006F605F8D9305950803250A004146EFE0F2
:10B6E000B049814679F94A86A6854E85EFF0DF9B01
:10B6F000F9BF83250A0013059408EF60600119C1A2
:10B70000C146D5B797A7FF1F938747579C4399E733
:10B7100097A7FF1F938747409C4389C72285EF6007
:10B72000A05479FD8547A30FF4002285EF80B05D1A
:10B730002285EF50A0634E8581464A86A685EFF0AC
:10B74000BF96A1679387570448003EC423020100B7
:10B7500002C6EFF05F88A5BFEF62BF8083C7950088
:10B760004111AA8993F7F707A384F50032852E8942
:10B77000B28AEFE0BFD685676370F50CAA84EF50FC
:10B78000805A2A841DE9416B014A97ABFF1F938BB6
:10B790006B50130C400E7D1B19A833048A0383A73A
:10B7A0000B0B3E948357C401638D6703050AEFE0DA
:10B7B0000F82E344AAFE954639A88357C5016392D8
:10B7C00097029305050303A50A004146EFE0D03A2E
:10B7D000994611E181462686CA854E85EFF0DF8CB9
:10B7E000A1A883A50A0013050403EF507072C14697
:10B7F0007DF12285231E9400EF80F0502285EF50CA
:10B80000E05697A7FF1F9387A77F9C438DCB23000C
:10B8100004022285EFA090614E8581462686CA8566
:10B82000EFF09F88A1679387070448003EC4230276
:10B83000010002C6EFF02FFA41016F600FF6894751
:10B840002300F402D1BF397106DE22DC4AD8800021
:10B8500052D456D25AD026DA4ED65ECE2E8A3289AD
:10B860002A8BEFD0DFF30605710541998A8A3301EF
:10B87000A140232224FC231404FCEFD05FF2834771
:10B880009A000605350593F7F7072315A4FCA304D2
:10B89000FA004A85232624FCEFE05FC493170501D4
:10B8A000C1876340F0025681130104FCF2506254D8
:10B8B000D2544259B259225A925A025BF24B216138
:10B8C0008280AA844A85EFE07FC1AA894A85EFE099
:10B8D000FFC0A1659385C5022A89130544FCEFD0FA
:10B8E0002F9E2685EFD0AF93854501C94A86CE8528
:10B8F000EFD06F8DAA8B15ED8945130544FCEFE061
:10B900003FB2A685130544FCEFE0DFB2CE851305F8
:10B9100044FCEFE03FB2CA85130544FCEFE09FB161
:10B9200001478146130644FCD2855A85EFD0CFB932
:10B930009DBF8145130544FCEFE09FAEA68513052E
:10B9400044FCEFE03FAFCE85130544FCEFE09FAE33
:10B95000CA85130544FCEFE0FFAD8144EFD03FE41E
:10B96000E3D0A4FC83A70B0113971400BA9783D5E7
:10B97000070089C5130544FCEFE0DFAB8504F9BF80
:10B98000797106D622D44AD000184ECE52CC56CA6F
:10B9900026D25AC8AE893289AA8AEFD05FE006055E
:10B9A000690541990A8A3301A140232A24FC231CFA
:10B9B00004FCEFD0DFDE83C7990006052D0593F761
:10B9C000F707231DA4FCA384F9004A85232E24FC39
:10B9D000EFE0DFB093170501C187634FF00052819C
:10B9E000130104FDB250225492540259F249624AA2
:10B9F000D24A424B45618280AA844A85EFE01FAE5D
:10BA0000A1659385A5022A89130544FDEFD04F8BCC
:10BA10002685EFD0CF80854519C5CA85EFC0BFFD0B
:10BA20002A8B0DE98945130544FDEFE07F9FA6852C
:10BA3000130544FDEFE01FA0CA85130544FDEFE0A8
:10BA40007F9F01478146130644FDCE855685EFD082
:10BA5000AFA771B78145130544FDEFE07F9CA68534
:10BA6000130544FDEFE01F9DCA85130544FDEFE07B
:10BA70007F9C8144EFD0BFD2E3D5A4FC83270B0188
:10BA800013971400BA9783D5070089C5130544FDA1
:10BA9000EFE05F9A8504F9BFEF622FCF834745003F
:10BAA000404DD5E7FD574DC0834694000947636D6F
:10BAB000D7080346B400854663E8C6088306E40059
:10BAC00063C406085C45F9562390D70097A7FF1F6B
:10BAD00083C747FC99E3A304E40097A7FF1F93875C
:10BAE000A7039C4381E78947A306F40097A7FF1F9C
:10BAF000938707519C4381E789472306F400970504
:10BB0000000093854505AA8413050401EFC0703F2A
:10BB1000FD57231AF40281471CDC014897A7FF1F39
:10BB200023A687F697A7FF1F938787F6232E040384
:10BB300004C08043EFD0FFD061463306C502814583
:10BB40002285EF608FC781473E856F604FC6FD57E6
:10BB5000E5BFEF628FC32A8403554502EF50A01C56
:10BB600009E5231E04006F608FC48357E401E5DFFD
:10BB7000930504FF17250100130545A9EFB01063D5
:10BB8000DDB7EF628FC02E89A16541119385E50372
:10BB90002A8436C432C6BE843AC2EFC07FF212474E
:10BBA0002285BA85EFE0DF8732462285B285EFE055
:10BBB0007F88A2462285B685EFE0DF87630D090006
:10BBC00091452285EFE05F811146A685EFE0207D5B
:10BBD00041016F60CFBD89452285EFE0EFFF83C74C
:10BBE00004002300F50083C71400A300F500CDB7BF
:10BBF000EF62AFB983C79500444D054793F7F70748
:10BC0000A384F5001C42411183C70700636DF7044C
:10BC10002E842A8985CC03C7D4006309F70217A7AD
:10BC2000FF1F130767EF184301CFA386F400EF80CF
:10BC3000902B83C7D40089E741657D15EF304075AF
:10BC400083D72403918B99C3EFB0B0624A85A28554
:10BC5000EFF0CFBFA167C10748003EC42302010037
:10BC600002C6EFF04FB741016F606FB4EF62EFB102
:10BC700003D745008D47AA8441112E8432892E8531
:10BC800063EDE700EFE09F85AA8523000900268584
:10BC9000EFC07FD641016F608FB1EFE03F842AC6CD
:10BCA0002285EFE0BF83B24585472A862300F9004D
:10BCB0002685EFC05FD1F9BF397106DE22DC26DAB6
:10BCC00080004ED652D456D24AD85AD05ECEAE89D3
:10BCD000B284AA8AEFD0BFAB0605130525024199AD
:10BCE0000A8A3301A140232224FC231404FCEFD050
:10BCF0001FAA83C7990006054D0593F7F70723157B
:10BD0000A4FCA384F9002685232624FCEFE00FFD84
:10BD100093170501C1876340F0025281130104FCAF
:10BD2000F2506254D2544259B259225A925A025B8A
:10BD3000F24B21618280AA8B03AB0400EFC03FCE9F
:10BD400035E983D7440001498544F11793B71700BB
:10BD5000A301F4FC834734FCA165BDC79385E504CA
:10BD6000130544FCEFC0DFD5A685130544FCEFE0C6
:10BD70002FEBDE85130544FCEFE0CFEB834734FC6B
:10BD8000114691E30946DA85130544FCEFE06FE7BD
:10BD9000814463080900416B7D1BEFD05F9F63C83E
:10BDA000A40201478146130644FCCE855685EFC0A8
:10BDB000BFF1A5B7A685130634FCEFF03FEB933433
:10BDC00015002A89860479B79385C50451BF832756
:10BDD000C90013971400BA9783D5070063866501DD
:10BDE000130544FCEFE00FE5850445BFEF626F9754
:10BDF00079711C103EC4B7070F003EC61C103EC828
:10BE000083C79500AA8A328593F7F707A384F500C4
:10BE1000AE893284EFE08FEC93170501C187635040
:10BE2000F0062A8A2285EFE06FEB2A895285032BE0
:10BE30000400EFC0DFBE39E5835744008144054468
:10BE4000F11793B71700A303F10083457100DA8758
:10BE50002287CA8652862800EFF0BFD2014781466A
:10BE60003000CE855685EFC03FE6A1679387D703A4
:10BE700048083ECC230A810026CEEFF0CF954561DD
:10BE80006F60AF91A28513067100EFF03FDEAA84C8
:10BE9000094445DD3544E30A55FB4A85EFF00FE7D9
:10BEA0000D4445D50144EFD09F8E634BA400C16B78
:10BEB0000144FD1BEFD0BF8D634EA400154471B744
:10BEC000DC4413171400BA9783D707006381270354
:10BED0000504D1BFD84493171400BA9703D70700BD
:10BEE00063197701239027012685EF80C054014410
:10BEF000A9BF0504C1B7EF62AF8783C795004111A1
:10BF00002A8A93F7F707A384F50032852E893284B5
:10BF1000EFE0CFDC93170501C187635BF004AA89CA
:10BF20002285EFE0AFDB2311A1004E85832A0400B8
:10BF3000EFC0FFAE29E18357440085440144F11767
:10BF400093B71700A300F100034811000357210025
:10BF5000D6875285CE862686CA85EFF0EFB3A167D5
:10BF6000F10748003EC42302910022C6EFF0AF86DD
:10BF700041016F602F83A28513061100EFF01FCFE0
:10BF80002A84894471D18357210011678544BA9767
:10BF9000C2071167C1831307F7EFE367F7FA97A7A3
:10BFA000FF1F9387A7CD9C4391C7854513052100AB
:10BFB000EF40300E8355210022858144EFC09F9DC4
:10BFC00041D5231005002285EF808048B5BFEF5290
:10BFD0005FF983C7950041112A8B93F7F707A38474
:10BFE000F50032852E8A3284EFE04FCF931705019A
:10BFF000C1876359F004AA8A2285EFE02FCE2A89EF
:10C000005685832B0400EFC09FA121E18357440094
:10C0100081440544F11793B71700A301F1000348C9
:10C020003100DE875A854A87D6862286D285EFF090
:10C03000AFA6A167ED0748003EC42302810026C6D3
:10C04000EFE07FF941016F505FF5A28513063100E3
:10C05000EFF0DFC1AA84094479D19167CA97C2077A
:10C060001167C1831307F7EF0544E36AF7FACA853E
:10C07000EFC05F92014445F58149EFD04FF263DB99
:10C08000A900984893971900BA9703D7070015E7B6
:10C0900023902701EFD0AFF01544E382A9F826855D
:10C0A000EF80003B97A7FF1F938747BD9C43014448
:10C0B000BDD74A85EF4040769DB785097DBFEF52D9
:10C0C0003FEB79713E847C083EC82E8AB707140086
:10C0D000A1653ECAE5057C08AA89080836C44289DC
:10C0E00032C6BA8AC6843ECCEFC09F9DCA85080876
:10C0F000EFE00FB332460808B285EFE0AFB3A246D7
:10C10000630E09029D450808EFE00FAD1D4681450D
:10C11000EF50BFEA63870A0691450808EFE0CFAB0E
:10C120001146A685EFE0A027100801478146D28579
:10C130004E85EFC07FB945616F50DFE6B6850808D0
:10C14000EFE04FAF1C400808D8439355C7018589DD
:10C1500012075183B205D98DEFE0CFAD1C4008081E
:10C1600083C58700EFE0CFAB1C40080883C5A7005C
:10C17000EFE00FAB1C40080883C59700EFE04FAA23
:10C1800051BF89450808EFE02FA583C704002300AD
:10C19000F50083C71400A300F50079B7EF525FDD07
:10C1A00083C795004111AA8993F7F707A384F50087
:10C1B0003285AE843284EFE06FB293170501C187F8
:10C1C0006357F0042A89032A0400EFC05F8519E948
:10C1D000835744000548F11793B71700A307F100F0
:10C1E000814621A81306F100A285EFF03FA81DC1EA
:10C1F0001C459DC383D6470001480347F1009307C0
:10C200008500D2884A86A6854E85EFF05FEB410116
:10C210006F505FD90948E9B71D48D9B7EF525FD5CC
:10C2200065715C083EC4B7077B013EC65C083EC82A
:10C2300083C795002A8A328593F7F707A384F50010
:10C24000AE89EFE04FA88357E100C5C389452800B8
:10C25000EFC01F8781452800EFE08F9CEFC0FF8B68
:10C2600097A7FF1F9387C7D99C4317A4FF1F0344B9
:10C270006482AA843334800099C31364240097A78E
:10C28000FF1F938767899C4399C31364440097A752
:10C29000FF1F9387A79E9C4399C31364840083D593
:10C2A000040028000149EFE0EF9883D5240028001E
:10C2B000EFE04F9883D544002800EFE0AF97EFD030
:10C2C0000FC993150501C1812800EFE0AF96A28543
:10C2D0002800EFE02F969C44636CF90001478146EB
:10C2E0003000CE855285EFC03F9E59616F509FCB85
:10C2F000DC441314490028003E94EFE06F8C834720
:10C3000044000347540089070607BA978607E36E7F
:10C31000F5FC835524002800814AEFE0AF91834566
:10C3200044002800EFE0CF8F834554002800EFE061
:10C330002F8F8347440063C9FA00814A8347540022
:10C3400063CFFA00050941BF1C4413975A00280027
:10C35000BA9783D50700850AEFE0CF8DD9BF032BAD
:10C36000C40093975A0028003E9B83552B00850AF2
:10C37000EFE04F8C83550B002800EFE0AF8B7DBFC3
:10C38000EF52BFC05C4993E717005CC9EF802033D0
:10C390006F50FFC1EF527FBF2E848145EFF08F9B1E
:10C3A00005C183570500FD172310F50009C4835705
:10C3B00025002310F400EFF0BFFC01456F503FBF94
:10C3C00031456DDC23100400D5BFEF527FBA83C71F
:10C3D000950041112A8A93F7F707A384F500328567
:10C3E0002E893284EFE08F8F93170501C187635E3A
:10C3F000F004AA89C1452285EFD0BFFA2A8B4E8569
:10C40000832A0400EFC0AFE121E5835744002311E4
:10C4100001000544F11793B71700A300F100814410
:10C420000348110003572100D6875285CE86228605
:10C43000CA85EFE07FE6A1679387170248003EC4F4
:10C440002302810026C6EFE01FB941016F509FB55E
:10C4500013061100A285EFF07F81AA8409E523115C
:10C460000100094475BF930521005A85EFF09FF242
:10C47000835721002A84CDD797A7FF1F9387078072
:10C480009C4391C7854513052100EF4080408355AB
:10C49000210026853144EFC0EFCF59D1231005008C
:10C4A0002685EF70F07A0144A5BFEF521FAE41110F
:10C4B0002E896C00AA8402C6EFF0CF8909CD0357FC
:10C4C000050005072310E500EFF09FEB81473E854F
:10C4D00041016F50DFAD3247954775DBCA85268530
:10C4E000EF20D008C147E34405FE3244854741466A
:10C4F0002310F40083570900A68513054400231177
:10C50000F400EFD0D0692285C1B7EF527FA683C770
:10C5100095004111AA8A93F7F707A384F5003285A5
:10C52000AE893284EFD09FFB93170501C187635E0C
:10C53000F0042A8AC1452285EFD0BFE6AA8452853D
:10C54000032B0400EFC0AFCD21E583574400231136
:10C5500001008544F11793B71700A300F1000144CF
:10C560000348110003572100DA875685D2862686B4
:10C57000CE85EFE07FD2A1679387070248003EC4D3
:10C580002302910022C6EFE01FA541016F509FA139
:10C59000A28513061100EFF06FED2A8409E523113F
:10C5A0000100894475BF268593052100EFF0FFEF58
:10C5B000AA845DF5835521002285EFC0AFBD4DF102
:10C5C0000149EFD0CF9D635DA9001848931719006A
:10C5D000BA9703D707001DE7035721002390E70010
:10C5E000EFD0EF9B630225039797FF1F938707699F
:10C5F0009C4389C703552100EF4000222285EF703C
:10C600003065B9BF050975BF954499BF05C193074A
:10C61000F00F630FF500C547630CF5009307F5FFB6
:10C6200005453315F5004205418182800145828030
:10C6300041657D158280B9E1EF523F9503450603C0
:10C640003284EFF0BFFC9305803EB305B502C2050E
:10C65000C18191C90357E402854763F6E7001305DA
:10C660000401EFC020168357E40241677D176385FC
:10C67000E700FD172317F4026F507F938280EF527B
:10C680005F8E004283C79500444D0349140093F721
:10C69000F707A384F5008347040022091167336973
:10C6A000F900A167B347F90041112A8BAE8A63EC08
:10C6B000E70C834724001307C00EB91793F7F70F51
:10C6C0006371F70E03473400C14763ECE70C8347FF
:10C6D00044001307E00793C707086373F70A834909
:10C6E000840083477400A209B3E9F900856763F900
:10C6F000F908034A6400834754004E85220A336ACE
:10C70000FA00EF40406245C123962403834B340076
:10C71000137AFA00239A3403238874032399440379
:10C7200093890401631A090023A6040223980402D2
:10C730004E85EFC0A00A1DA0034924004A85EFF0F2
:10C74000FFEC2397A402834744004E85A388F4029C
:10C75000E3810BFEE30F09FCEFC06005EF709079F9
:10C7600081460146D6855A85EFE09FA5A16793874C
:10C7700097033EC423020100480002C6EFE0BF85D4
:10C7800041016F509F818544A2862686D6855A85B1
:10C79000EFE01FA3A167938797033EC42302910094
:10C7A000E1BFBD44D5B79144C5B7EF526FFC01114D
:10C7B0001C08404D3EC2B7070F003EC41C083EC6D1
:10C7C0002A89AE89EFC01F9D585C1C5C634CB70A78
:10C7D0006394E50063E8A70A3385A740B3B7A700D1
:10C7E000B305B7401306803E81469D8DEFD0407B58
:10C7F00093140501C180A1659385C5034800EFC06E
:10C800002FAC81454800EFD0BFC1835504044800D8
:10C81000EFD05FC2835524044800EFD0BFC18145EB
:10C8200099C8C167FD179305F00F6386F40026854C
:10C83000EF402015AA854800EFD09FBE0355440461
:10C84000814511C9C167FD179305F00F6305F50018
:10C85000EF402013AA854800EFD09FBC83456404B5
:10C860004800EFD0FFBB834574044800EFD05FBBA6
:10C87000500001478146CE854A85EFC0EFC405616F
:10C880006F504FF2814485BFEF522FF083C7950060
:10C8900093F7F707A384F500EFF03FF16F502FF106
:10C8A000EF520FED83C795004111404D93F7F70705
:10C8B000A384F5002A8A3285B284AE89EFD01FC2E4
:10C8C0002A8B2685EFD09FC12A892685EFD0BFBF4E
:10C8D00093170B0163CA0702E177CA97C207C183A6
:10C8E000116763E3E70293070910C207C1831307C7
:10C8F000B00F637BF70093170901C187AA8A6348C9
:10C90000F000C54763FA570141016F50AFE9EFC02E
:10C910008F83E31B25FFF5B763060B02630409024F
:10C92000814463870A02B7077F002310640523113F
:10C9300024057CC05685EFF07FCD9304803EB30480
:10C94000950239A0B7077F00232004047CC08144EE
:10C9500003552404EFB0101095CCEFC0BF8326958B
:10C9600093D7F44133379500AE97BA9708DC5CDC77
:10C97000CE855285EFF07FE399E023220404A1677E
:10C980009387B70348003EC42302010002C6EFE0CC
:10C990008FE49DBF814701481CDC232E0403C9BFDF
:10C9A000EF52AFDEEFC0FFE9E1473305F5029145F5
:10C9B000EF30507FE55711C59797FF1F23AAA70CAB
:10C9C00081473E856F50AFDE85471797FF1F2303D2
:10C9D000F70C8280EF526FDB9797FF1F9387070B4F
:10C9E00080432DC083570404639EA7048357240407
:10C9F000639AB7043689B284EFC0CFF95C5C63C335
:10CA0000B7046395B7001C5C63EEA7028347640418
:10CA100063F3F400A6872303F4048347740463F3E9
:10CA20009700A687A303F4048357440441677D1746
:10CA30006385E70085072312F4043C4481C7CA8557
:10CA4000268582976F50AFD69797FF1F938707046D
:10CA50009C43014599C303C587008280EF52EFD202
:10CA60000111B70707003EC683C79500584D0AC499
:10CA700093F7F7070AC8A384F5002A89AE8401CB8F
:10CA80001C4283C707002304F700EF70D0452164E0
:10CA9000930554022800EFC0AF82EFF0FFFAAA8599
:10CAA0002800EFD0FF97300001478146A6854A85D0
:10CAB000EFC08FA113044402480822CC230A0100CE
:10CAC00002CEEFE04FD105616F506FCEEF52EFCB4A
:10CAD00001117C003ECAB70707003ECC7C003ECE69
:10CAE00083C795002E84AA8493F7F707A384F500E3
:10CAF000A165938555024808EFB09FFCEFF0DFF485
:10CB0000AA854808EFD0DF91500801478146A285E9
:10CB10002685EFC06F9B05616F506FC99797FF1F08
:10CB20009387C7F69C43094599C303C59700828044
:10CB30009797FF1F938787F59C43094599C303C5C2
:10CB4000D70082809797FF1F938747F49C43014546
:10CB500099C303C5A7008280EF528FC10111B707A7
:10CB600008003EC683C79500404D0AC493F7F707F7
:10CB70000AC8A384F5002A89AE8429C014428547D7
:10CB800003C7060063EEE706834794000946814920
:10CB9000638EC700B307F740A304E400B339F00085
:10CBA00083C716002305F400EF70F0330357240306
:10CBB000058B09C763840900EFA0B06B216493055E
:10CBC00084022800EFB0DFEFEFF05FF5AA852800C0
:10CBD000EFD01F85EFF01FF7AA852800EFD05F8404
:10CBE000014781463000A6854A85EFC0EF8D1304CA
:10CBF0007402480822CC230A010002CEEFE0AFBD48
:10CC000005616F502FBAEF524FB801117C003ECA38
:10CC1000B70708003ECC7C003ECE83C795002E842B
:10CC2000AA8493F7F707A384F500A165938585028D
:10CC30004808EFB0FFE8EFF07FEEAA854808EFD094
:10CC40002FFEEFF03FF0AA854808EFD06FFD5008A7
:10CC500001478146A2852685EFC00F8705616F5089
:10CC60000FB59797FF1F938767E29C43014599C3D0
:10CC700003C5B7008280EF524FB10111B70707001B
:10CC80003EC683C79500404D0AC493F7F7070AC80C
:10CC9000A384F5002A89AE8405C41C42054783C7D6
:10CCA0000700636AF7040347B400630BF700A305AA
:10CCB000F400EF7050238347B400A9C3EFD00FD91D
:10CCC00021649305B4002800EFB09FDFEFF07FF9F7
:10CCD000AA852800EFD0CFF4014781463000A68511
:10CCE0004A85EFB07FFE2904480822CC230A0100C0
:10CCF00002CEEFE04FAE05616F506FABEFD02FDA91
:10CD0000C1B7EF528FA801117C003ECAB7070700D8
:10CD10003ECC7C003ECE83C795002E84AA8493F738
:10CD2000F707A384F500A165AD054808EFB05FD90A
:10CD3000EFF03FF3AA854808EFD08FEE5008014787
:10CD40008146A2852685EFB03FF805616F502FA67A
:10CD50009797FF1F938787D39C43094599C303C5C2
:10CD6000C7008280EF526FA201117C00AE843ECAE0
:10CD7000A165B70707002A843ECCD1057C0048088E
:10CD80003ECEEFB0FFD3EFF0BFFCAA854808EFD04E
:10CD90002FE9500801478146A6852285EFB0DFF2D2
:10CDA00005616F50CFA0EF524F9E83C7950093F758
:10CDB000F707A384F500EFF0FFFA6F504F9FEF5293
:10CDC0002F9B83C795000329C501411193F7F707EE
:10CDD000A384F5001C4283C90700854763EC37052F
:10CDE0009797FF1F9387C7219C432E84AA8495C7DA
:10CDF000EFF01FF689476302F502630009028347DB
:10CE0000C900638C370123063901EF70D00D8357B9
:10CE10002903898B99C3EFA0D0452685A285EFF021
:10CE20007FF4A167CD0748003EC42302010002C67B
:10CE3000EFE06F9A41016F50EF969797FF1F93872E
:10CE4000E7C49C431D4599C303C5E7008280EF52A8
:10CE5000CF930111B70707003EC683C79500584D11
:10CE60000AC493F7F7070AC8A384F5002A89AE8499
:10CE700005C71C4283C7070093968701E18663C8F4
:10CE8000060485466385D7048346E7006386F6007B
:10CE90002307F700EF70300521649305E4002800B4
:10CEA000EFB01FC2EFF07FF9AA852800EFD04FD76F
:10CEB000014781463000A6854A85EFB0FFE0350482
:10CEC000480822CC230A010002CEEFE0CF90056192
:10CED0006F50EF8DEF526F8B01117C003ECAB70788
:10CEE00007003ECC7C003ECE83C795002E84AA84EA
:10CEF00093F7F707A384F500A165B9054808EFB0DB
:10CF00003FBCEFF09FF3AA854808EFD06FD15008DF
:10CF100001478146A2852685EFB01FDB05616F5072
:10CF20000F89EF52EF84AA8401441799FF1F130958
:10CF300029B6E149EFC0FF906344A400014519A858
:10CF400033053403832709003E95835725006395F5
:10CF5000970011056F500F850504E9BF032E85006A
:10CF600063040E101793FF1F130343D10323030021
:10CF7000631503002943639A060E03234E016315CC
:10CF800003001D436393070EEF42BFFDC689428A2B
:10CF90003E89BA8AB684328BAE8B2A84A1E90355C6
:10CFA0004E0009E501431A856F403FFFA167A98F35
:10CFB000116763F7E700EFF0DFF68145EFF08FBD13
:10CFC0000844B70700E05841F98F18455CC1B7071E
:10CFD000001FF98F1CC55C4981C76105EFB01000C7
:10CFE000E38209FC2285EF70606E6DBF3285EFA091
:10CFF000E0620D434DD91C44116703D54700A1677A
:10D00000A98F63F7E700EFF0DFF18145EFF08FB80C
:10D010000323840093164B01D1828347B300035648
:10D0200063008588FD8BA305F300FD777D8E558E0B
:10D03000FD76FD16B204F18E83274301C58E2312BF
:10D0400073012313D3002304530123052301A304F5
:10D050004301D9D72285EFB07FBBAA850844B5DD4F
:10D060006105EFB02076ADBF1D431A858280EF4287
:10D070003FF00569AA84AE89328A0144FD5A7D19C0
:10D08000EFC0EFF06345A40001456F40BFF1D84405
:10D0900093171400BA9703D70700631B3703239035
:10D0A000570163050A002685EF70E0389C448DC364
:10D0B00083D76700B3F72701639C3701D288014803
:10D0C000814701478146014681452685EFF01FE9EA
:10D0D00005047DB7EF42DFE979711C103EC4B70744
:10D0E0000F003EC61C103EC883C79500AA8A328531
:10D0F00093F7F707A384F5002E893284EFD00FBE93
:10D1000093170501C1876350F006AA892285EFD0E5
:10D11000EFBC2A8A4E85032B0400EFB05F9039E5FF
:10D120008357440081440544F11793B71700A303C4
:10D13000F10083457100DA872287D2864E86280067
:10D14000EFE03FA4014781463000CA855685EFB025
:10D15000BFB7A1679387F70348083ECC230A810035
:10D1600026CEEFD05FE745616F40DFE3A28513066F
:10D170007100EFE0BFAFAA84094445DD5285EFE0BE
:10D18000EFB80D445DD50546D2852685EFF03FEE1C
:10D190002A8445B7EF427FDF835507000346270007
:10D1A00041112A842E8532C62EC4EFE02FB611C558
:10D1B0003246A2452285EFF09FEB41016F403FDFF1
:10D1C000EF423FDA83C795004111AA8A93F7F70728
:10D1D000A384F5003285AE893284EFD02FB0931747
:10D1E0000501C1876357F008C1452A8A2285EFD01F
:10D1F0004F9B2A8D2285EFD06FAE2A892285EFD0F2
:10D200008FAC930705F893F7F70F1307E007AA8B86
:10D210006371F7062285EFD00FAB2A8C2285EFD001
:10D220008FAAAA8C5285032B0400EFB04FFF29E58B
:10D2300083574400231101008144F11793B717006D
:10D24000A300F10005440347110083562100938792
:10D2500084005685DA8822885286CE85EFE03FE644
:10D26000A167E90748003EC42302810026C6EFD02B
:10D270009FD641016F407FD213061100A285EFE0D7
:10D28000FF9EAA8409E52311010009446DBF93059F
:10D2900021006A85EFF06FA12A8455F5835521009E
:10D2A0009356C9001316490185486688E2875E8750
:10D2B000858A51822685EFF07FCA2A8469B7EF42BA
:10D2C0005FCA83C7950041112A8B93F7F707A384A0
:10D2D000F5003285AE893284EFD04FA09317050157
:10D2E000C1876352F0082A8A2285EFD02F9FAA8A2D
:10D2F0002285EFD0AF9E2A892285EFD0CF9C93075D
:10D3000005F893F7F70F1307E0072A8C637DF704FE
:10D310002285EFD04F9BAA8C2285EFD0CF9A2A8D01
:10D320005285832B0400EFB08FEF29E1835744002F
:10D3300085440144F11793B71700A301F100034797
:10D340003100930784005A85DE882688D686528667
:10D35000CE85EFE0DFD68D4748003EC42302910022
:10D3600022C6EFD05FC741016F403FC3A2851306BD
:10D370003100EFE0BF8F2A84894471D19356C900F0
:10D380001316490185486A88E6876287858A518233
:10D39000D685EFF0BFBCAA845DB7EF427FBD2A8976
:10D3A00081440144617A916A179BFF1F130B0B8D17
:10D3B000EFC0EFBE63C5A40022856F40BFBE8327C8
:10D3C000090093991400CE9703D507003307450150
:10D3D000420741836362570311CD03270B0009C73E
:10D3E00085453E85EF30E04A832709000504CE9746
:10D3F0002390070085046DBFEFF0BFB283270900BB
:10D400000504CE972390070075D58145EFE09FF87E
:10D41000D5B7EF42FFB583C7950041112A8A93F72C
:10D42000F707A384F50032852E893284EFD00F8B65
:10D4300093170501C1876354F004AA89832A040065
:10D44000EFB0EFDD21E18357440085440144F1173B
:10D4500093B71700A301F10003483100D687528526
:10D460000147CE862686CA85EFD01FE3A167F50760
:10D4700048003EC42302910022C6EFD0DFB541012F
:10D480006F405FB2A28513063100EFE02FFE2A84C1
:10D49000894479D19787FF1F9387477E9C4381CB2F
:10D4A0000449EFC0CFAFAA852685EF30803E130533
:10D4B0000401EFF09FEE2285EF609079814469BF0F
:10D4C000EF423FAA83C795004111AA8A93F7F70755
:10D4D000A384F5003285AE89328423110100EFC0A8
:10D4E000FFFF93170501C187635CF0042A8AC145D9
:10D4F0002285EFC01FEBAA8B5285032B0400EFB0EF
:10D500000FD231E18357440085440144F11793B7AA
:10D510001700A300F1000348110003572100DA8728
:10D520005685D2862686CE85EFD01FD7A1679387F2
:10D53000270248003EC42302910022C6EFD0BFA9B3
:10D5400041016F409FA5A28513061100EFE00FF285
:10D550002A84894469D19787FF1F9387277298434C
:10D560003E8901CB0449EFC08FA3AA852685EF3001
:10D57000403213050401EFF05FE2EFC04FA2954483
:10D5800059D9930521005E85EFE03FF2AA8441F569
:10D590001C480357210022852390E700EF60506B61
:10D5A00083270900ADDB03552100EF30E026A5B746
:10D5B000EF423F9B83C795004111AA8A93F7F70773
:10D5C000A384F5003285AE893284EFC03FF1931712
:10D5D0000501C1876359F0042A8A2285EFC01FF034
:10D5E0002A895285032B0400EFB06FC321E18357D2
:10D5F000440085440144F11793B71700A301F100DB
:10D6000003483100DA8756854A87D2862686CE853A
:10D61000EFD09FC8A167F90748003EC423029100DC
:10D6200022C6EFD05F9B41016F403F97A285130652
:10D630003100EFE0AFE32A84894479D19167CA973A
:10D64000C2071167C1831307F7EF8544E36AF7FA4E
:10D650009787FF1F938787629843BE8B01CB04494E
:10D66000EFC0EF93AA852685EF30A02213050401B1
:10D67000EFF0BFD2EFC0AF92954459D11C4822853C
:10D68000814423902701EF60B05C83A70B00ADDBE2
:10D690004A85EF306018ADB7EF423F8F2A844105CD
:10D6A000B284EFF09FCF01C52285EF60705A8146AA
:10D6B0000146A6852285EF70C00B1C4C89C7DC474C
:10D6C00099C3228582976F409F8E9787FF1F93870C
:10D6D000E73B9C43014599C31385070182809787E7
:10D6E000FF1F9387A73A88438280EF421F8A9317D0
:10D6F000C600DD8DC2054111C1812A8432C6EFC04A
:10D700007FD33246228511829375F60FEFC05FD129
:10D7100041016F40DF89EF42BF8579713C083ED2FD
:10D72000B7070C003ED43C083ED683C79500AE84B4
:10D730002A8993F7F707A384F500A165938535043B
:10D740004810EFB0EFB7C165FD150144178AFF1F00
:10D75000130A4A54930A400EAE892E8B2EC6EFC090
:10D760000F874205931704014181C183B24563E3EA
:10D77000A702C167FD176385F5004810EFC09FCB76
:10D78000501001478146A6854A85EFB0EFD3456129
:10D790006F405F813307540383270A0BBA9703D680
:10D7A000C70163083601638835014810EFF0FFF3C5
:10D7B000DA85050465B7B285EDBFEF428FFA79715E
:10D7C0007C083EC8B70711003ECA7C083ECC83C720
:10D7D0009500AA89328593F7F707A384F5002E896F
:10D7E000EFC0DFCF8567637EF502A165AA84890556
:10D7F0000808EFB0EFAC2685EF30E0521334150087
:10D800000A04A2850808EFC0BFC1A6850808EFC0BA
:10D810007FC235C0014781461008CA854E85EFB0EA
:10D82000AFCA45616F406FF7B30754030327CA0AB5
:10D83000BA9703D70700631A970003D62700638AB5
:10D8400065030808EFF07FEADE8505042EC6EFB019
:10D850001FF94205931704014181C183B245E3E5F5
:10D86000A7FCC167FD17E387F5FA0808EFC09FBC66
:10D8700055B7B285D9BFC165FD150144178AFF1F91
:10D88000130A4A41930A80022E8BAE8BC1B7EF4236
:10D89000CFEF18418347170083460700A207D58FB3
:10D8A000D207D1832390F500834727000347170051
:10D8B0008D45A207D98F91832310F600EFC03FADAD
:10D8C0006F40EFEEEF42CFEAC16401441789FF1FBA
:10D8D0001309493C93098002FD14EFB05FF06345E2
:10D8E000A40001456F400FEC330534038327C90AB8
:10D8F0003E9583570500E38797FE0504F9BFEF4285
:10D900002FE72A8AAE89B284B68AEF30C04109E592
:10D9100091473E856F400FE92A894E85EF90105060
:10D920002A84638A0A048D476DD503570500C547CD
:10D93000E31147FF0347F9018546AD47E31BD7FCD9
:10D940008347450091CB4146A6855D05EFC0D022B7
:10D95000814761D1AD4775BF130965012302E50019
:10D96000CA852685EF10202D15CDA547E3830AFA39
:10D970002302040079BF11CD83570500E39A47F9CC
:10D980004146A6851905EFC0301F814759D19947F7
:10D9900049B74E85EFF01FF32A8495473DD9130907
:10D9A00055007DBF4146A685231044012311340153
:10D9B00013051900EFC0B01E2285EF60B03C81470F
:10D9C00089BFEF428FDC79717C003ECCB7070A003B
:10D9D0003ECE7C003ED083C79500B2842E8493F760
:10D9E000F707A384F5001306A1002A892C002685D9
:10D9F000EFF0FFE9A16528088D05EFB06F8C90402E
:10DA00008355A100035581008546EFF05FEFAA849E
:10DA1000AA852808EFC0DFA00356A1008355810026
:10DA20002808EFF09FCC300801478146A2854A853F
:10DA3000EFB08FA9854748103ED42302910202D649
:10DA4000EFD06FD945616F408FD6EF420FD4797117
:10DA50007C003ECCB7070A003ECE7C003ED083C798
:10DA60009500B2842E8493F7F707A384F50013067C
:10DA7000A1002A892C002685EFF07FE1A165280806
:10DA80008D05EFB0EF8390408355A10003558100D1
:10DA90008146EFF0DFE6AA84AA852808EFC05F98E8
:10DAA0000356A100835581002808EFF01FC43008F9
:10DAB00001478146A2854A85EFB00FA14810230295
:10DAC000910202D402D6EFD00FD145616F402FCE24
:10DAD000EF42AFCBEFF0BFE26F406FCD9787FF1FF4
:10DAE000938707FB88438280EF422FCA8357250024
:10DAF0004111AE842A842307B10017F5FFFF1305F7
:10DB0000A5696C002316F100EFB0CFD581C4228542
:10DB1000EF60B02DFD572310F4001306200281455D
:10DB200013055400EF406FC941016F404FC8EF42E9
:10DB30002FC479717C003ECCB7070A003ECE7C0032
:10DB40003ED083C79500AA89AE8493F7F707328544
:10DB5000A384F5001306A1002C00EFF05FD303555A
:10DB600081001144EF30201C15C10355A100014470
:10DB7000EF90D02A01CD035705008357810045441B
:10DB80006316F7008545EFF03FF6014421699305E0
:10DB900039002808EFA0DFF2A2852808EFC05F88CF
:10DBA0000356A100835581002808EFF01FB4300808
:10DBB00001478146A6854E85EFB00F9148104AD4A3
:10DBC0002302810202D6EFD00FC145616F408FBDA5
:10DBD000EF420FBA9787FF1F938747EB2A8488434A
:10DBE0002E8915C1035745038357C401631DF700F0
:10DBF00023260502231805024105EFA0303E6304E9
:10DC00000900EF60302F81449789FF1F93898908AD
:10DC1000130A8002EFB0BFBC63CCA4029787FF1F3A
:10DC2000938787EF9C4389C70355C401EF10407663
:10DC3000630509002285EF6050031306400E8145FD
:10DC40002285EF408FB7FD57231EF4006F408FB53C
:10DC50003385440383A7C90A3E95035705008357BC
:10DC6000C4016315F700CA85EFF01FE885045DB7AE
:10DC7000EF420FB083C795004111AA8993F7F707C8
:10DC8000A384F5003285AE84EFC05F85856763703D
:10DC9000F5042A89EF302009014411C983D7040013
:10DCA0003144638627018545EFF09FF201444E859C
:10DCB000A2864A86A685EFD02FBFA1679387170457
:10DCC00048003EC42302810002C6EFD0CFB041011C
:10DCD0006F404FADEF42CFA99787FF1F938707DBB8
:10DCE00080431DCC0145EFA0E05681470148C16447
:10DCF0001CDC232E0403232004041789FF1F1309AF
:10DD000069F901449309400EFD14EFB05FAC634B19
:10DD1000A40081451705000013054598EFB08FB4A6
:10DD20006F404FA8330534038327090B3E95835773
:10DD3000C501638597008545EFF09FE90504F1B7BC
:10DD40009357050113D78700A380F50093170501AA
:10DD5000C183A1832380E5002381F500A381A50071
:10DD60008280EF428FA22300050083C71500A30025
:10DD7000F50083C725002301F50083C73500A30103
:10DD8000F50083C745002302F50083C75500A302B1
:10DD9000F50083C7650093059500A30305002303E1
:10DDA000F500230405003285EFF09FF96F402FA0A6
:10DDB000EF420F9C4111E9541DC995C993F9C5FF64
:10DDC0002E842A89AA84338AA900B7EA040063143E
:10DDD0009A020D88854401CCB7E704009C5F8297C6
:10DDE0002AC622866C0033053901EFC0405B2685C8
:10DDF00041016F402F9B83A78A0391048297931759
:10DE00000501C183A183A38EF4FE93570501238FDF
:10DE1000F4FEA183238EA4FEA38FF4FE4DBF63E026
:10DE2000D502EF428F96B28741113686BE8536C63F
:10DE3000EFC0E056B246410136856F404F978146AC
:10DE400036858280838705001387F5003D05FD87B1
:10DE500093F77708834607007D158606B58FA300E4
:10DE6000F5006307B7007D17834717009D83DDB773
:10DE70008280EF428F91B7E7040083A707093287BA
:10DE80002A863A858297133515006F404F9201CD4F
:10DE9000814799C9EF426F8F4146EFC04050854797
:10DEA0003E856F40CF9081473E8582801DC5EF4201
:10DEB000CF8D414681452A84EF402F9041468145D0
:10DEC00013050403EF406F8F0147C1672322040449
:10DED00038C87CC805456F408F8D014582808147D9
:10DEE00029CDA1CDEF426F8AB2842E891306800519
:10DEF00081452A84EF406F8CCA8524C42685EFF0C3
:10DF00001FF9414681452285EF402F8B3044A28581
:10DF10002285EFF01FF693040401A2852685EFF019
:10DF20007FF2A68513050402EFF0DFF12285EFF002
:10DF3000FFF785473E856F408F873E858280EF42A1
:10DF40002F834111E9541DC995C993F9C5FF2E844A
:10DF50002A89AA84338AA900B7EA04006394440397
:10DF60000D88814401CCB7E704009C5F82972AC6E4
:10DF700022866C0033053901EFC0604226854101DD
:10DF80006F404F8283A78A039104829793170501FC
:10DF9000C183A183A38EF4FE93570501238FF4FE62
:10DFA000A183238EA4FEA38FF4FE4DBF71CDEF326B
:10DFB0003FFCB28401E605456F30DFFE2A842E89DE
:10DFC0000145FDD93C487848B3E6E700F5D693868D
:10DFD000F7FFB3B7F6007D17032A4404BA9734C895
:10DFE0007CC8630F0A04C14913050A03B389494178
:10DFF0002295637B3601B2862E86A685EFF03FE23E
:10E000007C40BE9464C045BFCE862E86CE85EFF0A0
:10E010001FE1C114D2944E9923220404A2879306CF
:10E02000040103C7070003C607038507318FA38FC9
:10E03000E7FEE398F6FE3044A2852285EFF07FE309
:10E040002699C1493306994063EA9900ADD4A68662
:10E05000A68513050403EFF09FDC6DB78147B30677
:10E06000F4003307F6000347070083C50600850761
:10E070002D8F2380E600E39437FF3044A28522856C
:10E08000EFF03FDFC1147DBF0145828019C9EF3237
:10E09000DFEF130680058145EF303FF205456F3015
:10E0A0001FF10145828081473DC9B5C9EF32FFEDBF
:10E0B000FC4141462E84AA846393C704138605015C
:10E0C000A2878146C14503C7070003C5070385072B
:10E0D000298F3305D600034505008506298FA38FB8
:10E0E000E7FEE392B6FE3044A2852685EFF07FD8A6
:10E0F0002285EFF0BFF985473E856F305FEB1385D2
:10E1000007031D8E81452295EF303FEB7C401307BE
:10E1100000F813060402A2972388E70255B73E854C
:10E120008280EF329FE66D712E84B284AA859010B2
:10E1300028003689EFF0BFDA19E9D55705A050401D
:10E140000C402800EFF09FE66DD9FD142104E5F89E
:10E150002C004A85EFF03FF5814765D13E8551613E
:10E160006F30FFE4EF327FE241112EC432C62C0043
:10E170000546EFF01FFB41016F307FE3EF32FFE018
:10E1800001112A842EC602C802CA02CC02CEEFC0F8
:10E190006049B2462A86A2850808EFF0BFFC1375D5
:10E1A000F50F05616F30BFE0EF323FDE7971B28766
:10E1B0002A8421462308B10013051101BE853AC403
:10E1C00036C6EFC0C01DB246930591013685EFF00B
:10E1D0003FB72285141035460C08EFF0BFF82A84AB
:10E1E000224711E521460C103A85EFC0401B2285DD
:10E1F00045616F30DFDBEF325FD97171AE84AA8584
:10E200000A853284EFF0BFC801C90A86A685228537
:10E21000EFF03FC6814711E1C5473E854D616F3044
:10E220001FD9EF329FD31D712A8AB289BE84354629
:10E230008547130511012E8CB68A3A8BC28C468D08
:10E240002308F100EFC0A01510100C085285231F01
:10E250000100EFF05FFA2A842DE9A147631BFD0658
:10E260009307900591E0E5473546E28513051101D6
:10E2700013990A012308F10013590901EFC0201274
:10E280001357890093978A00D98F90080C085285FC
:10E29000231FF100EFF03FF62A8405E9A1E0938700
:10E2A000FA0091831379F9003EC6631309004149CE
:10E2B000668B8144C14B854DB2476397970C6A8644
:10E2C0008C0033855C01EFC0800D228525616F30A5
:10E2D0009FCC93079004C9F8A54779B783470105F8
:10E2E0000947C14B2308F10083471105A58FA308F7
:10E2F000F10093872400814463EFFB020147140877
:10E300003386E6008C08B386E400BA95DA9683C6B5
:10E31000060083C505000507AD8E2300D600E390F7
:10E32000E7FE41476398E70490080C085285EFF038
:10E330009FEC35D535A8B3069B00BA871008B30506
:10E34000F60090083E9603C50600034606008507C2
:10E350008506298E2380C500E39277FF998F900868
:10E360000C085285BE94EFF01FE98947014749D553
:10E370002A84A1BF90083E96034606001408BE9664
:10E380002380C600850779BFB2478504638B971247
:10E3900081471808B306F70098083E973386F900BE
:10E3A00003470700034606008507318F2380E600F8
:10E3B000E39177FF90080C085285EFF0DFE34DF909
:10E3C0003546E285130511012308B101EFB0307D18
:10E3D000139704014183939784002183D98F1018E8
:10E3E0000C085285231FF100EFF0FFE051F1814747
:10E3F00010183387F9003E960347070003460600CE
:10E40000B306FB008507318F2380E600E39277FF98
:10E4100075A01808B306F70098083E973386F900F0
:10E4200003470700034606008507318F2380E60077
:10E43000E3E127FFCA876398770990080C085285A3
:10E44000EFF07FDB15F581479800B306F7009008E1
:10E4500018103E973E9603470700034606008507BF
:10E46000318F2380E600E39177FF3546E28513057F
:10E4700011012308B101EFB0907213970401418399
:10E48000939784002183D98F10180C085285231F7D
:10E49000F100EFF05FD6E31D05EC814710183387DC
:10E4A000F9003E960347070003460600B306FB004B
:10E4B0008507318F2380E600E3E227FFC109410B86
:10E4C000E5BB8147B5B79408BE9683C60600180819
:10E4D0003E972300D7008507B9BF638E062CEF3225
:10E4E000DFA759712A84BE89B28B8547354613054B
:10E4F00011022E8B468C4289BA8A368A2300F10299
:10E50000EFB0F06910180C10228523170102EFF00C
:10E510009FCE631E0510A1476319FC069307900563
:10E5200063930900E5473546DA8513051102931414
:10E530000A012300F102C180EFB0706693178A00D0
:10E5400013D78400D98F90080C1022852317F1026D
:10E55000EFF07FCA69ED639009049307FA00BD8864
:10E56000918391E0C144C207C183DE8C814A3EC6DB
:10E57000414DB24763EAFA0C6286B3854B018810BD
:10E58000EFB0905F4DC53D555DA093079004E39CAF
:10E5900009F8A54749BF834701050947C14C230036
:10E5A000F10283471105B3C7F900A300F102938775
:10E5B0002900814963EFFC02814618103306D70019
:10E5C0008C083387D900B69556970347070083C553
:10E5D000050085062D8F2300E600E390D7FE414716
:10E5E000639AE70490080C102285EFF0DFC035D560
:10E5F0003DA8B3863A01BA871010B305F60090081B
:10E600003E9603C506000346060085078506298E4B
:10E610002380C500E39297FF3387EC4090080C10ED
:10E620002285BA99EFF03FBD8947014741D5656121
:10E630006F307F9690083E96034606001410BE96F3
:10E640002380C600850769BFB247850A93990A01EE
:10E65000939D8A0093D909016399570D85473546E3
:10E66000DA85130511022300F10293D98900EFB076
:10E670001053B3ED3D0190000C1022852317B10318
:10E68000EFF07FB74DF58147A68963E697062686AA
:10E690000C084A85EFB0B05081471810B306F70058
:10E6A000100898083E973E96034707000346060069
:10E6B0008507318F2380E600E3E197FE639DA9057E
:10E6C00090080C102285EFF01FB335F181479810A8
:10E6D000B306F700900818183E973E9603470700C8
:10E6E000034606008507318F2380E600E391A7FFEC
:10E6F0004109C10CBDBD18089000B306F7003E9655
:10E700003387FC0003470700034606008507318F67
:10E710002380E60095BF98084E97034707001C101A
:10E72000CE972380E700850951BF85473546DA85B6
:10E73000130511022300F10293D98900EFB030468E
:10E74000B3ED3D0190000C1022852317B103EFF0CB
:10E750009FAAE31E05EC814718089000B306F70056
:10E760003E963387FC0003470700034606008507F3
:10E77000318F2380E600E391A7FF41460C084A85CC
:10E78000EFB0F04181471810B306F7001008980861
:10E790003E973E9603470700034606008507318FE4
:10E7A0002380E600E391A7FF90080C102285EFF08C
:10E7B0009FA41DDDADBD7D558280EF320FFD01119F
:10E7C0002A842E8593055100328902C002C202C4F8
:10E7D00002C693047400EFF0AFD61D46A68513055C
:10E7E0009100EFB0D03B10088A854A85EFF0BFA0BA
:10E7F00019ED93071400180883C6070003460700A5
:10E8000085070507B18EA38FD7FEE397F4FE056158
:10E810006F30EFF9EF32CFF52E848C414111AA8988
:10E82000838715003289914463D30700A144977709
:10E83000FF1F9387E77C9C43B1C3B5CE8D47231060
:10E84000F10083C725004A852301F10083C7350005
:10E85000A301F10083C745002302F10083C75500DF
:10E86000A302F10083C7650093059100A303010093
:10E870002303F10023040100EFF08FCC0C404A8603
:10E880000A85EFF00FCE0328040083564400A688C3
:10E890001D0881470147E51642868A854E85EFF0BF
:10E8A0005F982A8909E5A6852285EFB0FFB24A85DF
:10E8B00041016F302FEF4A860A85EFF08FCA7DBF86
:10E8C000EF320FEB2E848C414111AA89838715000A
:10E8D0003289914463D30700A1449777FF1F938740
:10E8E00027729C43B1C3A5CE8D472310F10083C787
:10E8F00025004A852301F10083C73500A301F100FB
:10E9000083C745002302F10083C75500A302F1002D
:10E9100083C7650093059100A30301002303F10061
:10E9200023040100EFF0CFC10C404A860A85EFF0C6
:10E930004FC383564400032804008A85858EC2068F
:10E940001D08C1822312D400A68881470147E5161D
:10E9500042864E85EFF07FB841016F30AFE44A86C2
:10E960000A85EFF00FC0C9B7EF322FE2B335B00020
:10E97000011185052A891315F60133651501230850
:10E98000B1009305110136843AC632C03EC442C27A
:10E99000EFF00FBBA2471248425593D68700230BD6
:10E9A000F1009305910193578800A30AD100A30BAE
:10E9B000F100230C0101EFF0AFB832470246032803
:10E9C0000400B337E000835644009207914411C21B
:10E9D000A1444A85A68842860C08EFF09F842A89C4
:10E9E00009E5A6852285EFB03F9F4A8505616F3016
:10E9F0000FDCEF32EFD701113EC68647B335B000CA
:10EA00008505AA891315F6015D8D2308B1009305CC
:10EA1000110136843A89B28442C446C2EFF04FB243
:10EA200022489248164593578800A30AF10093059F
:10EA3000910193D78800230B0101A30BF100230C54
:10EA40001101EFF0EFAF3247104083564400B33767
:10EA5000E000920703280900914891C0A1480C08E2
:10EA60004E85EFF09FA7AA8411E5835544004A859F
:10EA7000EFB09F96268505616F30CFD2AA95930798
:10EA8000F00F17F700001307E7BB6317B50013C5B6
:10EA9000F7FF1375F50F828005058346F5FFB58FE7
:10EAA000BA9783C70700D5B70357450014419307AA
:10EAB000F00F17F600001306E6B8369742074183B9
:10EAC000139506014181631BE500AD8FB29703C525
:10EAD0000700130515F3133515008280850603C55D
:10EAE000F6FFA98FB29783C70700D9BFEF32EFC9EE
:10EAF000B28736842E86BA86AA853E85BA84EFF020
:10EB00006FE6634B05002285EFB0D0312A86A686DA
:10EB1000A2852685EFF00FE56F306FC9EF324FC544
:10EB20005D712A8BAE8A17F50000130525AF2C0006
:10EB3000B284368ABA893E89EFF04FE42A8459E5D7
:10EB400034104146DA852800EFF0CFE12A843DED0C
:10EB50008547A303F100A6C2930771002408BEC431
:10EB6000A68685470D462C18281002DC02DED6C08A
:10EB7000BEC6EFF00FDB2A8431E983477102A68617
:10EB80000D4693F7F7072300FA00C1473EDE2C1825
:10EB90008947281026DCA303F100EFF08FD82A84E0
:10EBA00015E54146A6854E85EFB0607F8D47A68668
:10EBB0000D462C182810A303F100EFF08FD62A84FD
:10EBC00011E54146A6854A85EFB0607D22856161E9
:10EBD0006F304FBDEF326FBB97D700009387870B25
:10EBE000984383C7470079712A89AE8417F50000DE
:10EBF000130545A30C083AC42306F100EFF00FD823
:10EC00002A8415E514104146CA850808EFF08FD50F
:10EC10002A8411ED140815462C000810EFF08FD44B
:10EC20002A8411E521462C082685EFB040772285FD
:10EC300045616F30CFB7EF324FB597D7000093875C
:10EC400067059C477971AA842E8417F50000130587
:10EC5000E59D0C083EC6EFF06FD20DE5141041465D
:10EC6000A6850808EFF00FD011ED140811466C00CE
:10EC70000810EFF02FCF19E58347F10193F7F70361
:10EC80002300F40045616F308FB2EF320FB0368849
:10EC9000A14881470147E546EFF0AFD86F302FB16B
:10ECA000EF32AFAE3688A14881470147E546EFF025
:10ECB000DF826F30CFAFEF324FAD01112A842E8546
:10ECC0000C0832C6EFF08FCB19E9324797F60000F7
:10ECD000938646941008C1452285EFF03FE1056117
:10ECE0006F30EFACEF326FAA4111C1472EC032C472
:10ECF0008A8509463EC23EC6EFF0AFC241016F3081
:10ED00000FABEF328FA84111AE8613061009AA850A
:10ED10000A8502C002C202C402C6EFF0AFC44101BC
:10ED20006F30EFA8EF326FA6328797F60000938618
:10ED300066902E8693050002EFF05FDB6F302FA701
:10ED4000EF32AFA47971C1472ACC2ED032D42C082F
:10ED50000D4628003ECE3ED23ED602C402C602C8B0
:10ED600002CAEFF00FBC45616F306FA4EF32EFA124
:10ED70000111AA842E8417F500001305258C8A85BD
:10ED8000EFF0CFBF05E514084146A6850A85EFF0F0
:10ED90006FBD09ED8347E1010347F101A207D98F58
:10EDA000CA07C9836177D98F2310F40005616F30DA
:10EDB0000FA005C9EF326F9D9777FF1F9387C7D1CB
:10EDC00090439775FF1F938565D11775FF1F130536
:10EDD000A5CCEFB080091775FF1F1305E5CB6F3089
:10EDE0000F9D1775FF1F130525CB82809DC5EF3240
:10EDF000CF999777FF1F938727CE944301112E84D5
:10EE00000A869775FF1F938565CDEFB0800A0A8546
:10EE10000294014505616F308F997D558280EF32F4
:10EE2000CF96EFB080149777FF1F23A7A7CA17F5D7
:10EE3000FFFF130525F8EF90D0406F304F971777FD
:10EE4000FF1F1307A7CB9317150008433E95FD57E7
:10EE50002310F5008280EF324F932A84084019E195
:10EE60006F30EF941C4158401CC06313E5005CC038
:10EE70008347550023200500F99BA302F500EFB05E
:10EE8000EFF9E9BFEF32CF8E9777FF1F938707C95E
:10EE900098432A8411CB8347350093F7070289C72B
:10EEA000035505008945029713054401EF9010139F
:10EEB000835504000355E400EF20701B485809C532
:10EEC000EFB0CFF5232A040213058403EFF0BFF857
:10EED0008144B149EFA0FF9A63C5A402834734007F
:10EEE0002320040493F727FCA301F4000048EFA0BB
:10EEF0005F9A1316150081452285EF300F8C6F3015
:10EF00006F8AB38734030329040385043E994A8535
:10EF1000EFF07FF42304090075BF8347350093F7B2
:10EF2000070299E3014582808357E500E39CB7FE21
:10EF3000C167FD176316F600054582800545B9A037
:10EF4000EF32AF8493170601C187B2842A84014946
:10EF50006359F002835705008DCB01456367F600C6
:10EF6000034584003E953325A6001375F50F39A897
:10EF70001C4813171900BA9783D70700E38097FC42
:10EF80000509EFA01F91E345A9FE01456F302F82CF
:10EF9000EF221FFEAE89AA84EFA07F852A84EFD0DE
:10EFA000BFAAAA860147130684019705000093852E
:10EFB00045E91775FF1F1305A5B4EFA0AFD52A8942
:10EFC00021CD8C441304C50022859E0593F50508C8
:10EFD000EFB00FC5CC4083877400E18163D1070493
:10EFE00093E505082285EFB0AFC30D469385440035
:10EFF0002285EFB00FC183D504002285EFB0EFC5A5
:10F0000083D524002285EFB04FC503D6490083A5E0
:10F0100009002285EFB0EFBE4A856F20BFF893F557
:10F02000F507C9B7EF227FF601112A84328532C66F
:10F03000EFB06FB4EF903F91835704001777FF1F35
:10F04000130747C53246231BF100930700F8A30DB1
:10F05000F1001C471843231AA1008983858BB3074D
:10F06000F740B28548083ECE231C0100230D010065
:10F07000EFF01FF205616F209FF3EF227FEF004159
:10F08000014529CC9304C40026853289AE89EFB0AE
:10F090008FB295452A8A2685035B0401EFB02FAF16
:10F0A0002685EFB02FC68D45AA8A2685EFB02FAEF4
:10F0B0002685EFB02FC55C48420A135A0A01D29741
:10F0C0005CC423186401814763983A0146054D8169
:10F0D000330625419337160013F5F70F6F209FEC89
:10F0E000EF223FE889692A8BAE8B328AB68A814447
:10F0F0000144314CFD19EFA0CFF863C9A400EFA083
:10F100004FFB018D33B5AA006F203FE9338984039B
:10F1100083270B003E9963170A0083478900850403
:10F120003E94D1BF03560A00DE854A8533F6C900F6
:10F13000EFF0BFF47DD10545C1BFEF221FE50111FE
:10F140002A847C000355E5003ECAB70707003ECC81
:10F150007C003ECEEF10303D2A8985454808EFB04F
:10F16000EFC199454808EFB02FA7AA844A85EF1050
:10F17000B03D2380A4009777FF1F9387A7B19C43DE
:10F180004166130606F09396870113D78701558FC2
:10F1900093D68700F18E558FA207B706FF00F58F33
:10F1A000D98F11462C00138514003EC4EFB0201FE8
:10F1B0005008A382040089452285EFF0BFE609C903
:10F1C000AA8513058403EFB0EFBB3C4085073CC024
:10F1D00005616F20DFDDEF225FDBEFA08FED2A847A
:10F1E0000504EFA00FEC3305A402F1479145330568
:10F1F000F502EF10207B01E565556F205FDB977707
:10F20000FF1F23A5A790EFA0CFEA2A840504EFA053
:10F210004FE93305A40289450605EF10A07869DDA2
:10F220009777FF1F23ACA78CEFA0AFE82A840504D3
:10F23000EFA02FE73304A4029777FF1F2392878C58
:10F24000EFA02FE72A84EFA0CFE5930714003385C2
:10F25000A7029777FF1F2396A78A97E70000938757
:10F26000A7011777FF1F2321F78A014579B7EF22FE
:10F270003FD0AA842E8901449779FF1F938989A1E1
:10F28000130A8006EFA0EFE16345A40001456F205B
:10F290007FD13305440383A709024A86A6853E959C
:10F2A000EFF0BFC719E10504F1BF0545CDB7EF2267
:10F2B0005FCBAA8A2E8BB28B368C3A8A814401446A
:10F2C0008149977CFF1F938CEC9C130D8006EFA067
:10F2D0004FDD63C7A40011E085494E856F20FFCB49
:10F2E0003389A40383A70C025E86D6853E994A859E
:10F2F000EFF0BFC219CDEFA0CFDB0544636B450132
:10F30000D2866286DA8513050903EFF07FDD11C12D
:10F31000854985046DBFEF22BFC5C16441112A89AB
:10F3200001449779FF1F9389E996130A8006FD141B
:10F3300036C632C42EC2EFA0CFD692452246B24680
:10F340006346A400014541016F20DFC53305440336
:10F3500083A709023E9509C683473500C18B9DC727
:10F3600091C68347350093F707028DC36306990062
:10F370008357E500639C27010357050001CB63E732
:10F38000E50083478500BA97E3CFF5FA05044DB74A
:10F39000EF221FBEC1642A8901449779FF1F938918
:10F3A000698F130A8006FD14EFA0AFCF6344A40059
:10F3B0006F205FBF3305440383A709023E9583573F
:10F3C000E500638897006304990063942701EFF0D8
:10F3D0007FAB0504D1BFEF225FB889692A8AAE8A64
:10F3E000328BB68B8144177CFF1F130CAC8A930CB5
:10F3F0008006314DFD19EFA0CFCA63C4A4006F2071
:10F400009FB93389940383270C028355CA015A8616
:10F410003E994A85EFF07FB005CD814D05A033843C
:10F42000AD038327090303D60B00D68533F6C90045
:10F430003E942285EFF07FC419E5850DEFA06FC4DF
:10F44000E3CFADFC31A02285EFF0FFA02304040040
:10F45000850455B7EF22FFB04169AA8A014A177B9C
:10F46000FF1F130B2B837D19C14B054CEFA06FC3FE
:10F470006344AA006F207FB293098006B3073A0362
:10F4800083290B02BE9983D7E900638C270163842B
:10F490002A016398570103A4890311E44E85EFF014
:10F4A000DFC9050AE1B7835704016399770793041D
:10F4B000C4002685EFA03FF085452A8D2685835C14
:10F4C0000401EFA0DFEC2685EFA0FFFF6205618558
:10F4D000635F05028D452685EFA07FEB8945268574
:10F4E000EFA0FFEA89452685EFA07FEA85452685BE
:10F4F000EFA03FEB83470500094793F7F7076398B1
:10F50000E70099452685EFA0DFE9A3028501484879
:10F51000337D2D01231894016A9548C40040B5BF7E
:10F52000EF22BFA637E404008327041D8297976764
:10F53000FF1F83C727631745FF1F130565EAA30055
:10F54000F5008327441C82978327841C8146130679
:10F55000F00F8145014582976F207FA51767FF1F38
:10F560001307475018439765FF1F83C5A55F97672B
:10F57000FF1F9387A75D834687030346970363971F
:10F58000D5009767FF1F238FC75C828083C58701E3
:10F590000347A7036317B6009767FF1F2384E75C41
:10F5A000828003C687016317C7009767FF1F238BFD
:10F5B000D75A828083C68701130750026319D70088
:10F5C000930760021767FF1F230EF758828083C6D8
:10F5D0008701130660026315D60093077002DDB73A
:10F5E00083C7870155BF9767FF1F93872756D44B63
:10F5F00009476385E608EF225F991769FF1F130922
:10F6000029523E8483470900918B9DCFB7E40400C3
:10F6100083A7041D829783A7441C1765FF1F13054A
:10F62000A550829783A7841C81461766FF1F034657
:10F63000A65181450145829721C183470900ED9B71
:10F640001767FF1F230EF74C8347040093F7F70F4C
:10F6500085C791471767FF1F2324F750EFF05FEC32
:10F66000EFF0DFEFB7E70400BC4F41469145176567
:10F67000FF1F0345254E82976F207F938280EF22E4
:10F68000DF908D4741116304F504C5476306F50219
:10F6900085476310F5029767FF1F2387A74CB7E7DD
:10F6A0000400BC4B930500101765FF1F0345854AF6
:10F6B000829741016F20BF8F85471767FF1F230582
:10F6C000F74AB7E70400BC4B93050020F1BF9767EA
:10F6D000FF1F9387A747D44B1147638DE600B7E719
:10F6E000040083A7071D8297B7E70400BC4B93056E
:10F6F00000045DBF05491767FF1F2323274783C702
:10F70000070032C62E8493F7F70FC5D7B7E404007D
:10F7100083A7041D7D141374F40F8297E37689FC8C
:10F72000B245994703C61500E3F0C7FCFC4409063F
:10F730001765FF1F130585438297BC489305000892
:10F740001765FF1F03450541829779BFEF22FF83AD
:10F750001767FF1F1307873F4047184B1C409766EA
:10F76000FF1F23ABF63E6316E4001767FF1F232736
:10F77000F73E130584FEEF907FF3035564FFEF908F
:10F780003FC6EFA0BFE96F209F82EF221F809767DF
:10F79000FF1F9387A73BD84BDC4799C3EFF01FFBB4
:10F7A00085471767FF1F232DF73A9767FF1F93873A
:10F7B000672B9C43930500021765FF1F034585399E
:10F7C00083C787031767FF1F230EF738B7E70400C7
:10F7D000BC4B82976F20AFFD9767FF1F23AAA73608
:10F7E0008280EF22EFF837E404007C4CA1451765D6
:10F7F000FF1F0345253682977C48A1451765FF1FEB
:10F80000034545359764FF1F938444348297DC4455
:10F8100089E7EFF05FDD6F20EFF803D567FFEF902A
:10F820003FBCAA897DD5D84891476310F7027C4C2C
:10F8300091451765FF1F0345E53182977C48914547
:10F840001765FF1F03450531829703A9490103D4BA
:10F8500009018947B7E904001767FF1F2322F73022
:10F8600083A7091D21044204829783C78401174599
:10F87000FF1F1305E5B661191747FF1FA302F7B66F
:10F8800083A7491C418082979767FF1F238E072C0F
:10F8900083A7C91C814609469375F40F4A85829750
:10F8A00011E99767FF1F83C7673C89C79730FF1F20
:10F8B000E780C021B7E70400BC4F2146A14517658A
:10F8C000FF1F034525298297B9B7EF220FEC93F765
:10F8D000052001112E8481CBEFF03FEB134504206E
:10F8E00005616F20CFEC93F70510A9CB9764FF1F3C
:10F8F0009384C425DC48EFF07FC61767FF1F13070A
:10F900006716184383C78401034787036316F7000C
:10F91000DC4499C3EFF09FE385471767FF1F23215E
:10F92000F724B7E70400BC4B930500021765FF1FDF
:10F93000034545228297134504105DB793F70508E8
:10F94000ADC79767FF1F83C77722E91719469765E9
:10F95000FF1F9385C5211305D10093F4F70F176995
:10F96000FF1F0349A920EFA0902393970401C183AF
:10F970001767FF1F13070720231DF100231CF10049
:10F980009767FF1F9387871C3ACE3ACAD84323064E
:10F99000010009CBDC439315890154080D46E1852C
:10F9A000680082971345040825BF93F72500B1CF5F
:10F9B0009767FF1F93878719D84B89476306F7021C
:10F9C0009767FF1F83C7C71513F7270011EF918BA8
:10F9D00099CFB7E70400BC4F1306000A89451765A5
:10F9E000FF1F03452517829713452400D5BD976750
:10F9F000FF1F938727079C4383C787031767FF1F52
:10FA00002302F716EFF0FFDDC5B793F7050291C7A4
:10FA1000EFF03FDD13450402E1B593F7850091C790
:10FA2000EFF0BFD61345840065BD93F7150091C76D
:10FA3000EFF07FBB1345140065B593F7450091C700
:10FA4000EFF07FBA1345440061BD93F7050485C309
:10FA50009767FF1F83C7870F81CBEFF07FAC91477C
:10FA60001767FF1F232EF70E1345040495BD93F768
:10FA700005010145E38607E69767FF1F9387070D9A
:10FA8000D84B91476310F7049767FF1F9387470987
:10FA90009C4313D727008583D98F858B91E7B7E7E0
:10FAA000040083A7071D8297B7E70400FC4F914528
:10FAB0001765FF1F0345050A829785471767FF1FD4
:10FAC0002320F70A1345040121BD9767FF1F238FE9
:10FAD000A7188280EF226FCB9767FF1F23AE070620
:10FAE0009767FF1F23AC070685471764FF1F1304A2
:10FAF00064F71767FF1F2325F7061C4083C787039A
:10FB00001767FF1F2300F706EF90FFDF39C1974704
:10FB1000FF1F23ABA78C1C4017050000130525DB36
:10FB200083C787031767FF1F230EF7021747FF1FBF
:10FB3000A308F78A9767FF1FA38A0700B7E70400A7
:10FB400083A7070882979767FF1F2385A7006F2069
:10FB50000FC6B7C7898E938767ED1747FF1F232509
:10FB6000F78855BF1767FF1F034747FE795555E3D1
:10FB70009767FF1F938787FD03C7170005079766E1
:10FB8000FF1FA385E6FC03C717008D463377D70216
:10FB90009766FF1FA38CE6FA83C617001767FF1F3F
:10FBA000130747EC184393F6F60FA9EA8347870338
:10FBB0001767FF1F2308F7FA85471767FF1F2307FB
:10FBC000F7F89767FF1F9387A7F59C430145998B2B
:10FBD000A9E3EF228FBB37E404007C48C1451765D9
:10FBE000FF1F034525F782973C4885451765FF1F92
:10FBF000034545F6829701456F206FBB83C7170009
:10FC000085466395F600834797035DB78347A7034F
:10FC100045B782809767FF1F83C747F3A1CBEF22C9
:10FC2000CFB637E404009767FF1F238107F27C48B3
:10FC300085451765FF1F0345E5F182977C4C91458B
:10FC40001765FF1F034505F182977C4891451765AD
:10FC5000FF1F034525F082973C48C1451765FF1FEC
:10FC6000034545EF829701456F206FB47955828037
:10FC7000EF22AFB12A84035565FFEF906FF69767C7
:10FC8000FF1F9387A7ECD847BE841DEBEFA05F98BA
:10FC90009C48232004008DEB9767FF1F23A087EC6F
:10FCA0009767FF1F23AA87EAB7E70400BC4B894583
:10FCB0001765FF1F034505EA829701456F202FAFA7
:10FCC000630A87001843D1B780C39767FF1F23A734
:10FCD00087E8D9BF7955DDB7EF222FAB9767FF1FB4
:10FCE000938707F98843232605002324050051053F
:10FCF000EF80D02E6F20AFABEF222FA91764FF1F2C
:10FD0000130404F71C40411189CF9C472302B5001E
:10FD10002AC61CC1EFF05FFC1C409C4B99C33245C6
:10FD2000829741016F20AFA8EF222FA64111444DC9
:10FD3000328532842EC6EFA00FF92AC42285EFA0A7
:10FD4000EFF903A84400630C0800B2458357440050
:10FD50001840224683D54500AA862685029841018F
:10FD60006F20EFA4EF226FA2404D1DC408C097057D
:10FD700000009385E50213054401EF809018976712
:10FD8000FF1F9387E7EE9C43014589E79767FF1FB5
:10FD900023A087EE6F20AFA17D55EDBFEF22EF9E30
:10FDA000011168009305F00F02C602C802CA02CC16
:10FDB00002CEEFF07FF405616F206F9F9767FF1F02
:10FDC000938707EB9C43D847A1679D076311F70210
:10FDD000EF22AF9B01113285EFA0EFEE230AA100C5
:10FDE00081456800EFF05FF105616F204F9C8280D4
:10FDF0009767FF1F9387C7E79C43D847A1679387FF
:10FE000077036311F702EF224F9801113285EFA0BB
:10FE10008FEB230AA10081456800EFF0FFED05613B
:10FE20006F20EF9882809767FF1F938767E49C435A
:10FE3000D8479547631CF702EF222F9501113285B1
:10FE40003284EFA04FE8230AA1002285EFA00FE93A
:10FE500083574400231BA10081453ECC1C40680011
:10FE60003ECEEFF07FE905616F206F9482809307AB
:10FE700085FF89CF8327C5FF91CBDC4B81CBEF2258
:10FE8000CF90032585FF82976F206F928280EF22AB
:10FE9000CF8F2A843285EFA00FE3BD4763EBA70025
:10FEA00018449377F5000345B70041995D8DA3058C
:10FEB000A7006F20CF8FEF224F8D01117C003ECA2B
:10FEC000B70707003ECC7C003ECE5C4D8DCF2A8428
:10FED00013858700AE84EF807004A1652A899D0593
:10FEE0004808EF80FFBD9305803EB345B90248083E
:10FEF00093F5F50FEFA0CFD2014781465008A685B4
:10FF00002285EF807FDC05616F206F8AEF22EF870B
:10FF1000EFF07FFA6F20AF89EF222F8701117C006D
:10FF2000AE843ECAA165B70707002A843ECC4808C4
:10FF30007C00938575033ECEEF809FB81C44480833
:10FF400083C5B700BD89EFA0AFCD500801478146FA
:10FF5000A6852285EF805FD705616F204F85EF2250
:10FF6000CF822A84AE84EFF09FF2A6852285EFF03F
:10FF7000BFFA6F20CF83EF224F81EFF0FFF96F20A0
:10FF80000F83EF228F800329C50141116304090209
:10FF90002A843285B284EFA00FD32AC62685EFA02B
:10FFA000EFD3832749002A8691C7DC4781C7B24532
:10FFB0002285829741016F109FFFEF121FFD444D74
:10FFC00081CC2A843285EFA06FD1DC40AA8589C715
:10FFD0009C4799C3228582976F107FFDEF125FF9CE
:10FFE000032AC501411163030A062E89AA84954597
:10FFF00032853284EF80DFAC85452285EFA0CFBD0E
:020000040001F9
:10000000AA89CA852285EFA0EFC283274A009DC72F
:10001000DC438DC72285EFA0AFBA83274A0010408A
:1000200083564400DC437115A307A100B296130761
:10003000F1004E86CA852685829701C52380090076
:1000400031A08345F1002285EFA00FB941016F1067
:100050007FF5EF129FF365711C083EC2B707800160
:100060003EC41C0832893EC62A84AE84EFF07FF17C
:100070004A85EFA0AFC68357A10089CFAA8550005B
:100080002285EFF0BFF5014781465000A685228505
:10009000EF809FC359616F109FF1EF127FED657183
:1000A0001C088329C5013EC2B70780013EC41C0855
:1000B0002A84AE8432893EC6EFF03FF063840902A1
:1000C0004A85EFA0AFC18357A100AA8581CF500018
:1000D0002285EFF0BFF0014781465000A6852285BA
:1000E000EF809FBE59616F10FFEBEF121FEA657141
:1000F0001C083EC2B70780013EC42A841C08328512
:100100003EC6AE84EFA08FBD8357A10089CFAA85DC
:1001100050002285EFF09FEC014781465000A685F4
:100120002285EF807FBA59616F107FE8EF12FFE5FB
:10013000444D91E88347450093B71700B307F0405B
:100140003E856F10DFE61845FD577DDB9707000001
:10015000938707032A845CCB97050000938565D1BC
:1001600013858400EF80E05980C003474400814735
:1001700061FB1767FF1F232F97AED9B7EF125FDF21
:100180008329C5014111032985008147638B090833
:100190000324090191452A8A2285EF807F928545B3
:1001A0002285EFA06FA38945AA8A2285EFA0CFA25E
:1001B000AA84EF809F9683A749002A8B9DC79C4302
:1001C0008DC72285EFA0CF9F83A74900A306A1007A
:1001D0001040835644009C431307D100B296D68545
:1001E0001306E1005285829709CD83570B002380C7
:1001F000F400A183A380F40023800A00A306010079
:1002000029A88357E10022852380F4008345D1008B
:10021000A183A380F400EFA02F9C8347D100B337C4
:10022000F0000347B900920701453D9BD98FA30514
:10023000F90041016F101FD7EF123FD541111DE9A1
:100240009767FF1F938707A3804305C804401309DE
:1002500084009DC55C4099C79C4B89C726852EC6E6
:100260008297B2459307803EB385F5024A85EF80B9
:10027000605521A0404DAA8479F841016F103FD309
:100280004A85EF80A0555C40EDDBDC4BFDD7268531
:100290008297E5B7EF127FCF2A843285EFA0AFA215
:1002A000AA852285EFF05FF96F107FD0EF12FFCDA6
:1002B0002A84AE84EFF01FFEA6852285EFF0BFBF33
:1002C0006F10FFCE08413355B50005898280EF12CB
:1002D000DFCB1764FF1F1304E49B1C5C0111231781
:1002E00001008D83858BA303F1008327040B231862
:1002F00001002319010003D7C7013ECA3C002314A3
:10030000E1007D572315E1000357C4023ECC02CE25
:100310002316E100EF802FE38357E101231EA100A4
:1003200093F707E093E71710231FF1009767FF1F6C
:1003300083C7E79885C305470145638AE70083477C
:10034000840393E727001767FF1F2301F7980561D0
:100350006F10FFC5814717D700001307E74D85468B
:100360001306710085454808EF70E04B6DF1834737
:100370008403F59B1767FF1F230AF79485471767C8
:10038000FF1F230EF792E1B7EF123FBD976DFF1FDE
:10039000938D4D9003A6CD0639712A8981478144FA
:1003A000930600023357F600058B01C7850493F4CA
:1003B000F40F8507E398D7FE83A70D0B23170102DF
:1003C0002318010203D7C7013EDA3C102314E102CF
:1003D0007D572315E10203D7CD023EDC231901022C
:1003E0002316E10202DEEF800FD68357E103231EBE
:1003F000A102014593F707E093E71710231FF102CD
:100400009767FF1F83C7A78BA9EF9767FF1F83C756
:10041000F78B3EC69769FF1F9389C9870144014D39
:100420009D4A054B954B176CFF1F130CEC8D976C79
:10043000FF1F938CEC8C03DAC90563090A00EA8577
:10044000631459036685EFF0FFE71DC1050DA14751
:100450008909E312FDFE2DE09767FF1F23A4078A99
:10046000014521616F103FB36285EFF0BFE579DD93
:100470003247B3878400E3F0E7FE9C0013061400C4
:1004800006043E9413178A0093578A00D98FC20737
:10049000C183A30EF4FCA183230FF4FC03A70D0773
:1004A000B317AB01D98F1767FF1F232DF7846304A0
:1004B0007601328461BF15449767FF1F83C70780A9
:1004C000138717009756FF1F238AE67E93161400A2
:1004D000230EF10017D70000130707368147850662
:1004E0007008CA854818EF700034E34705F6834763
:1004F000C10105451757FF1FA302F77C9757FF1F40
:10050000238F277BB9BFEF12BFA60111AA892E84C2
:10051000EFD0EF9C2A899754FF1F9384A4776399A7
:10052000090A9C5C414793F707036393E70A17574F
:10053000FF1F03471779894763ECE70883A7040B7C
:10054000231701002318010003D7C7013ECA3C004E
:100550002314E1007D572315E10003D7C4023ECCEC
:10056000231901002316E10002CEEF80CFBD231E28
:10057000A100EFC06FCD8357C101230FA1009146A9
:1005800013D78700A207D98F2312F1009757FF1FB7
:1005900083D7E77313D78700A207D98F2313F100FE
:1005A00017D700001307C728814750009545480812
:1005B000EF70602705889317240003C484036D98A7
:1005C0005D8C9757FF1F2383877005616F109F9D78
:1005D000EF70B0781755FF1F1305C56FEF8000202F
:1005E00083A7040B9755FF1F83D5856D03D5C701DE
:1005F000EF10E0279757FF1F83C7476D93F6070259
:10060000014789E61757FF1F0357876B9756FF1F50
:100610002390E66C1757FF1F13078766184309CB13
:10062000C18B99C789451755FF1F03556569029707
:100630009757FF1F23A607689757FF1F2381076857
:100640009757FF1F23AE076A9757FF1F23AC076A10
:100650009757FF1F23AA076A83D7840393F7270CB2
:1006600093E717001757FF1F2312F76683572903D5
:10067000A18B99C3EF70E03F11C49757FF1F23ADC3
:100680000762A1B78D471757FF1F2327F762EF9027
:100690002FA59305803EB305B5021755FF1F13051F
:1006A0006563EF80201215B79757FF1F9387875E0A
:1006B000D85325C791C99757FF1F238207609757C3
:1006C000FF1F23A107648280EF123F8C83C7F702CC
:1006D00041112EC685071757FF1FA304F75E9757D2
:1006E000FF1F2398A75E9D471757FF1F2326F75C20
:1006F000EF900F9E2A84EF90AF9DB24501E5EF90F9
:100700002F9DAA85B305B4401755FF1F1305855CBF
:10071000EF80400B41016F109F8982809757FF1F28
:1007200093874757D85331C7EF123F8603C7F70265
:1007300005079756FF1FA386E65811CD8C5F0D471E
:100740000145898185899756FF1F23A7E656EFF05B
:100750009FDB6F10DF8585479305C0441755FF1F4A
:10076000130545571757FF1F2328F754EF808005BF
:10077000CDB78280EF127F811757FF1F03472754A1
:100780008547631EF7009757FF1F9387A75083C7BE
:10079000870393C787001757FF1F2309F752175581
:1007A000FF1F13052553EF806003EF807FEF99470C
:1007B0001757FF1F2322F7509757FF1FA383075098
:1007C0009757FF1F238D074EEF90AF8F930740067B
:1007D0003305F5029757FF1F23A6A74E6F102FFD75
:1007E0009757FF1F83C7874EC18B99C7EF12EFF949
:1007F000EFF0FFAD6F10AFFB695582809757FF1F79
:1008000093874749DC5381CBEF122FF88545EFF0F2
:100810009FCF6F10CFF982801757FF1F13078747AD
:1008200001468146BA852148631E06019DCA239070
:10083000A60083C7850393E717001757FF1F2307F9
:10084000F74805A08357C705631DF502F85985478A
:10085000B397C70093C7F7FFF98F1757FF1F2325DB
:10086000F74A9C5D9183858B85C79757FF1F83C788
:10087000074599EFEF126FF11D45EFF0FFB06F10D4
:100880000FF381E699E39306C7050506090769BFDB
:100890008280EF120FED8605AA84B309B500975A3E
:1008A000FF1F938AEA45054B975BFF1F938B8B4590
:1008B000214C639434039757FF1F9387A73D9C5F98
:1008C0009183858B89CB9757FF1F83C7473F81E76C
:1008D0002145EFF07FAB6F104FEC03DA0400630BA0
:1008E0000A041759FF1F1309E93A0144CA8C8357B8
:1008F000C905639D4703A2855685EFF0BF9C11E5AE
:10090000A2855E85EFF01F9C05C903A74C07B317AE
:100910008B00D98F1757FF1F2328F73E83C78C03FF
:1009200093E717001757FF1F2302F73A0504090939
:10093000E31F84FB8904B5BF231E0904C5BF1757F5
:10094000FF1F0347C7378547631AF700EF12EFE32E
:10095000EFF05FE2EFF0BF976F106FE582808147A5
:1009600085451306000293861700B397F500E98FBB
:1009700013F7F60F89E7B687E397C6FE01473A8576
:100980008280FD4785457D56B396F5001387170095
:10099000E98E1377F70F89E6FD17E397C7FE014746
:1009A0003A85828089E901473A85828001473A8504
:1009B00041016F10CFDFEF124FDD41112AC62E85A6
:1009C0002EC4EFF0DFF9A2457D158547B397A70048
:1009D000E39EF5FC32469377360099C3719A11066F
:1009E0009757FF1F9387C72A94433E871758FF1FC7
:1009F0001308482989EA832708009107F19B975635
:100A0000FF1F23A7F628032588001843B307A70074
:100A1000B3F7B702B387F540FD15FD8D8327480076
:100A2000AA95B306B600E3F3F6F8E371D5F82E976E
:100A30009757FF1F23ACD7243DDB3A858145EF1044
:100A4000CFD72A87ADB718419757FF1F93878723C2
:100A500023A4070098C35841D8C39757FF1F23A961
:100A600007228280EF12CFD0AA8401441759FF1FBA
:100A7000130949229309400EEF807FD56345A400F6
:100A800001456F102FD2330534038327090B3E95A0
:100A90008357C501E38797FE0504F9BFEF126FCCBA
:100AA0009759FF1F9389091F3E84BA848347060024
:100AB00003A7090041119D83058B3D8F83C7440126
:100AC000AE8A2A89F99BD98F238AF4001C44B68503
:100AD000231204001CC02285328A36C6EF90DF8FB5
:100AE000B246D2853686EF90900BDC4883A509008C
:100AF0000840858B56869D8DEFD03FCC61E918402C
:100B00007D558347570003476700A207D98FC20767
:100B1000C1872394F4006358F00A83C7440193F714
:100B20000703B5CBD0489377160003A609001D8EA6
:100B30009757FF1F9387C74C9C43ADEB814641A05D
:100B400003A70B0093172A00BA97184094438347D2
:100B500057008345670033F65601A207CD8F631116
:100B6000F602834737000346470003472700A207E2
:100B7000D18F4207D98FBD82B3F76701638AF6042C
:100B8000050AEF80DFC3420593170A014181C18343
:100B9000E3E8A7FA41BFA16A370B0200014A975B5D
:100BA000FF1F938BEB1CFD1A7D1BE1BF83C7440124
:100BB00013070003854693F70703E391E7F8A2853F
:100BC0004A85EFD0FFCF41016F102FBD6155E5BFC2
:100BD0007955D5BFEF12CFB99754FF1F9384C4F353
:100BE0009C40D9EF9757FF1F938747099C43639910
:100BF000070CEF80DFBE930780023305F5028945BD
:100C0000EFF05FDA41C99757FF1F23ABA712EF80C0
:100C10001FBC9307400E3305F5029145EFF09FD8B6
:100C200035C99757FF1F23AFA710EF805FB201CDE3
:100C3000EF80FFB191450E05EFF0DFD621CD97573C
:100C4000FF1F23A3A710EF801FCB11CDEF80BFCADA
:100C5000D9473305F5028945EFF0DFD405CD975725
:100C6000FF1F23ADA70CEF809FB591450A05EFF05C
:100C70007FD30DC19757FF1F23ACA70E014521A8B5
:100C8000EF803FC2930780063305F5029145EFF0F0
:100C90007FD101E565556F10EFB09757FF1F23AB6C
:100CA000A7000144130A80061759FF1F130989FE84
:100CB000B14AEF801FBF6364A4029C40E38407F243
:100CC000EF803FBE9307A0043305F5028945EFF09E
:100CD0007FCD69D19757FF1F23A0A70A19BFEF80C7
:100CE0005FBB89450605EFF0FFCB4DD5B309440343
:100CF000032709024E9708CBEF80BFB83305550391
:100D00009145EFF03FCA59D58327090205041374B2
:100D1000F40FCE9788DB71BF9757FF1F938787F734
:100D2000884705898280C167FD176319F5009757C9
:100D3000FF1F938727F603A5070B8280EF12EFA40E
:100D4000EFF05FD26F10AFA6814709C58347E50179
:100D5000B337F0001757FF1F1307C7F3184709836E
:100D6000058B19C393E727003E858280EF12EFA120
:100D70002A84EFF07FFD8347E401AA8513059408D8
:100D800099E3130504039756FF1F9386A6F0944238
:100D9000130615021307840213059504EFD0CFC084
:100DA0006F10EFA0EF12CF9C9754FF1F938484EE37
:100DB00098442A892E840983058B9C4019C76314A3
:100DC000F5006380050E014401A2E3FEA7FE138730
:100DD000A702E36AA7FE850763FCA70883A9440B63
:100DE000EF80FF961316350081454E85EF10EF9C7E
:100DF0009757FF1F23A027EB9757FF1F23AE07E846
:100E000049CC9C4493E747001757FF1F2328F7E876
:100E10009757FF1F238C07EE630F040C9757FF1F94
:100E200023AA27E701440549EF807F926341A40A82
:100E3000EF80FF9493050006B3C5A502B7F736000F
:100E4000938707E81755FF1F130585EC4169014497
:100E50009309400E7D19B385F502EF70B016EF804F
:100E60001F97634FA4080145EF3040700544A9A8BF
:100E70006398A7029DE583A9440BEF805F8D13164D
:100E8000350081454E85EF104F939757FF1F23A3E1
:100E900027E19757FF1F23A107E09C44ED9BADB7C7
:100EA00085C51757FF1F034767E69307F005E3FC67
:100EB000E7F021F8EF60F03C6DD19C4493E7070226
:100EC0001757FF1F232CF7DC22856F10AF8D83A7E8
:100ED000440B131534003E958357050081CB83479F
:100EE000250099C721468145EF102F8D05042DBFA0
:100EF00023012501E5BF9757FF1F23AF07D80DBF7B
:100F00003305340383A7040B3E958357C5016384DF
:100F10002701EFF0BFE5050499B7EF120F87EF80C7
:100F20001F86130400063345A4029754FF1F9384C1
:100F300064D683C784073E951375F50F9757FF1F37
:100F40002386A7DC9307F00563E7A7020545EF308A
:100F5000E061EF80DF823345A402B7F53600938568
:100F600005E8B305B5021755FF1F130565DAEF70E5
:100F700070056F10CF839C4405458983858B81CB99
:100F8000EF904F8888408145EFF0DFE1DDB7EF302B
:100F9000E05DC5B7EF02DFFD130495082A8913064B
:100FA0009005A28513050503EF90603F1306900599
:100FB00081452285EF106F804A85EF30C05481440F
:100FC000175AFF1F130A0ACD930A8002EF803F8150
:100FD00063C4A4006F001FFD338454038327CA0A2F
:100FE0003E94035704008357C9016317F7028347F0
:100FF00044009DC3930964014546CE851305540002
:10100000EF90E039454681454E85EF001FFB228574
:1010100023020400EF30005785044DBFEF02FFF6B6
:101020009757FF1F938747AF9C432A8491C70DC5ED
:101030000355C501EFE00FC29757FF1F938747FC89
:101040009C4389CBEFB0DFD085476315F50022853F
:10105000EF50C05D6F00BFF541657D15E1BFEF0248
:10106000DFF21754FF1F1304E4C2444093871400B7
:101070001757FF1F2322F7C2EF30605E1C4489839D
:10108000858B9DE75840B7E7B0009387075063F121
:10109000E7020145EFF01F9D01CD0545EF809FF66A
:1010A000084085450505EFF0FFCF0145EFF01FF73C
:1010B00026856F00DFEFEF02BFEBA1642A890144B0
:1010C0009759FF1F9389C9CAFD14338AA500EF8081
:1010D0000FEF6344A4006F00FFEC03A70900931710
:1010E0002400BA979843658F42074183634C2701D8
:1010F000635A470123800700A3800700238107006C
:10110000A38107000504E1B7EF023FE583594500DD
:10111000C547411163F537310441C1E533853401D9
:10112000834785FF034795FF0348B5FFA207D98F83
:101130000347A5FFC207220733670701D98F03477B
:10114000C5FF0348D5FF2207336707010348E5FFC2
:101150000345F5FF420722083365A800498FB98F80
:101160001757FF1F130787BE1758FF1F130808C024
:101170003A85832807006384172B1107E31B07FFB9
:101180001757FF1F130787BE1843131827004295F0
:101190001CC10507A1473367F7029757FF1F23A715
:1011A000E7BC93F735001397470083474601C16BAF
:1011B000368993F7F7FCD98F32842E8A230AF600FA
:1011C000814A175CFF1F130CECACFD1B975CFF1FE3
:1011D000938C8C94175DFF1F130D0DBAEF802FDFDA
:1011E00063C7AA00E154268541016F00DFDA1308C6
:1011F000400EB3870A0303280C0BB30DF800638E6F
:101200000D2083D7CD01638A772183A70C00014B82
:10121000639707169757FF1F938747A69C436390D2
:10122000071683C7040003C70D0493F7F707631B72
:10123000F71ACA872287CE86268693859D06138550
:101240001D04EFF0BF85631F051883D7CD01032769
:1012500009002320B4012312F400FD572313F400E6
:101260008347170093F6F7078347D40093F707F8EF
:10127000D58FA306F40093F7F707B337F000B30751
:10128000F0402307F400834717009D8393963700AF
:1012900083474401DD9BD58F230AF4008347370041
:1012A00083464700A207D58F83462700C206D58F05
:1012B0001CC88347770003478700A207D98F2315EF
:1012C000F4000D476304EA00BD5491DF93870710D3
:1012D000C207C1831307B00FBD54E376F7F0EF8068
:1012E0000FC98144E31105F09756FF1F83C686A8F6
:1012F000938716001757FF1F230EF7A61757FF1FD8
:10130000130707A7231BD400939726001443035702
:101310008400E175BE96A1671386F7FFB377C70017
:1013200098426D8FD98F9CC21848F18F3E07D98F94
:101330009CC2EF80CFC89757FF1F83C7A7A333F581
:10134000A7029757FF1F2387A7A271BD9307A00489
:10135000B308FB0283270D00BE9803D7080083D78C
:10136000CD01631DF70083C7040003C7880093F70E
:10137000F707630BF70083C7FD019DEB050BEF80BB
:101380004FD2E345ABFC71BD93859801138598005E
:10139000CA872287CE86268646C6EFF02FF0B2484F
:1013A00079F98347440193E74700230AF40071BDAC
:1013B00083C7040003C7980293F7F707E310F7FC0D
:1013C000CA872287CE8626869385A8031385A8021E
:1013D000EFF0CFEC45F58347440193E72700230A5C
:1013E000F400C1B783C7FD018DCB83C7040003C7D9
:1013F0009D0993F7F7076312F702CA872287CE8603
:10140000268693852D0C1385AD09EFF02FE911E5A4
:101410008347440193E7270049BF850AC1B3FD54C0
:10142000D9B3EF021FB4797183544500AA8B2E847F
:10143000B28AEF80CFBB590563499504B7E4040035
:1014400003A90407EF80AFBA59054205418102990B
:101450002A8905CD2AC623180100EF804FB9590506
:101460002319A1006146814528089759FF1F9389D8
:1014700069824ACAEF007FB42302810203A4890073
:10148000058819E4BC544A85829745616F00FFB016
:1014900074003008D6855E85EFF01FC765F56800DB
:1014A000EF807FF1175AFF1F130A8AB583270A00BE
:1014B000AA84035B010189CB89476397FA008355AE
:1014C00001025E85EF50203003552102EF704FC8B6
:1014D00019E503552102EF708FD43334A000931720
:1014E00064000344C1022C0868001374F4FB5D8C93
:1014F00023068102EF60B056E9576314F502835664
:10150000E1029757FF1F9387A7869C4313972600F6
:101510006176BA979843718F98C39757FF1F238BB3
:10152000D784831721026345F00085476396FA004C
:10153000B25793F7070C95E7D247C2040347C1029D
:10154000C180BE9426C62318610113770703C147E3
:10155000631DF70083475102054793F7F707639030
:10156000E704B7E70400BC5739BF92570544A1838D
:1015700093F7F707E377F4FE15C78347C102130714
:10158000000293F707036397E700EFB06FFC85470E
:10159000E319F5FC8347C10293F7070389CFEFB046
:1015A000AFCA21A8EFB08FD7E30985FCEFB04FFA9F
:1015B000E31985FAD9B7EFB0EFD8AA8501460545FA
:1015C000EF707FF82A8451DD8347C102414793F7CA
:1015D00007036384E70232478347170093F707F84E
:1015E000A300F7003247925783461700A18393F771
:1015F000F707FD17D58FA300F70003560101B24589
:10160000130BC4005A85EF80DFDFE24A1306900512
:101610008347C10283C4EA01918BB384C40213855A
:101620001404569595C35444B3879A0083C707049E
:1016300003C70600137707F82380E6005844834663
:101640000700D58F2300F700B25703A60900814693
:10165000858B1D8EDA85EFD0EF9B15E9B25783A5F8
:101660000900484413869406858B56969D8DEFD0CD
:10167000CF9411ED83270A0099EFB2570547918364
:101680008D8B6387E7049DCF09476389E704228533
:10169000EF80DFF8F9B5EFB0AFEB85476309F500F0
:1016A0008347C102414793F70703E398E7FC83555B
:1016B00021025A85EF40907C69D183172102E35EB5
:1016C000F0FAF1B7EFB08FC57D151335150061D174
:1016D000014681452285EF70FFEF55BFEFB04FE720
:1016E000E5B7EF029F8A9744FF1F9384245C268509
:1016F000EF809FEB2A8419E16F007F8B1305C400F4
:1017000005468145EFF0FFD12285EF803FF1C5B757
:10171000EF02BF874111AE842A8493079503130714
:1017200015019306F10005466C002685230601008D
:10173000EFD0CFBE1DEDA68541462285EF80304615
:101740008347F1009305140226852308F400EFD0A7
:101750006FC805E19757FF1F9387878A9C4389EFDE
:101760001306940497C500009385850D2685EFD058
:101770008FD441016F00BF831306940297C5000008
:101780009385850C2685EFD00FD379D9DDB7EF028D
:101790002FFE9747FF1F9387A75D8043AE84B289D2
:1017A000368AAA8AEF80AF811316250081452285EB
:1017B000EF00BF809747FF1F238E075A9747FF1FF1
:1017C0009387474D03A4070B13F714003E89230F9B
:1017D000E400CE8525C713059408EFF07FF301C51B
:1017E00055556F002FFC8947A30FF4009757FF1F33
:1017F000938707819C4303278900858093B717004F
:1018000086072300F402231E54019747FF1F23A3DA
:10181000474985889377B7FF99C093674700174773
:10182000FF1F232DF7462285930700061747FF1F4A
:10183000230EF74CEFF08FD3014565B71305040372
:10184000EFF01FED45D569BFEF022FF4FD572310D0
:10185000F5002311050023120500231305001306CC
:10186000200481452105EF004FF56F004FF4EF0292
:101870002FF04111AA8401441749FF1F1309C94FD2
:101880009309A0042EC6EF80CF81B2456344A40023
:1018900061550DA033053403832709003E95835716
:1018A0002500639CB7008357050063989700EFF00D
:1018B000BFF9014541016F00EFEE0504E1B7EF020A
:1018C0002FEB9747FF1F9387673B9C434111AA84E7
:1018D0002E84B28903592500C1C39747FF1F83D7C0
:1018E000273E639B2707EF700F862A8903D52400C4
:1018F00093051002B305B40285472302F100935704
:101900008900A302F10093578500A303F10083D758
:1019100044002304A100254613D787002305F100C6
:1019200083D76400A304E1004E8513D78700A30585
:10193000E1002306F1001387950093879501A10527
:10194000B386B400A6974C00269723032101EFD05D
:10195000EF9C41016F000FE5EF60FFFE51BFEF020A
:101960002FE14111AA8401441749FF1F1309C940FF
:101970009309A0043AC636C432C22EC0EF707FF27B
:1019800082451246A24632476344A400615599A09D
:10199000B307340303250900AA9703D8070003D52A
:1019A000C4016310A80495E91DEE91CA03C6E401C1
:1019B000930510023306B60225063E9690C20145F5
:1019C00011CB83C6E40113061002B386C602E506F6
:1019D000B6971CC341016F00EFDC03D52700E30578
:1019E000B5FC050441BF83C5E40113051002B385AE
:1019F000A502BE9583C585002300B6007DB7EF0222
:101A00002FD75C4141112A8403DA2700C167FD17F3
:101A1000AE843289630CFA002685EF807F9A8D4769
:101A200063EDA7007D5541016F00CFD72E85EF8074
:101A30003F999D47E3E2A7FEF5B75C40268583D535
:101A40004700EF809F90835584002685EF80FF8FAD
:101A50008D452685EF803F8EAA89EFF04FE09357A2
:101A600005012380F90093578500A380F9002381A5
:101A7000A9005840C167FD178345A7006314FA0009
:101A800093E505082685EF801F8F9747FF1F9387F3
:101A9000E71E9C430840D9CF8347B400858BD9CB40
:101AA00078003400130671008145EFF05FEB1DC92B
:101AB0008347B400184093069005F99BA305F400F2
:101AC0008347E701B387D702B306F70083C606044E
:101AD000A303D1009386170493879706BA96BA9703
:101AE00036C43EC61744FF1F1304C41A1C440C40DE
:101AF00026858983858B9D8D834771009E05DD8DAD
:101B000093F5F50FEF803F871C44104022458983F1
:101B1000858BCA861D8EA685EFC0DFCFE31505F045
:101B20001C440C40324689838840858B9D8DEFC0D4
:101B3000DFC8D5BD8347B40013079005F99BA30503
:101B4000F4008347E501B387E7023307F500034755
:101B50000704A303E10013871704938797062A97C6
:101B60003E953AC42AC6BDBFEF028FC0032A450086
:101B70009307F00FAA840347AA00AE8932843689FE
:101B80006316F700EFB06FAB2305AA00938AC90074
:101B90000146D6852685EFF09FE62A8A21E517477C
:101BA000FF1F1307E7451843DC4039C383C6A7006E
:101BB0000547638FE60283D547005685EF40102C1A
:101BC00005C9DC40839747006354F00201CC1C40F8
:101BD00089C74A868145014582975C4081C7CA858D
:101BE000014582974E85EF807FA352856F008FBBA2
:101BF000DC4003D54700EF60BFD501E9DC4003D5E9
:101C00004700EF60DFE181471DCD19C41C4089C743
:101C10004A868145014582974E85EF807F9FAA8540
:101C20001745FF1F13058508EF80DF9511C45C4041
:101C300081C7CA85014582971745FF1F13054506D1
:101C4000EF60F0368547D84085460346A700E30B92
:101C5000D6F8031747006353E000C9F74A86A28508
:101C60004E85EF703F97BDBFEF028FB0AA8401444D
:101C70001749FF1F130949109309A004130A950877
:101C8000EF703FC26344A400014535A0330534031F
:101C9000832709003E958357250099E30504CDB7B6
:101CA0000357050083D7C401E31AF7FE5286854522
:101CB000EFF0FFC065D56F00EFAEEF026FABAA8407
:101CC00001441749FF1F1309290B9309A004EF7062
:101CD0005FBD6344A4006F00EFAC3305340383277A
:101CE00009003E958357250081CF835705006399EE
:101CF000970093059502130610022105EF80206AD4
:101D00000504F1B7EF026FA80347E5012A84834772
:101D1000F5016307B70089E781452E856F002FA97C
:101D2000230FB400054781C9E398E7FE8947A30F55
:101D3000F4008545DDB7638BE7020947E39FE7FCC5
:101D40002285EFF02FA59747FF1F938727F39C432A
:101D500099E79747FF1F938727DC9C4389C7035563
:101D6000C401EFF09FF5A30F0400E1B755D6C9BF3A
:101D7000EF020FA0EFA0FFEE85476312F508EF809A
:101D8000EFCC1744FF1F1304A4271C4081CBEFA006
:101D90003FFC89476304F5001C4082979747FF1F6B
:101DA0009387C7ED9C43B9CF82979747FF1F9387CF
:101DB000A7D69C4391C382971744FF1F130484ED59
:101DC0008327040B83D4C701EF60FFB78327040B7D
:101DD000AA85144003C6E7011C448983858B99C3F7
:101DE0001366260026854169EF40C03D8144D949EC
:101DF0007D19EF705FB063CAA4006F00AF9AEF80E7
:101E00000FCA41B7EF705F884DB7B387340303271C
:101E1000840ABA9703D527006308250103C6470142
:101E200083D50700EF40A03B8504E1B7EF024F9454
:101E300001449744FF1F9384E4E51309400EFD59C4
:101E4000EF70FF98634FA40401449744FF1F9384ED
:101E500064E413098002FD59EF707F98634CA40479
:101E600001449744FF1F9384E4E25949FD59EF7000
:101E70009FA8634AA40497F5FFFF9385450A174579
:101E8000FF1F1305E5E8EF60D00797050000938575
:101E900085851745FF1F1305A5E0EF6050056F000E
:101EA0006F903307240383A7040B0504BA97239E7E
:101EB000370179B73307240383A7C40A0504BA9707
:101EC0002390370151BF3307240383A7840A0504F5
:101ED000BA972391370161BFD44103873500854705
:101EE0003356F5026377E600A54899E7238006009C
:101EF0008280B387E702EDB73358F50203873500D8
:101F00003375F502B3D7E7021307000363DA08015C
:101F100003C6050013077003118A19E21307700541
:101F200085064297A38FE6FEC9B718451C41637624
:101F3000F7005C41BA972380B7001C4585071CC594
:101F40008280EF028F844111AA872E85B285368662
:101F500036C6829763480500B246158D3335A0001A
:101F60003305A04041016F008F84EF026F80056947
:101F700041112A8A2320060001448149974AFF1F04
:101F8000938A0AE2056B7D1932C62EC4EF703F8535
:101F9000AA84EF70DF832695A24532466346A400EB
:101FA0004E8541016F000F8003A70A0093171400AC
:101FB000BA9703D707003377670101E71CC205040E
:101FC000E1B703D707009356D700858AE39946FF08
:101FD00033772701E315B7FEBE89D5B7EFF2FEFAD6
:101FE00001112EC6B2843689EFB02FEE2A846155D6
:101FF00001C8B24589E9232E0400232004020145CB
:1020000005616FF0DEFAA1463008CA852685EFF03B
:102010005FF37DF5835781010357A101231EF4006F
:102020008357C1012310E4022311F4028357E10115
:10203000D207D1832312F4028357E10113973701AA
:1020400063560700FD57231FF4005DBF231F0400E4
:1020500045BFEFF2FEF11744FF1F1304A4C383270B
:10206000040B03D7C701C167FD17630EF71097472D
:10207000FF1F938727F99C4381C70545EF40607791
:10208000C1690149930A400EFD19174BFF1F130B3D
:102090002BF7EF70CFF3634BA90E1747FF1F0347D2
:1020A000E7C69307F00563E4E702EF704FED930591
:1020B0000006B3C5A502B7F73600938707E81745B2
:1020C000FF1F1305E5C4B385F502EF60A06F8145DE
:1020D0001705000013058520EF60DFF8EFB0EFDE95
:1020E00001CD0357C50109CB0357E50111C783474C
:1020F000050299C3EF60A06BEFB06FDE31C51747E3
:10210000FF1F034767CD9747FF1F9387E7CC0DCF8E
:1021100003C717002304E50003C72700A304E50055
:1021200003C737002305E50003C74700A305E50003
:1021300003C757002306E50003C7670083C777007E
:10214000A306E5002307F5001C4493E71700174793
:10215000FF1F2325F7B45C4085E7EF708FEF0DC1BB
:10216000EF702FEF44402A89EF70AFEE33F5A402F1
:102170005C40FD17CA97898F1747FF1F232EF7B0C2
:102180000145EF70DF9F01456FF0DEE1B3045903B5
:102190008327040BBE9483D7C40163883703138A53
:1021A0000403D2855285EFF0AFD605E183C7F40171
:1021B00099CF938594082E85EFF08FD509C9130622
:1021C000900581455285EFF05EDF0509D9B583277B
:1021D0000B00268593B7170086072380F402EFE0F3
:1021E000FFB8E5B7854763F8A7009307F5FFBE95ED
:1021F0003305A040E98D2E8582809841C167BA974A
:1022000013D707016304A7009CC182804207998FFE
:10221000E5BFEFF29ED741112EC63284B684EFB0EF
:102220000FCCE15701C9B24591E99747FF1F2385BC
:1022300007BA81473E8541016FF07ED79D4617461C
:10224000FF1F130676B9A6852285EFF09FCFAA87D8
:1022500075F105479746FF1F2380E6B8E1BFEFF20F
:102260003ED1411191E99747FF1F23A707A20144DF
:10227000228541016FF01ED3B68532858D467000F0
:10228000EFF03FCC2A846DF58347D1000347E1008E
:102290001749FF1F130909A0A2074207D98F034757
:1022A000C100D98F1747FF1F2328F79EEF706FDA01
:1022B00061D1EF700FDA83244900AA89EF706FD9DA
:1022C00033F5A40283274900FD17CE97898F17475E
:1022D000FF1F2323F79C69BFEFF23ECB1C45AA8466
:1022E00091CFD84B01CF83D7470089CBEF601F92A6
:1022F000AA8509C588446105EF60C04C9747FF1F58
:102300009387C7979C43014489EF6FF05ECA9C484E
:1023100013171400BA9703D5070019C1EFE0CFCF08
:102320000504EF70CFC7E344A4FEC5B7EFF2FEC5C6
:10233000011185E9EF605FDA01449747FF1F23A78A
:10234000079E9747FF1F23A5079E9747FF1F23A3BD
:10235000079E9747FF1F23A1079E228505616FF007
:102360001EC5B6873285C9467000BE85EFF07FBDB9
:102370002A8465F541469305E1001745FF1F1305C3
:10238000E59AEF80C0010355C100EF608FD7F1B728
:102390008DE19747FF1F23AF078E9747FF1F938756
:1023A000678F9C470145ED9B1747FF1F2328F78E3A
:1023B0008280EFF29EBD4111B68532859546300090
:1023C000EFF03FB815EDA2471747FF1F2324F78C06
:1023D0009747FF1F9387078C9447B24713F7B6FFC1
:1023E00013F6170019C213E74600858393F7F70722
:1023F0009746FF1F23A4E68A1747FF1F2308F7907D
:1024000041016FF0DEBAEFF2BEB603841500DC4185
:102410002A89AE8485070387F7FF19C36340800CC0
:102420008387240091C7635580007D146204618412
:102430009C40370700FF0907F98F3707001009078D
:102440006392E70A6355800079146204618483C74C
:102450000400858B95E39379F40F4E8A93178A01D4
:10246000E187634AF008A2876353040081473384FD
:10247000F9407D14620461848385240081C54A8506
:10248000EFF0BFAA9C40370700FF0907F98F370715
:1024900000100907639AE706930500034A85EFF0E9
:1024A000DFA883C7040093058005918B99E393050A
:1024B00080074A85EFF07FA783C70400858B81CB17
:1024C0001374F40F93178401E1876347F004C0404D
:1024D00005048305F4FFA1E96FF0DEAC7D1462040E
:1024E00061840DBF370700080907E392E7F6E35060
:1024F00080F67D1499BF930500024A857D1AEFF09E
:10250000DFA2137AFA0F99BF370700080907E3958E
:10251000E7FA9305000371BF930500034A85EFF0C6
:10252000DFA07D1471BF4A85EFF03FA055B7EFF2F1
:10253000DEA5EF70CFAA2A84EF706FA92295894596
:102540000605EFE02FC6E55711C59747FF1F23A9E2
:10255000A78481473E856FF09EA59307000263061E
:10256000F5005D1513355500828005458280EFF238
:102570003EA04111AA892A89130419008304F4FF9B
:1025800032C62EC42685EFF05FFDA245324659E1E2
:102590009307D0026392F4088304040005481304EF
:1025A00029009377F6FEC9E793070003639FF40EB3
:1025B000830704001307800593F7F7FD6399E70687
:1025C0008304140041460904B70600806314080020
:1025D00093C6F6FFB3FEC6028147254F654EFD5FE9
:1025E00033D3C602138704FD6368EF06BA8463D54C
:1025F000C408630DF5017D55636AF30063946700B9
:1026000063C69E000545B307F602A697050483043A
:10261000F4FFC9BF22898DB79307B0020148E39246
:10262000F4F8830404002A88130429009DBF01CA1A
:102630008947E31BF6F893070003E397F4F8830751
:1026400004001307200493F7F7FD639BE70483045A
:102650001400094609048DBF13E704021307F7F9B4
:10266000636CEE009388F4FB1307700363741E0120
:1026700013077005998CA5BF7D576300E5026304BD
:102680000800B307F04091C519C19309F4FF23A0D6
:1026900035013E8541016FF0FE90B687FDF5D5BF4F
:1026A0009304000315F2214605B719FE294629BFF8
:1026B000EFF21E8C011161540DC53284AE89414682
:1026C00081453689EFF0BFEA93140501C180639E0E
:1026D00009002685EF30102B014401C58145EF200C
:1026E0005016228505616FF0FE8B2285CD46700065
:1026F000CA85EFF01F852A846DF52685EF30902876
:1027000009E90356C1008345E1012685EF20500BFE
:1027100001C941469305E1001105EF705048D1B75A
:102720005D54C1B7EFF2DE840111E15401CDB284F2
:10273000AE89414681453689EFF07FE32A8463976D
:1027400009008144268505616FF0DE852685D14626
:102750007000CA85EFF0EFFEAA846DF58357C100C3
:10276000EDD3EF700F8E4205931704014181C183B1
:1027700063F9A702EFB08FB64204E147418033040A
:10278000F40241460C082A9413054400EF703041CE
:102790008357E1002311F4008357C1002310F40094
:1027A00055B7E55445B7EFF2AEFC7971E15415C564
:1027B0003284AE8941468145B684EFF05FDB131960
:1027C000050113590901639E09004A85EF40106510
:1027D000814401C58145EFB02FB1268545616FF079
:1027E0006EFCA6859306300270002285EFF06FF52F
:1027F000AA8465F54A85EF4070622A8411E54A850E
:10280000EFB04F8C2A8431C58357C10023112401B6
:10281000930964002310F4008347E1009305F1005D
:1028200041462302F4004E85EF707037130974019E
:1028300041469305F1014A85EF70703693055400C7
:102840004E85EFC04FBF930564014A85EFC0AFBE10
:1028500069B7DD5459B7EFF2AEF1797111E5E15482
:10286000268545616FF00EF4B284AE8941468145FC
:102870003689EFF0DFCF131A0501135A0A0152858A
:10288000EFE06FCA2A846398090071D98145EFB0DF
:102890002FB48144F1B72685930610027000CA85D3
:1028A000EFF02FEAAA844DFD31C8B2479305D1005D
:1028B0004146858B230FF400B2471305040385833B
:1028C00093F7F707A30FF400EF70702D41469305BF
:1028D000D10113059408EF70902C59B733046903A4
:1028E00083A70A0B3E948357C4016383370305090A
:1028F000EF60FFEDE344A9FEDD549DB7C1690149D6
:10290000973AFF1F938A0A39130B400EFD19CDB772
:10291000231E440159BF49CDEFF28EE54111B28922
:10292000AE8441468145368AEFF07FC4931A050193
:1029300093DA0A010149173BFF1F130BAB35EF6018
:102940001FE1634AA9000145ADCC81441739FF1F3F
:102950001309493481A883274B0B131439003E9483
:1029600083570400638857050509D1BF8327490BA6
:10297000139434003E948357040085E723105401D8
:1029800091467000D2854E85EFF0AFDB1DE9B2476E
:1029900013978700E1832183858B58C02301F400BE
:1029A0000DA08504EF60BFDAE3C2A4FC5D5511A859
:1029B00061558280F1F4214681452285EFF0EEDFFA
:1029C000014541016FF00EDE1971D2C4130AC10630
:1029D00086CEA2CCA6CACAC8CEC6D6C2B6D6BAD8E9
:1029E000BEDAC2DCC6DE52C463810524FD151C10AC
:1029F0002ACC2ECA02CE3EC89304B0021549A9497A
:102A000083050600130416009DE1F2465247E24793
:102A100063FBE620B697238007007245F6406644C4
:102A2000D6444649B649264A964A096182809307A8
:102A300050026386F5004808EFF02FCFF5A88357C2
:102A4000C10023070100014593F7C70F2316F100CA
:102A5000814501480147014681469308D00213038E
:102A60000003130E300205048307F4FF99C7638C3B
:102A7000970463C3F404638BC70501CA0346C1000E
:102A8000858A799AD18E2306D1006309080083468E
:102A9000C100098BF59A558F2306E10019C1230760
:102AA000B100138707FD1377F70FA54663E2E6062B
:102AB0008146A545294535A0E38717FBE39F67FAC3
:102AC0000546FD564DB70545854571BF05487D57FF
:102AD00059BFB386A60205048307F4FFBA96E2063F
:102AE000E18613F7F70F130607FD1376F60F63E57C
:102AF000C500138707FDF1BF1306F7F91376F60F2C
:102B0000636EC902138797FAE30537FDA306D10068
:102B1000130790066385E704634BF70613078005E8
:102B20006384E70A6345F702E38107EE1307500267
:102B300093055002E381E7F02286D9B51307F7FB2E
:102B40001377F70FE364E9FC138797FC75BF13074E
:102B500030066386E70A13074006E39FE7FC032578
:102B60000A00A947A307F100930A4A006358050029
:102B70009307D0023305A0402307F1006C00EFF06B
:102B8000AFB56C004808EFF01F88568A75B7130779
:102B90003007638EE7066341F7021307F006638E82
:102BA000E70413070007E399E7F80347C100136739
:102BB00027002306E10009A813075007638BE702EB
:102BC00013078007E39AE7F6938787FA414793B79D
:102BD0001700A307E100139727008347C100ED9B6F
:102BE000D98F2306F100930A4A006C0003250A00DE
:102BF00079B7A947A307F100FDB7A147E5BF830552
